:020000040800F2
:1080000000000120E94601089D4501089F4501083F
:10801000A1450108A3450108A5450108000000008D
:10802000000000000000000000000000A74501085B
:10803000A945010800000000AB450108AD45010855
:10804000314701083147010831470108314701082C
:10805000314701083147010831470108314701081C
:10806000314701083147010831470108B14501088E
:108070003147010831470108BD450108C9450108DC
:1080800031470108D5450108E1450108314701089C
:1080900031470108314701083147010831470108DC
:1080A00031470108314701083147010831470108CC
:1080B000ED45010831470108314701083147010802
:1080C00031470108314701083147010831470108AC
:1080D00031470108F9450108054601083147010803
:1080E000314701083147010831470108314701088C
:1080F000314701083147010831470108114601089D
:10810000314701083147010831470108314701086B
:1081100031470108314701081D4601083147010870
:108120003147010831470108314701082946010854
:10813000000000000000000000000000000000003F
:10814000000000000000000000000000000000002F
:10815000000000000000000000000000000000001F
:10816000000000000000000000000000000000000F
:1081700000000000000000000000000000000000FF
:1081800000000000000000000000000000000000EF
:1081900000000000000000000000000000000000DF
:1081A00000000000000000000000000000000000CF
:1081B00000000000000000000000000000000000BF
:1081C00000000000000000000000000000000000AF
:1081D000000000000000000000000000000000009F
:0481E0005FF8E0F173
:1081E80010B5054C237833B9044B13B10448AFF3E9
:1081F80000800123237010BD3829002000000000F2
:108208009058010808B5034B1BB103490348AFF365
:10821800008008BD000000003C290020905801089B
:10822800D0400B1CD1409C46203AD34018435242C0
:10823800634693401843704781F0004102E000BF55
:1082480083F0004330B54FEA41044FEA430594EA0E
:10825800050F08BF90EA020F1FBF54EA000C55EA49
:10826800020C7FEA645C7FEA655C00F0E2804FEA1A
:108278005454D4EB5555B8BF6D420CDD2C4480EAFC
:10828800020281EA030382EA000083EA010180EA2C
:10829800020281EA0303362D88BF30BD11F0004F7A
:1082A8004FEA01314FF4801C4CEA113102D04042B0
:1082B80061EB410113F0004F4FEA03334CEA1333EB
:1082C80002D0524263EB430394EA050F00F0A78003
:1082D800A4F10104D5F1200E0DDB02FA0EFC22FAFE
:1082E80005F2801841F1000103FA0EF2801843FAF2
:1082F80005F359410EE0A5F120050EF1200E012AE3
:1083080003FA0EFC28BF4CF0020C43FA05F3C01820
:1083180051EBE37101F0004507D54FF0000EDCF199
:10832800000C7EEB00006EEB0101B1F5801F1BD342
:10833800B1F5001F0CD349085FEA30004FEA3C0C46
:1083480004F101044FEA445212F5800F80F09A803C
:10835800BCF1004F08BF5FEA500C50F1000041EB40
:10836800045141EA050130BD5FEA4C0C404141EB44
:10837800010111F4801FA4F10104E9D191F0000F6B
:1083880004BF01460020B1FA81F308BF2033A3F1EE
:108398000B03B3F120020CDA0C3208DD02F1140CE5
:1083A800C2F10C0201FA0CF021FA02F10CE002F120
:1083B8001402D8BFC2F1200C01FA02F120FA0CFC19
:1083C800DCBF41EA0C019040E41AA2BF01EB045162
:1083D800294330BD6FEA04041F3C1CDA0C340EDC60
:1083E80004F11404C4F1200220FA04F001FA02F3A3
:1083F80040EA030021FA04F345EA030130BDC4F161
:108408000C04C4F1200220FA02F001FA04F340EA55
:108418000300294630BD21FA04F0294630BD94F006
:10842800000F83F4801306BF81F480110134013DED
:108438004EE77FEA645C18BF7FEA655C29D094EA5E
:10844800050F08BF90EA020F05D054EA000C04BFDC
:108458001946104630BD91EA030F1EBF00210020C7
:1084680030BD5FEA545C05D14000494128BF41F066
:10847800004130BD14F580043CBF01F5801130BDCA
:1084880001F0004545F0FE4141F470014FF0000055
:1084980030BD7FEA645C1ABF194610467FEA655C06
:1084A8001CBF0B46024650EA013406BF52EA0335A8
:1084B80091EA030F41F4002130BD00BF90F0000F96
:1084C80004BF0021704730B54FF4806404F13204D2
:1084D8004FF000054FF0000150E700BF90F0000F8B
:1084E80004BF0021704730B54FF4806404F13204B2
:1084F80010F0004548BF40424FF000013EE700BF82
:1085080042004FEAE2014FEA31014FEA02701FBF11
:1085180012F07F4393F07F4F81F06051704792F0E3
:10852800000F14BF93F07F4F704730B54FF460745D
:1085380001F0004521F0004120E700BF50EA0102A8
:1085480008BF704730B54FF000050AE050EA010255
:1085580008BF704730B511F0004502D5404261EBC5
:1085680041014FF4806404F132045FEA915C3FF406
:10857800DCAE4FF003025FEADC0C18BF03325FEA9F
:10858800DC0C18BF033202EBDC02C2F1200300FA54
:1085980003FC20FA02F001FA03FE40EA0E0021FA79
:1085A80002F11444C1E600BF70B54FF0FF0C4CF463
:1085B800E06C1CEA11541DBF1CEA135594EA0C0F19
:1085C80095EA0C0F00F0DEF82C4481EA030621EA54
:1085D8004C5123EA4C5350EA013518BF52EA03358F
:1085E80041F4801143F4801338D0A0FB02CE4FF041
:1085F8000005E1FB02E506F00042E0FB03E54FF071
:108608000006E1FB03569CF0000F18BF4EF0010E68
:10861800A4F1FF04B6F5007F64F5407404D25FEA64
:108628004E0E6D4146EB060642EAC62141EA555117
:108638004FEAC52040EA5E504FEACE2EB4F1FD0C59
:1086480088BFBCF5E06F1ED8BEF1004F08BF5FEAD7
:10865800500E50F1000041EB045170BD06F0004689
:1086680046EA010140EA020081EA0301B4EB5C0436
:10867800C2BFD4EB0C0541EA045170BD41F480112E
:108688004FF0000E013C00F3AB8014F1360FDEBF53
:10869800002001F0004170BDC4F10004203C35DA2F
:1086A8000C341BDC04F11404C4F1200500FA05F3B2
:1086B80020FA04F001FA05F240EA020001F0004253
:1086C80021F0004110EBD37021FA04F642EB0601C9
:1086D8005EEA430E08BF20EAD37070BDC4F10C04F3
:1086E800C4F1200500FA04F320FA05F001FA04F2B7
:1086F80040EA020001F0004110EBD37041F10001A3
:108708005EEA430E08BF20EAD37070BDC4F12005AD
:1087180000FA05F24EEA020E20FA04F301FA05F215
:1087280043EA020321FA04F001F0004121FA04F2BD
:1087380020EA020000EBD3705EEA430E08BF20EA8D
:10874800D37070BD94F0000F0FD101F000464000C7
:1087580041EB010111F4801F08BF013CF7D041EA49
:10876800060195F0000F18BF704703F0004652004D
:1087780043EB030313F4801F08BF013DF7D043EA1E
:108788000603704794EA0C0F0CEA135518BF95EAD4
:108798000C0F0CD050EA410618BF52EA4306D1D15B
:1087A80081EA030101F000414FF0000070BD50EA7A
:1087B800410606BF1046194652EA430619D094EA04
:1087C8000C0F02D150EA013613D195EA0C0F05D1EE
:1087D80052EA03361CBF104619460AD181EA030142
:1087E80001F0004141F0FE4141F470014FF00000FA
:1087F80070BD41F0FE4141F4780170BD70B54FF095
:10880800FF0C4CF4E06C1CEA11541DBF1CEA135514
:1088180094EA0C0F95EA0C0F00F0A7F8A4EB0504F6
:1088280081EA030E52EA03354FEA013100F08880ED
:108838004FEA03334FF0805545EA131343EA1263B6
:108848004FEA022245EA111545EA10654FEA00266B
:108858000EF000419D4208BF964244F1FD0404F524
:10886800407402D25B084FEA3202B61A65EB030580
:108878005B084FEA32024FF480104FF4002CB6EB3D
:10888800020E75EB030E22BFB61A754640EA0C00BD
:108898005B084FEA3202B6EB020E75EB030E22BFFD
:1088A800B61A754640EA5C005B084FEA3202B6EB3E
:1088B800020E75EB030E22BFB61A754640EA9C00FD
:1088C8005B084FEA3202B6EB020E75EB030E22BFCD
:1088D800B61A754640EADC0055EA060E18D04FEA8B
:1088E800051545EA16754FEA06164FEAC30343EA2B
:1088F80052734FEAC2025FEA1C1CC0D111F4801FF8
:108908000BD141EA00014FF000004FF0004CB6E7F0
:1089180011F4801F04BF01430020B4F1FD0C88BF8F
:10892800BCF5E06F3FF6AFAEB5EB030C04BFB6EB9A
:10893800020C5FEA500C50F1000041EB045170BD8D
:108948000EF0004E4EEA113114EB5C04C2BFD4EBBA
:108958000C0541EA045170BD41F480114FF0000E3E
:10896800013C90E645EA060E8DE60CEA135594EABA
:108978000C0F08BF95EA0C0F3FF43BAF94EA0C0FBD
:108988000AD150EA01347FF434AF95EA0C0F7FF432
:1089980025AF104619462CE795EA0C0F06D152EA86
:1089A80003353FF4FDAE1046194622E750EA41066A
:1089B80018BF52EA43067FF4C5AE50EA41047FF47B
:1089C8000DAF52EA43057FF4EBAE12E74FF0FF3CE0
:1089D80006E000BF4FF0010C02E000BF4FF0010CB1
:1089E8004DF804CD4FEA410C7FEA6C5C4FEA430C2A
:1089F80018BF7FEA6C5C1BD001B050EA410C0CBF79
:108A080052EA430C91EA030F02BF90EA020F0020DA
:108A1800704710F1000F91EA030F58BF994208BF41
:108A280090422CBFD8176FEAE37040F001007047FE
:108A38004FEA410C7FEA6C5C02D150EA013C07D155
:108A48004FEA430C7FEA6C5CD6D152EA033CD3D0A0
:108A58005DF8040B704700BF8446104662468C469A
:108A68001946634600E000BF01B5FFF7B7FF0028CD
:108A780048BF10F1000F01BD4DF808EDFFF7F4FFF6
:108A88000CBF012000205DF808FB00BF4DF808ED81
:108A9800FFF7EAFF34BF012000205DF808FB00BFA4
:108AA8004DF808EDFFF7E0FF94BF012000205DF8C6
:108AB80008FB00BF4DF808EDFFF7CEFF94BF01207B
:108AC80000205DF808FB00BF4DF808EDFFF7C4FF74
:108AD80034BF012000205DF808FB00BF4FEA4102C7
:108AE80012F5001215D211D56FF47873B3EB6252F8
:108AF80012D94FEAC12343F0004343EA505311F01F
:108B0800004F23FA02F018BF404270474FF00000B0
:108B1800704750EA013005D111F0004008BF6FF0EE
:108B2800004070474FF00000704700BF4A0011D264
:108B380012F5001211D20DD56FF47873B3EB6252AF
:108B48000ED44FEAC12343F0004343EA505323FABB
:108B580002F070474FF00000704750EA013002D130
:108B68004FF0FF3070474FF000007047BFF34F8F52
:108B78000549064BCA6802F4E0621343CB60BFF3B1
:108B88004F8F00BFFDE700BF00ED00E00400FA05CD
:108B98000278437810B543EA02230C784A7842EA0F
:108BA80004229A421EBF04704B78437010BD000027
:108BB80010B50A4C00224FF40041094808F0D2FFD2
:108BC800204601224FF4804108F0CCFF2046BDE842
:108BD800104001224FF4004108F0C4BF00140140C6
:108BE8000010014070B52A4D2A4E95F8CB30CBB90C
:108BF8003368B3F5FA7F3CD94FF40041264808F0B2
:108C0800B6FF4FF48041254808F0B1FF244B1A788D
:108C180002B101224FF40041204808F0A3FF0023CD
:108C2800336070BD3368B3F5FA7F22D91D4C2278C2
:108C380012F001021ED001224FF40041164808F03C
:108C480091FF00224FF40041144808F08BFF0022E6
:108C58004FF48041114808F085FF23780133DBB2D7
:108C68002370002333602278052A84BF85F8CB302F
:108C7800237070BD4FF40041074808F073FF0122CC
:108C88004FF40041054808F06DFF0122E0E700BFFE
:108C9800CF3800204C300020001001400014014063
:108CA80022330020C22A00202DE9F041054616464D
:108CB80008461F462C469DF81880631B984501DC22
:108CC800BDE8F08104F8010BFFF708FC32463B468B
:108CD800FFF7B8FAFFF702FF40B2EEE773B50024DA
:108CE800314B324D324E93F99E1093F89F30224605
:108CF800009330462B46FFF7D7FF2E4B224693F9B9
:108D08009E1093F89F3006F1460000932B46FFF71C
:108D1800CBFF294B224693F99E1093F89F3006F11A
:108D28008C0000932B46FFF7BFFF244B224693F994
:108D38009E1093F89F3006F1D20000932B46FFF760
:108D4800B3FF1F4B1F4E93F99E1093F89F30224696
:108D5800009330462B46FFF7A7FF1B4B224693F99B
:108D68009E1093F89F3006F1460000932B46FFF7BC
:108D78009BFF164B224693F99E1093F89F3006F1FD
:108D88008C0000932B46FFF78FFF114B224693F977
:108D98009E1093F89F3006F1D20000932B46FFF700
:108DA80083FF02B070BD00BF1A4C00200000F0BF66
:108DB80043330020EF3B0020FF35002082320020A3
:108DC800FA4A0020DF4C00209F340020B9310020EF
:108DD800EF490020002310B5934200DB10BDCC5CA6
:108DE800C4540133F8E700002DE9F04705469046E2
:108DF8009946002400260027C0B042464B4630461C
:108E0800394604F1010AFFF741FEB0B9602229464C
:108E18006846E4B2FFF7DEFF1DF90400FFF75EFBCA
:108E280000220B4BFFF7C0FB02460B464046494663
:108E3800FFF708FA40B0BDE8F0873046394600220F
:108E4800034BFFF7FFF9544606460F46D5E700BF28
:108E58000000E03FF8B5064608461746FFF73EFB18
:108E68000022124BFFF7CAFC0546384601F10044C0
:108E7800FFF734FB00220023FFF7E4F900220B4B35
:108E8800FFF7BCFC02460B4628462146FFF7D8F9F7
:108E98000022074BFFF7D6F902460B463046FFF78C
:108EA800A3FFBDE8F84006F059BF00BF000024400A
:108EB800000014402DE9F84F1D46CB18C833BCBF3D
:108EC8006FF063052946834608461646FFF706FBFA
:108ED80000221E4BFFF792FC824630460C46FFF7F5
:108EE800FDFA00220023FFF7ADF9064628460F4693
:108EF800FFF7F4FA00220023FFF7A4F900228046C6
:108F08008946124B30463946FFF778FC04F1004495
:108F180002460B4650462146FFF792F900220446C6
:108F28000D460A4B40464946FFF768FC02460B4689
:108F380020462946FFF784F902460B465846FFF7B4
:108F480053FFBDE8F84F06F009BF00BF00002440FA
:108F5800F0B5A24CA24D237C94F84500617C94F8AE
:108F68004620697485F8462041EA032142EA002236
:108F780085B085F8450012B209B29A482B74FFF7FC
:108F880069FF994E029006F1100393E803008DE8FB
:108F9800030096E80F0006F023FFA37C94F847002F
:108FA800E17C94F84820E97485F8482041EA0321D7
:108FB80042EA002285F8470012B209B28B48AB7426
:108FC800FFF748FF06F14803029093E803008DE895
:108FD800030006F138030FCB06F002FF237D94F857
:108FE8004900617D94F84A20697585F84A2041EA6C
:108FF800032142EA002285F8490012B209B27C48EE
:109008002B75FFF727FF06F18003029093E8030012
:109018008DE8030006F170030FCB06F0E1FEA37D97
:1090280094F84B00E17D94F84C20E97585F84C20C4
:1090380041EA032142EA002285F84B0012B209B244
:109048006C48AB75FFF706FF06F1B803029093E88A
:1090580003008DE8030006F1A8030FCB06F0C0FE5D
:1090680094F8283194F84D7085F8283194F829310E
:1090780094F84E20207E94F82EE1617E85F82931FF
:1090880094F82F3185F84D7085F84E2042EA072272
:10909800594F43EA0E23697641EA002128761BB22C
:1090A80012B209B23846FFF705FF06F12C03029009
:1090B80093E803008DE8030006F11C030FCB06F0CC
:1090C8008FFE94F82A3194F84FE085F82A3194F805
:1090D8002B31A07E85F82B310023E17E94F85020B7
:1090E800E97685F8502041EA002142EA0E22A87666
:1090F80012B209B2384685F84FE084F82A3184F86C
:109108002B31FFF7D7FE06F16403029093E80300C2
:109118008DE8030006F154030FCB06F061FE94F8C6
:109128002C31207F85F82C3194F82D3194F851702A
:1091380094F82EE1617F94F8522085F82D3194F847
:109148002F31697743EA0E2385F8522041EA00213E
:1091580042EA072228771BB212B209B2274885F8DB
:109168005170FFF7A7FE06F19C03029093E80300F5
:109178008DE8030006F18C030FCB06F031FEA07FCB
:1091880094F82EE1E17F94F8537094F8542094F801
:109198002F31E97785F8542085F82F3142EA0722E4
:1091A80043EA0E2341EA0021A8771BB212B209B2A2
:1091B800134885F82EE185F85370FFF77BFE06F11A
:1091C800D403029093E803008DE80300C43696E8C0
:1091D8000F0006F005FE05B0F0BD00BFCF38002037
:1091E8008F4000205931002020560020F9300020FF
:1091F800BA4B00203F350020783000209A4A0020E2
:109208009F35002084B02DE9F04FA3B02CAC84E842
:109218000F009DF8C5309DF8C0E005939DF8C63055
:109228009DF8C11006939DF8C7309DF8C29007932A
:109238009DF8C8309DF8C35008939DF8C9309DF833
:10924800C47009939DF8CA300A939DF8CB300B93EC
:109258009DF8CC300C939DF8CD300D939DF8CE3011
:109268000E939DF8CF300F939DF8F5C09DF8FB3015
:109278009DF8F62010939DF8FC309DF8F7A0119307
:109288009DF8FD309DF8F86012939DF8FE309DF82A
:10929800F98013939DF8FF309DF8FA4014939DF8D8
:1092A800003115939DF8013116939DF802311793FB
:1092B8009DF8033118939DF8043119939DF8D8311E
:1092C8001A939DF8D9311B939DF8DA311C939DF8B8
:1092D800DB311D939DF8DC311E939DF8DD311F9322
:1092E8009DF8DE3120939DF8DF3121939DF82032DF
:1092F80073450BD19DF821328B4207D19DF8553229
:10930800634503D19DF85632934225D0C048C14BDE
:1093180090F810B042EA0C2283F810B090F811B01F
:1093280041EA0E2183F811B090F845B090F8460054
:1093380012B283F8460009B2B74883F845B0FFF780
:1093480089FDB64B029003F1100292E803008DE804
:1093580003000FCB06F044FD9DF822324B450BD19C
:109368009DF82332AB4207D19DF85732534503D1BC
:109378009DF85832B34220D0A54AA64B917CA84804
:109388009974D17CD97492F8471092F8482083F8E0
:10939800471083F8482045EA092146EA0A2212B212
:1093A80009B2FFF757FD9F4B029093E803008DE841
:1093B800030013E90F0006F013FD9DF82432BB42A9
:1093C8000CD19DF82532059A934207D19DF8593260
:1093D800434503D19DF85A32A34221D08C4A8D4B84
:1093E800117D91481975517D597592F8491092F877
:1093F8004A2083F8491083F84A20059B44EA08224A
:1094080043EA072112B209B2FFF724FD874B029005
:1094180093E803008DE8030013E90F0006F0E0FC71
:109428009DF82632069A93420ED19DF82732079A64
:10943800934209D19DF85B32109A934204D19DF86A
:109448005C32119A934224D0714A724B917D7848CC
:109458009975D17DD97592F84B1092F84C2083F804
:109468004B1083F84C20119B109A069943EA02226C
:10947800079B12B243EA012109B2FFF7EBFC6D4BDF
:10948800029093E803008DE8030013E90F0006F04B
:10949800A7FC604B93F84D20FF2A1CBFFF2283F8DE
:1094A8004D2093F84F20FF2A1CBFFF2283F84F203E
:1094B80093F85120FF2A1CBFFF2283F85120554BF7
:1094C80093F85320FF2A1CBFFF2283F853209DF8EE
:1094D8002832089A934218D19DF82932099A934262
:1094E80013D19DF85D32129A93420ED19DF85E32E7
:1094F800139A934209D19DF838331A9A934204D1AA
:109508009DF839331B9A934231D0414A414B117E21
:1095180008981976517E597692F84D1083F84D10B7
:1095280092F84E1083F84E1092F8281192F82921DB
:1095380083F8281183F829211A9A1B9B129943EA68
:109548000223139A1BB242EA0122099912B241EA94
:10955800002109B23848FFF7ADFC384B029093E878
:1095680003008DE8030013E90F0006F039FC9DF8AD
:109578002A320A9A934218D19DF82B320B9A9342B9
:1095880013D19DF85F32149A93420ED19DF8603240
:10959800159A934209D19DF83A331C9A934204D103
:1095A8009DF83B331D9A93424ED0194A194B917E30
:1095B8000A989976D17ED97692F84F1083F84F1091
:1095C80092F8501083F8501092F82A1192F82B2133
:1095D80083F82A1183F82B211C9A1D9B149943EABE
:1095E8000223159A1BB242EA01220B9912B241EAF0
:1095F800002109B21248FFF75DFC124B029093E874
:1096080003008DE8030013E90F0006F0E9FB1BE0F7
:10961800CF3800208F4000205931002020560020EC
:10962800F930002068560020BA4B0020A0560020D0
:109638003F350020D8560020783000204C560020B6
:109648002F3A0020845600209DF82C320C9A934221
:1096580018D19DF82D320D9A934213D19DF861329D
:10966800169A93420ED19DF86232179A934209D105
:109678009DF83C331E9A934204D19DF83D331F9ABE
:10968800934231D0414A424B117F0C981977517F50
:10969800597792F8511083F8511092F8521083F8C4
:1096A800521092F82C1192F82D2183F82C1183F87E
:1096B8002D211E9A1F9B169943EA0223179A1BB263
:1096C80042EA01220D9912B241EA002109B2314859
:1096D800FFF7F0FB304B029093E803008DE803009E
:1096E80013E90F0006F07CFB9DF82E320E9A934288
:1096F80018D19DF82F320F9A934213D19DF86332F7
:10970800189A93420ED19DF86432199A934209D15E
:109718009DF83E33209A934204D19DF83F33219A15
:1097280093422DD0194A1A4B917F0E989977D17F81
:10973800D97792F8531083F8531092F8541083F89D
:10974800541092F82E1192F82F2183F82E1183F8D5
:109758002F21209A219B189943EA0223199A1BB2B8
:1097680042EA01220F9912B241EA002109B20B48DC
:10977800FFF7A0FB23B0BDE8F04F04B006F086BBAE
:1097880023B0BDE8F04F04B0704700BFCF380020C9
:109798008F4000209A4A0020BC5600209F350020A8
:1097A800FFF718BB002310B50124437083780470B9
:1097B800403B132BC47006D802710B4604305C1A68
:1097C800A24203DC10BD53080371F6E713F8014BFE
:1097D80000F8014FF3E70123037000234370037E71
:1097E8008370403B132B88BF490801717047000004
:1097F800232938B504460D4600F0198127D81129C8
:1098080000F0D58011D8022900F0B38006D80029CD
:1098180000F09780012900F0A28038BD032900F0EC
:10982800B280102900F0B98038BD202900F0DD8011
:1098380006D8122900F0C580132900F0CC8038BD65
:10984800212900F0E080222900F0E78038BD412975
:109858002FD010D8322900F0088106D8302900F01E
:10986800F080312900F0F78038BD332900F00781F6
:1098780040290ED038BD50293BD004D8422924D0E5
:1098880043292CD038BD522947D03CD353294ED038
:1098980038BD60237F4A1946A02006F047FB6022A6
:1098A8007C49A01DFFF796FA0023A3706423E37098
:1098B80038BD794AC0216023A02006F037FB60221A
:1098C8007549A01DFFF786FAF0E7744A4FF49071C6
:1098D8006023A02006F02AFB60227049F1E7704A55
:1098E8004FF4C0716023A02006F020FB60226C4971
:1098F800E7E76C4A4FF4F0716023A02006F016FBEE
:1099080060226849DDE7684A4FF410716023A0209F
:1099180006F00CFB60226449D3E7644A4FF42871CF
:109928006023A02006F002FB60226049C9E7604A74
:109938004FF440716023A02006F0F8FA60225C49D9
:10994800BFE7A0235B4A4FF45871184606F0EEFAB9
:10995800A0225849A01DFFF73DFAA423A7E7A0239A
:10996800554A4FF48061184606F0E0FAA0225249A1
:10997800F0E7A023514A4FF49461184606F0D6FA4E
:10998800A0224E49E6E7A0234D4A4FF4A8611846A5
:1099980006F0CCFAA0224A49DCE7A023494A4FF452
:1099A800BC61184606F0C2FAA0224649D2E7A023B5
:1099B800454A4FF4D061184606F0B8FAA022424949
:1099C800C8E7A023414A4FF4E461184606F0AEFA0E
:1099D800A0223E49BEE7A0233D4A4FF4F86118464D
:1099E80006F0A4FAA0223A49B4E70B46394A4FF4E4
:1099F8000661A02006F09AFA2A463649A01DFFF70C
:109A0800E9F9242353E7344A4FF408612023A020BE
:109A180006F08CFA20223049F0E7304A4FF40A6108
:109A28002023A02006F082FA20222C49E6E72C4ABF
:109A38004FF40C612023A02006F078FA2022284950
:109A4800DCE7284A4FF40E612023A02006F06EFAC6
:109A580020222449D2E7244A4FF410612023A02071
:109A680006F064FA20222049C8E7204A4FF4126120
:109A78002023A02006F05AFA20221C49BEE71C4ADF
:109A88004FF414612023A02006F050FA2022184930
:109A9800B4E700BF59310020F9300020BA4B00204C
:109AA8003F350020783000202F3A00209A4A0020C5
:109AB8009F3500201A4C0020EF3B0020FF35002086
:109AC80082320020FA4A00209F340020B931002059
:109AD800EF49002059320020F74D00207B34002048
:109AE8005B340020D9300020233300209A4B00201B
:109AF800BB4C0020232970B50C4600F0398227D8CA
:109B0800112900F0808111D8022900F0348106D88B
:109B1800002900F00081012900F0158170BD03299A
:109B280000F04181102900F0568170BD202900F015
:109B3800B28106D8122900F07E81132900F09381A2
:109B480070BD212900F0BD81222900F0D08170BDAF
:109B580041293AD010D8322900F04C8206D8302951
:109B680000F01C82312900F02F8270BD332900F0EB
:109B78005782402910D070BD50296CD004D8422992
:109B880039D043294FD070BD522900F094807AD340
:109B9800532900F0A88070BDE24D811D602228463F
:109BA800FFF718F9002385F85E3060232A46194626
:109BB800A02085F85F4006F0EBFA60232A46194694
:109BC800BDE87040A02006F0B1B9D74C811D6022D5
:109BD8002046FFF7FFF8002384F85E304023224632
:109BE80084F85F30C0216023A02006F0D1FA6023FA
:109BF8002246C021E4E7CD4C811D60222046FFF7B4
:109C0800E9F8002384F85E304023224684F85F3068
:109C18004FF490716023A02006F0BAFA6023224620
:109C28004FF49071CCE7C24C811D60222046FFF7AB
:109C3800D1F8002384F85E304023224684F85F3050
:109C48004FF4C0716023A02006F0A2FA60232246D8
:109C58004FF4C071B4E7B74C811D60222046FFF76E
:109C6800B9F8402384F85F300023224684F85E3038
:109C78004FF4F0716023A02006F08AFA6023224690
:109C88004FF4F0719CE7AC4C811D60222046FFF731
:109C9800A1F8402384F85F300023224684F85E3020
:109CA8004FF410716023A02006F072FA6023224658
:109CB8004FF4107184E7A14C811D60222046FFF704
:109CC80089F8402384F85F300023224684F85E3008
:109CD8004FF428716023A02006F05AFA6023224628
:109CE8004FF428716CE7964C811D60222046FFF7DF
:109CF80071F8402384F85F300023224684F85E30F0
:109D08004FF440716023A02006F042FA60232246F7
:109D18004FF4407154E78B4C811DA0222046FFF779
:109D280059F8212384F89F30072384F89E30A02314
:109D380022464FF45871184606F02AFAA023224604
:109D48004FF458713CE7804C811DA0222046FFF754
:109D580041F8212384F89F30072384F89E30A023FC
:109D680022464FF48061184606F012FAA0232246D4
:109D78004FF4806124E7754C811DA0222046FFF72F
:109D880029F8212384F89F30072384F89E30A023E4
:109D980022464FF49461184606F0FAF9A0232246A9
:109DA8004FF494610CE76A4C811DA0222046FFF70E
:109DB80011F8212384F89F30072384F89E30A023CC
:109DC80022464FF4A861184606F0E2F9A02322467D
:109DD8004FF4A861F4E65F4C811DA0222046FEF7EF
:109DE800F9FF2E2384F89F30F12384F89E30A023B6
:109DF80022464FF4BC61184606F0CAF9A023224651
:109E08004FF4BC61DCE6544C811DA0222046FEF7CD
:109E1800E1FF2E2384F89F30F12384F89E30A0239D
:109E280022464FF4D061184606F0B2F9A023224624
:109E38004FF4D061C4E6494C811DA0222046FEF7AC
:109E4800C9FF2E2384F89F30F12384F89E30A02385
:109E580022464FF4E461184606F09AF9A0232246F8
:109E68004FF4E461ACE63E4C811DA0222046FEF78B
:109E7800B1FF2E2384F89F30F12384F89E30A0236D
:109E880022464FF4F861184606F082F9A0232246CC
:109E98004FF4F86194E6334D0A46811D2846FEF7D3
:109EA80099FF0A23EB77F6232A46AB774FF406612E
:109EB8002346A02006F06CF923462A464FF4066193
:109EC8007EE6294C811D20222046FEF783FF0A23C7
:109ED800E377F6232246A3774FF408612023A020D6
:109EE80006F056F9202322464FF4086168E61F4C15
:109EF800811D20222046FEF76DFF0A23E377F62313
:109F08002246A3774FF40A612023A02006F040F9E7
:109F18002246BDE8704020234FF40A61A02006F0D5
:109F280037B900BF59310020F9300020BA4B002062
:109F38003F350020783000202F3A00209A4A002030
:109F48009F3500201A4C0020EF3B0020FF350020F1
:109F580082320020FA4A00209F340020B9310020C4
:109F6800EF49002059320020F74D00207B340020B3
:109F7800364C811D20222046FEF72CFF0A23E3776A
:109F8800F6232246A3774FF40C612023A02006F085
:109F9800FFF8202322464FF40C6111E62C4C811D5A
:109FA80020222046FEF716FF0A23E377F6232246EF
:109FB800A3774FF40E612023A02006F0E9F82023B0
:109FC80022464FF40E61FBE5224C811D20222046DB
:109FD800FEF700FF0A23E377F6232246A3774FF420
:109FE80010612023A02006F0D3F8202322464FF446
:109FF8001061E5E5184C811D20222046FEF7EAFE97
:10A008000A23E377F6232246A3774FF4126120232D
:10A01800A02006F0BDF8202322464FF41261CFE5B8
:10A028000E4C811D20222046FEF7D4FE0A23E3773A
:10A03800F6232246A3774FF414612023A02006F0CC
:10A04800A7F8202322464FF41461B9E55B340020B9
:10A05800D9300020233300209A4B0020BB4C00202D
:10A06800C02370B58374837E0446462B84BF462381
:10A07800837623290D4600F0E48026D8112900F0C4
:10A08800AF8010D8022900F0998005D800297BD02C
:10A09800012900F08D8070BD032900F095801029FA
:10A0A80000F0988070BD202900F0AC8006D81229F5
:10A0B80000F09C80132900F09F8070BD212900F0DA
:10A0C800B380222900F0BB8070BD412933D010D85D
:10A0D800322900F0CB8006D8302900F0BB80312926
:10A0E80000F0BE8070BD332900F0C68040290ED034
:10A0F80070BD502930D004D8422921D0432925D019
:10A1080070BD522934D02DD3532937D070BD602368
:10A118005C4D19462A46A02005F008FF6022294612
:10A1280004F11600FFF73EFB95F85E30637695F86C
:10A138005F30A37670BD544D60232A46C021EAE7FC
:10A14800524D60232A464FF49071E4E7504D602346
:10A158002A464FF4C071DEE74E4D60232A464FF47D
:10A16800F071D8E74C4D60232A464FF41071D2E7BE
:10A178004A4D60232A464FF42871CCE7484D6023A6
:10A188002A464FF44071C6E7464DA0232A464FF4AD
:10A198005871184605F0CAFEA022294604F1160097
:10A1A800FFF700FB95F89E30637695F89F30C0E77F
:10A1B8003D4DA0232A464FF48061EAE73B4DA0239A
:10A1C8002A464FF49461E4E7394DA0232A464FF418
:10A1D800A861DEE7374DA0232A464FF4BC61D8E7D3
:10A1E800354DA0232A464FF4D061D2E7334DA02342
:10A1F8002A464FF4E461CCE7314DA0232A464FF4B8
:10A20800F861C6E72F4E0B4632464FF40661A02090
:10A2180005F08CFE2A46314604F11600FFF7C2FA13
:10A22800B37F6376F37F84E7274D2022294604F124
:10A238001600FFF7B7FAAB7F6376EB7F79E7234D1C
:10A24800F3E7234D20232A464FF40C61A02005F0A4
:10A258006DFEEAE71F4D20232A464FF40E61F5E70D
:10A268001D4D20232A464FF41061EFE71B4D202394
:10A278002A464FF41261E9E7194D20232A464FF484
:10A288001461E3E759310020F9300020BA4B00206F
:10A298003F350020783000202F3A00209A4A0020CD
:10A2A8009F3500201A4C0020EF3B0020FF3500208E
:10A2B80082320020FA4A00209F340020B931002061
:10A2C800EF49002059320020F74D00207B34002050
:10A2D8005B340020D9300020233300209A4B002023
:10A2E800BB4C0020F8B5837E0446462B84BF46232A
:10A2F8008376C12323290D46837400F0C18127D8B2
:10A30800112900F0458111D8022900F0088106D8EA
:10A31800002900F0DE80012900F0EE80F8BD032955
:10A3280000F01081102900F02081F8BD202900F0EC
:10A33800688106D8122900F03E81132900F04E8169
:10A34800F8BD212900F07A81222900F08881F8BD22
:10A3580041293AD010D8322900F0F18106D83029A5
:10A3680000F09F81312900F0D981F8BD332900F030
:10A37800F78140290FD0F8BD50295ED004D8422972
:10A3880035D0432946D0F8BD52297CD068D353290B
:10A3980000F08C80F8BDCB4D00F11B0660223146E1
:10A3A8002846FEF717FD637E2A4685F85E30A37EB1
:10A3B80085F85F3060231946A02005F0E9FE304695
:10A3C800BDE8F8406021FFF706BABF4D00F11B0653
:10A3D800602231462846FEF7FDFC637E2A4685F852
:10A3E8005E30A37EC02185F85F306023E4E7B74D77
:10A3F80000F11B06602231462846FEF7EBFC637E1F
:10A408002A4685F85E30A37E4FF4907185F85F3058
:10A418006023D1E7AE4D00F11B0660223146284685
:10A42800FEF7D8FC637E2A4685F85E30A37E4FF49B
:10A43800C07185F85F306023BEE7A64D00F11B06AA
:10A44800602231462846FEF7C5FC637E2A4685F819
:10A458005E30A37E4FF4F07185F85F306023ABE780
:10A468009D4D00F11B06602231462846FEF7B2FCDE
:10A47800637E2A4685F85E30A37E4FF4107185F816
:10A488005F30602398E7954D00F11B066022314646
:10A498002846FEF79FFC637E2A4685F85E30A37E39
:10A4A8004FF4287185F85F30602385E78C4D00F103
:10A4B8001B06602231462846FEF78CFC637E2A463E
:10A4C80085F85E30A37E4FF4407185F85F306023D5
:10A4D80072E7844D00F11B06A02231462846FEF79C
:10A4E80079FC637E2A4685F89E30A37E4FF4587126
:10A4F80085F89F30A0235FE77B4D00F11B06A02263
:10A5080031462846FEF766FC637E2A4685F89E306B
:10A51800A37E4FF4806185F89F30A0234CE7734DEC
:10A5280000F11B06A02231462846FEF753FC637E45
:10A538002A4685F89E30A37E4FF4946185F89F30B3
:10A54800A02339E76A4D00F11B06A02231462846B0
:10A55800FEF740FC637E2A4685F89E30A37E4FF4C2
:10A56800A86185F89F30A02326E7624D00F11B06FD
:10A57800A02231462846FEF72DFC637E2A4685F840
:10A588009E30A37E4FF4BC6185F89F30A02313E76B
:10A59800594D00F11B06A02231462846FEF71AFC49
:10A5A800637E2A4685F89E30A37E4FF4D06185F8F5
:10A5B8009F30A02300E7514D00F11B06A022314631
:10A5C8002846FEF707FC637E2A4685F89E30A37E60
:10A5D8004FF4E46185F89F30A023EDE6484D00F183
:10A5E8001B06A02231462846FEF7F4FB637E2A4666
:10A5F80085F89E30A37E4FF4F86185F89F30A0233C
:10A60800DAE6404E00F11B070A4630463946FEF7A7
:10A61800E1FB637E3246B377A37E4FF40661F3779E
:10A62800A0202B4605F0B4FD38466021FFF7D3F88B
:10A63800A17E3548BDE8F8400AF0B6B8334D00F1C0
:10A648001B06202231462846FEF7C4FB637E2A46B5
:10A65800AB77A37E4FF40861EB772023ACE62C4D53
:10A6680000F11B06202231462846FEF7B3FB637E25
:10A678002A46AB77A37E4FF40A61EB7720239BE64B
:10A68800244D00F11B06202231462846FEF7A2FB86
:10A69800637E2A46AB77A37E4FF40C61EB772023C9
:10A6A8008AE61D4D00F11B06202231462846FEF79A
:10A6B80091FB637E2A46AB77A37E4FF40E61EB775E
:10A6C800202379E659310020F9300020BA4B0020C8
:10A6D8003F350020783000202F3A00209A4A002089
:10A6E8009F3500201A4C0020EF3B0020FF3500204A
:10A6F80082320020FA4A00209F340020B93100201D
:10A70800EF490020593200201C590108F74D00205C
:10A718007B3400205B340020D9300020194D00F133
:10A728001B06202231462846FEF754FB637E2A4644
:10A73800AB77A37E4FF41061EB7720233CE6124DF4
:10A7480000F11B06202231462846FEF743FB637EB4
:10A758002A46AB77A37E4FF41261EB7720232BE6D2
:10A768000A4D00F11B06202231462846FEF732FB2F
:10A77800637E2A46AB77A37E4FF41461EB772023E0
:10A788001AE600BF233300209A4B0020BB4C002060
:10A7980000232DE9F14F954ADFF8A0B2DFF8A0A217
:10A7A800DFF8A092DFF8A082914F924E924D82F886
:10A7B8005E308BF85E308AF85E3089F85E3088F853
:10A7C8005E3087F85E3086F85E3085F85E300723A5
:10A7D8008A498B4C81F89E308A49A02081F89E30A6
:10A7E800894981F89E30894981F89E30F12388494A
:10A7F80081F89E30874981F89E30874981F89E30DC
:10A80800864981F89E30F6238549A3778B77854959
:10A818008B7785498B7785498B7785498B778549F0
:10A828008B7785498B77402382F85F308BF85F30D0
:10A838008AF85F3089F85F3088F85F3087F85F30D2
:10A8480086F85F3085F85F3021236C4981F89F30A6
:10A858006C4981F89F306C4981F89F306B4981F8C9
:10A868009F302E236A4981F89F306A4981F89F30CA
:10A87800694981F89F30694981F89F300A236849FE
:10A88800E377CB776749CB776749CB776749CB774E
:10A898006749CB776749CB776749CB7760231946F8
:10A8A80005F076FC5A466023C021A02005F070FC14
:10A8B800524660234FF49071A02005F069FC4A4687
:10A8C80060234FF4C071A02005F062FC424660236B
:10A8D8004FF4F071A02005F05BFC3A4660234FF47A
:10A8E8001071A02005F054FC324660234FF4287103
:10A8F800A02005F04DFC2A4660234FF44071A020AB
:10A9080005F046FCA0233D4A4FF45871184605F05F
:10A918003FFCA0233B4A4FF48061184605F038FC01
:10A92800A023394A4FF49461184605F031FCA0235E
:10A93800364A4FF4A861184605F02AFCA023344A89
:10A948004FF4BC61184605F023FCA023314A4FF4AC
:10A95800D061184605F01CFCA0232F4A4FF4E4618F
:10A96800184605F015FCA0232C4A4FF4F861184648
:10A9780005F00EFC20232A4A4FF40661A02005F0BA
:10A9880007FC2023274A4FF40861A02005F000FCAB
:10A998002023254A4FF40A61A02005F0F9FB202363
:10A9A800224A4FF40C61A02005F0F2FB2023204A34
:10A9B8004FF40E61A02005F0EBFB20231D4A4FF455
:10A9C8001061A02005F0E4FB20231B4A4FF412611C
:10A9D800A02005F0DDFB202322464FF41461A020BF
:10A9E80001B0BDE8F04F05F0D3BB00BF59310020DE
:10A9F8002F3A00209A4A00209F3500201A4C002048
:10AA0800BB4C0020EF3B0020FF35002082320020A5
:10AA1800FA4A00209F340020B9310020EF49002075
:10AA280059320020F74D00207B3400205B34002091
:10AA3800D9300020233300209A4B0020F930002021
:10AA4800BA4B00203F35002078300020BE22064B4C
:10AA58001A7077225A705B229A705D22DA70EB22A4
:10AA680083F85F21704700BFCF38002010B54FF43E
:10AA780080612F4807F070F82E4C4FF4006184F87D
:10AA8800CD002B4807F068F894F8CD304FF480518A
:10AA980003EB400084F8CD00254807F05DF894F8F2
:10AAA800CD30012103EB800084F8CD00224807F067
:10AAB80053F894F8CD20234602EBC000C0B20C280E
:10AAC80008D8DFE800F00A0F141B2022312F3324A6
:10AAD800292B2D0084F8CD0010BD802283F8CD20CD
:10AAE800012208E0812283F8CD20022203E082229D
:10AAF80084F8CD20042283F8E92010BD832283F84E
:10AB0800CD200322F7E78422EDE78522E6E78622B7
:10AB180083F8CD200022EEE78722F9E78822F7E7BD
:10AB28008922F5E78A22D9E78B22E8E78C22DAE73F
:10AB380000100140CF38002000140140764B774ABE
:10AB48002DE9F0411360764A183B13607549764B3E
:10AB5800764A0B60183B1360FF200023ADF52C7D6F
:10AB68000C68E0541468E0540133042BF8D1704C9D
:10AB780094F85A31802B15D1012222720022202B01
:10AB8800627215D10122A2720022082BE27215D13D
:10AB9800012222730022022B627315D10123A373B1
:10ABA800002315E00022402B2272E7D101226272B5
:10ABB8000022102BA272E7D10122E2720022042B9C
:10ABC8002273E7D1012262730022012BA273E7D11D
:10ABD800227A4FF400415748E37306F0C3FF627AC4
:10ABE8004FF48061544806F0BDFFA27A1021534803
:10ABF80006F0B8FFE27A4FF48041514806F0B2FF00
:10AC0800227B40214F4806F0ADFF627B4FF4006184
:10AC1800494806F0A7FFA27B2021484806F0A2FF7A
:10AC2800E27B4FF40041464806F09CFF0A2006F0FC
:10AC380041F84FF4B072444954A809F0A1FDD4F882
:10AC480000806768A668E5684FF4A8723F496846BF
:10AC580009F096FD3246404639462B46FEF7D2FAB1
:10AC68002279002A37D14FF48071344806F07AFFF0
:10AC780001224FF40071314806F074FF627992BBEB
:10AC88004FF480612D4806F06DFF01224FF40061FA
:10AC98002A4806F067FFA2796ABB4FF4805127481B
:10ACA80006F060FF01224FF40051244806F05AFFD5
:10ACB800E27942BB4FF48041204806F053FF01225D
:10ACC8004FF400411D4806F04DFF0DF52C7DBDE801
:10ACD800F041FFF7BBBE01224FF48071174806F020
:10ACE80041FF0022C5E701224FF48061134806F0B6
:10ACF80039FF0022CAE701224FF480510F4806F0BD
:10AD080031FF0022CFE701224FF480410B4806F0C3
:10AD180029FF0022D4E700BFEB390020AC820020D5
:10AD2800D881002020820020AB410020D07B002069
:10AD3800CF380020000C01400014014000200140E1
:10AD480000180140001001408F400020DF3800202B
:10AD5800F8B5E02383750023C3750A23037680239F
:10AD68004376FF230F228376C3764377AC4B027773
:10AD780093F8EA20044622B193F86B20012A40F0A8
:10AD8800908593F86B20002A40F07985A277E277C6
:10AD980084F8202084F8212084F822200120E02251
:10ADA800052584F8232084F8240084F8255093F896
:10ADB800661084F8261093F8671084F8271093F823
:10ADC800681084F8281093F8691084F8291093F80B
:10ADD8006A1084F82B2084F82A10022184F82D00A8
:10ADE80084F82C1093F86B1084F82F2084F82E1018
:10ADF800032184F8315084F8301093F86C5084F8AB
:10AE0800325093F86D5084F8335093F86E5084F8AC
:10AE1800345093F86F5084F8355093F8705084F894
:10AE28003650042584F8372084F8385084F83910CF
:10AE380093F8715084F83A5093F8725084F83B5064
:10AE480093F8735084F83D2084F83C50062584F824
:10AE58003F0084F83E5093F8740084F8412084F849
:10AE68004000082084F8431084F8420093F87610D4
:10AE780004F1720084F8441093F8771084F84510B0
:10AE880093F8781084F8472084F84610092184F84C
:10AE9800495084F8481093F8791084F84A1093F8C8
:10AEA8007A1084F84B1093F87B1084F84C1093F8C0
:10AEB8007C1084F84D1093F87D1084F84E1093F8A8
:10AEC8007E1084F850200A2284F84F1084F851200C
:10AED8002021224602F8521F524911F8015F02F858
:10AEE800015F8242F9D10B21E02284F8741003211A
:10AEF80084F8732084F8751093F89F1004F1A40067
:10AF080084F8761093F8A01084F8771093F8A110BD
:10AF180084F8792084F878100C2184F87A100621B6
:10AF280084F87B1093F8A21084F87C1093F8A3108F
:10AF380084F87D1093F8A41084F87E1093F8A51077
:10AF480084F87F1093F8A61084F8801093F8A7105F
:10AF580084F882200D2284F8811084F8832020212F
:10AF6800224602F8841F304911F8015F02F8015F98
:10AF78008242F9D193F83000102184F8A8001120FA
:10AF880084F8AA0093F85700E02284F8AC00122055
:10AF980084F8AE0093F8580084F8A61084F8B0003E
:10AFA8000121162084F8A52084F8A92084F8AD2072
:10AFB80084F8B12084F8A71084F8AB1084F8AF1097
:10AFC80084F8B20084F8B31093F8CC0084F8B52064
:10AFD80084F8B400172084F8B71084F8B60093F802
:10AFE800CD1084F8B92084F8B810182184F8BA1064
:10AFF800022184F8BB1093F8CE1004F1D40084F831
:10B00800BC1093F8CF1084F8BD1084F8BE20192224
:10B01800142184F8BF20224602F8C01F034907E024
:10B02800CF3800204D390020763900209E39002085
:10B0380011F8015F02F8015F8242F9D11A21E0227A
:10B04800012084F8D61003261B2184F8D52084F823
:10B05800D70083F8E40084F8D80084F8D92084F86D
:10B06800DA1084F8DB6093F8E51084F8EB2084F8B4
:10B07800DC1093F8E61084F8DD1093F8E71084F8F4
:10B08800DF2084F8DE101D2184F8E10084F8E01048
:10B0980093F8E81084F8E32084F8E2101E2184F87D
:10B0A800E50084F8E41093F8E91084F8E72084F8C0
:10B0B800E6101F2184F8E90084F8E81093F8EA10F4
:10B0C80084F8EA10202184F8EC10022184F8ED10AD
:10B0D80093F8285084F8F02084F8EE5093F829501B
:10B0E80084F8F21084F8EF50212584F8F15093F891
:10B0F8002A5084F8F52084F8F35093F82B5084F8FC
:10B10800F71084F8F450222584F8F65093F82C5060
:10B1180084F8FA2084F8F85093F82D5084F8FC103D
:10B1280084F8F950232584F8FB5093F82E5084F8BE
:10B13800FF2084F8FD5093F82F5084F8011184F80B
:10B14800FE50242584F8005193F8205084F80251C9
:10B1580093F8215084F80351252584F8042184F8B4
:10B16800055193F8225084F8061184F8075193F892
:10B17800235084F8092184F80851262584F80A51B7
:10B1880093F8245084F80B1184F80C5193F8255047
:10B1980084F80E2184F80D51272584F80F5193F86F
:10B1A800265084F8101184F8115193F8275084F828
:10B1B800132184F81251302584F814511D7A84F82B
:10B1C800150184F81651312584F818515D7A84F8F0
:10B1D800172184F81A51322584F8190184F81B21A3
:10B1E80084F81C5184F81D019D7A1F7C84F81E5137
:10B1F800332584F82051DD7A84F81F2184F8225100
:10B20800342584F824515D7C84F8210145EA07251A
:10B218002DB22F1284F82751352584F8267184F829
:10B2280029519F7CDD7C84F8232145EA07252DB22E
:10B238002F1284F82C51362584F82B7184F82E515E
:10B248001F7D5D7D84F8251145EA07252DB22F1253
:10B2580084F83151372584F8282184F82A1184F894
:10B268002D2184F82F1184F8307184F832219F7DC4
:10B2780084F8341184F83351DD7D84F8372145EAA8
:10B2880007252DB22F1284F83651382584F83571E8
:10B2980084F8385193F8457093F8465084F839117A
:10B2A80045EA07252DB22F1284F83B51392584F839
:10B2B8003A7184F83D5193F8477093F8485084F8F0
:10B2C8003C2145EA07252DB22F1284F840513A2532
:10B2D80084F83F7184F8425193F8497093F84A50C2
:10B2E80084F83E1145EA07252DB22F1284F84551FE
:10B2F8003B2584F8447184F8475193F84B7093F8D0
:10B308004C5084F8412145EA07252DB22F1284F8C4
:10B318004A513C2584F8431184F8462184F84811A1
:10B3280084F8497184F84B2184F84C5193F85A50A9
:10B3380093F83BE084F84E5193F85B50082784F863
:10B348004F513D2584F8515193F85C5084F84D11C4
:10B3580084F8535193F85D5084F8502184F854517F
:10B368003F2584F8565193F83C5084F8521145EA29
:10B378000E2505EB85058540ADB245F3072E84F80B
:10B3880058E184F8595193F83DE093F83E5084F819
:10B39800552145EA0E2505EB85058540ADB245F3F7
:10B3A800072E84F85AE184F85B5193F83FE093F84C
:10B3B800405084F8602145EA0E2505EB8505854057
:10B3C800ADB245F3072E84F85CE184F85D5193F83B
:10B3D80041E093F8425084F8577145EA0E2505EB91
:10B3E80085058540ADB245F3072E84F85F514925A0
:10B3F80084F85EE184F8615193F8F35084F86B2186
:10B4080084F8635193F8F45084F86D0184F864511A
:10B4180093F8F55084F86F2184F8655193F8F65045
:10B4280084F8710184F8665193F8F75084F8732111
:10B4380084F8675193F8F85084F8750184F86851D6
:10B4480093F8F95084F8627184F8695193F8FA50C6
:10B458004FF0040E84F86A514A2584F86C5193F829
:10B46800FB5084F86E514B2584F8705193F8FC50CA
:10B4780084F87251502584F8745193F8315084F847
:10B488007651512584F8772184F8785193F8FD5046
:10B4980084F887E184F87A5193F8FE5084F879119A
:10B4A80084F87B51532584F87D5193F8005184F832
:10B4B8007C2184F87F51542584F8815193F80151F7
:10B4C80084F87E0184F8835193F8025184F880212E
:10B4D80084F88451562584F8865193F8045184F8E9
:10B4E800821184F8885193F8055184F8852184F8ED
:10B4F800895193F8065184F88C2184F88A5193F87D
:10B50800075184F88E0184F88B51602584F88D5199
:10B518001D7B84F8902184F88F51612584F891511E
:10B528005D7B84F8920184F89351622584F89551E3
:10B538009D7B84F8942184F89751632584F8995168
:10B54800DD7B84F8960184F89B51642584F89D512D
:10B558001D7E84F8982184F89F515D7E84F89A01B5
:10B5680084F8A051652584F8A2519D7E84F89C2119
:10B5780084F8A451DD7E84F89E1184F8A5516625CF
:10B5880084F8A12184F8A31184F8A62184F8A7518E
:10B598001D7F93F84DC084F8A9515D7F84F8A811E8
:10B5A80084F8AA51672584F8AC519D7F84F8AB21B3
:10B5B80084F8AE51DD7F84F8AD1184F8AF51682569
:10B5C80084F8B15193F84E5084F8B02145EA0C251F
:10B5D8002DB245FA07FC84F8B451692584F8B3C143
:10B5E80084F8B65193F84FC093F8505084F8B211CC
:10B5F80045EA0C252DB245FA07FC84F8B9516A25AD
:10B6080084F8B8C184F8BB5193F851C093F85250EC
:10B6180084F8B52145EA0C252DB245FA07FC84F8D3
:10B62800B71184F8BA2184F8BC1184F8BDC184F834
:10B63800BE516B2593F853C084F8C05193F8545009
:10B6480084F8BF2145EA0C252DB245FA07FC84F899
:10B65800C3516C2584F8C55193F8105184F8C2C1C0
:10B6680084F8C75193F8115193F833C084F8C8513E
:10B678006F2584F8CA5193F8345084F8C11145EA0B
:10B688000C2505EB85058540ADB245F3072C84F8FC
:10B69800CCC184F8CD5193F835C093F8365084F86E
:10B6A800C42145EA0C2505EB85058540ADB245F377
:10B6B800072C84F8CEC184F8CF5193F837C093F89B
:10B6C800385084F8C61145EA0C2505EB85058540F8
:10B6D800ADB245F3072C84F8D0C184F8D15193F862
:10B6E80039C093F83A5084F8C92145EA0C2505EB8E
:10B6F80085058540ADB245F3072C84F8D2C184F89E
:10B70800CB7184F8D351742584F8D5511D7984F808
:10B71800D42184F8D751752584F8D9515D7984F8F6
:10B72800D60184F8DB51762584F8DD519D7984F8BB
:10B73800D82184F8DF51772584F8E151DD7984F840
:10B74800DA0184F8E351802584F8E55193F8325002
:10B7580084F8DC2184F8E751812584F8E95193F8CD
:10B76800435084F8DE0184F8EB5193F8445084F890
:10B77800E02184F8EC51832584F8E20184F8E4217F
:10B7880084F8E60184F8E82184F8EA1184F8ED21C8
:10B7980084F8F31193F8191184F8F12184F8F4115D
:10B7A80093F81A1184F8F62184F8F51184F8FD212C
:10B7B80086218F2284F8EE5193F8185184F8F711F6
:10B7C80084F8F051842593F81C1184F8FE2193F82D
:10B7D800282184F8F91184F8002293F81D1193F8B0
:10B7E800292184F8FA1184F8012293F81E1193F89C
:10B7F8002A2184F8FB1184F8022293F81F1193F888
:10B808002B2184F8F8E184F8EF0184F8F25184F8E8
:10B81800FC1184F8FF7184F8032293F82C214FF46B
:10B82800F97184F8042293F82D2184F8052293F8FD
:10B838002E2193F82F3184F8062284F80732F22358
:10B84800E074237504F1160003F0AAFF05462046AC
:10B8580003F085FF25FA07F3607584F80832294656
:10B8680084F8095284F80A62264808F09DFF2046A9
:10B8780040F20B2105F0F2F94FF4F970F8BD93F896
:10B888006C20A27793F86D20E27793F86E2084F805
:10B89800202093F86F2084F8212093F87020FFF778
:10B8A8007BBA93F866200AB193F85F20A27793F8E1
:10B8B80067200AB193F86020E27793F8682042B1D4
:10B8C80093F8622093F8611022F00F0201F00F0143
:10B8D8000A4384F8202093F869200AB193F8642079
:10B8E80084F8212093F86A20002A3FF455AA93F897
:10B8F800632093F8651022F00F0201F00F010A434C
:10B90800FFF74ABA0C5901082DE9F0410D46002706
:10B91800ADF52C7D1570B29A03280446177088BFC0
:10B9280000214FF0FF0298BF1A49B39E9CBF51F8FF
:10B9380020001949327094BF31F814100846174E88
:10B948000DBB2A4606F00EF901233370144C4FF450
:10B95800B072144954A808F013FFD4F8008067683F
:10B96800A668E56804F110014FF4A872684608F06B
:10B9780007FF4046394632462B46FDF743FC0DF596
:10B988002C7DBDE8F0811A705A700122375506F0F7
:10B99800E9F8DBE7C8580108D8580108B02A0020A0
:10B9A800CF3800208F4000202DE9F04105460328BC
:10B9B8000C4698BF1D49ADF52C7D9CBF51F8200061
:10B9C8001B49147098BF31F815104FF00005B29A52
:10B9D80088BF002115704FF0FF02B39D88BF08464D
:10B9E8002A70FCB92246134C06F0BCF84FF4B0722A
:10B9F800114954A808F0C4FED4F800806768A66806
:10BA0800E56804F110014FF4A872684608F0B8FE22
:10BA18004046394632462B46FDF7F4FB0DF52C7DA2
:10BA2800BDE8F0811A705A700122DCE7E458010879
:10BA3800F4580108CF3800208F40002050232DE90A
:10BA4800F3478E4CFF2684F8583084F8EA304623B2
:10BA580001274FF000084FF0E20984F85B304FF0FF
:10BA6800FE0A522384F8667084F8677084F8687058
:10BA780084F8697084F86A7084F85780277267724E
:10BA8800A772E77284F8108084F8128084F8148012
:10BA980084F8168084F8118084F8138084F815805F
:10BAA80084F8178084F85A6184F8456084F84690D1
:10BAB80084F8476084F8489084F8496084F84A908C
:10BAC80084F84B6084F84C9084F85A8084F85CA021
:10BAD80084F85D30072384F8FB309C2384F8FE301B
:10BAE800F623674D84F8023105F1F403019304F558
:10BAF8008273009304F108022B463946404684F8C5
:10BB0800F38084F8F48084F8317084F8FD6084F858
:10BB1800007184F80161FFF7F7FE05F1F503019361
:10BB280004F20513617A009304F10902AB1C38464C
:10BB3800FFF7EAFE05F1F603019304F58373A17A92
:10BB4800009304F10A022B1D0220FFF7DDFE05F128
:10BB5800F703019304F20713E17A009304F10B024F
:10BB6800AB1D0320FFF7D0FE38236376E3766377B7
:10BB7800E3774C2384F81131702384F84430602330
:10BB880084F81A3105F5867327736773A773E7730B
:10BB98002676A6762677A67784F84D6084F84E90A8
:10BBA80084F84F6084F8509084F8516084F852907B
:10BBB80084F8536084F8549084F8106184F8048001
:10BBC80084F8058084F8068084F8078084F8327049
:10BBD80084F843A084F8187184F81961019304F576
:10BBE8008E73009304F10C0205F1080339464046B0
:10BBF800FFF7DAFE05F20D13019304F21D13617BC2
:10BC0800009304F10D0205F10A033846FFF7CCFE54
:10BC180005F58773019304F58F73A17B009304F1F5
:10BC28000E0205F10C030220FFF7BEFE05F20F130A
:10BC3800019304F21F13009304F10F0205F10E03A0
:10BC4800E17B0320FFF7B0FE63220E4B05F8106975
:10BC58001A805A809A80DA80AE742E75AE756E742A
:10BC6800EE746E75EE752E76AE762E77AE776E76AE
:10BC7800EE766E77EE7702B0BDE8F087CF38002019
:10BC88009F400020B42A0020F0B5154B93F8FC50D3
:10BC980025B393F83120012A20D1124A93F8FB10DA
:10BCA8001478A142114619D9022D17D00E4D002241
:10BCB8002E46875C57550132062AFAD10B4AAD78D1
:10BCC800907885421FBF01340C70012183F8FC1065
:10BCD8000023F15CD1540133062BFAD1F0BD00BF2B
:10BCE800CF380020D8300020BC2A0020C32A0020EA
:10BCF8002DE9F047964C974E0128ADF52C7D054669
:10BD080004F5827306F1010A04F2051906F1020826
:10BD180004F5837740F088808DE848000146A6F155
:10BD2800F40320726072A072E07220736073A073D3
:10BD3800E07304F108020020FFF7E6FDA6F1F20324
:10BD48002946284604F109028DE80006FFF7DCFDC4
:10BD58008DE88001A6F1F003294604F10A020220C9
:10BD6800FFF7D2FDF31C019304F207132946009351
:10BD780004F10B02A6F1EE030320FFF7C5FD06F15F
:10BD88001803019304F58E732946009304F10C02FD
:10BD9800A6F1EC030020FFF707FE06F11903019353
:10BDA80004F21D1329462846009304F10D02A6F15A
:10BDB800EA03FFF7F9FD06F11A03019304F58F73FF
:10BDC8002946009304F10E02A6F1E8030220FFF7CA
:10BDD800EBFD06F11B03019304F21F1329460093A0
:10BDE80004F10F02A6F1E6030320FFF7DDFDA6F537
:10BDF80082714FF4B07254A808F0C2FCD4F80080E5
:10BE08006768A668E5684FF4A87204F110016846EF
:10BE180008F0B6FC4046394632462B46FDF7F2F9A3
:10BE28000DF52C7DBDE8F08700258DE8480004F16C
:10BE38000802A6F1F4032946284625726572A57200
:10BE4800E57225736573A573E573FFF75DFDA6F1CC
:10BE5800F20304F10902294601208DE80006FFF7E4
:10BE680053FDA6F1F00304F10A02294602208DE8E9
:10BE78008001FFF749FDF31C019304F207130093B7
:10BE880004F10B02A6F1EE0329460320FFF73CFD5F
:10BE980006F11803019304F58E73009304F10C0264
:10BEA800A6F1EC0329462846FFF77EFD06F11903A3
:10BEB800019304F21D13009304F10D02A6F1EA03A5
:10BEC80029460120FFF770FD06F11A03019304F5D6
:10BED8008F73009304F10E02A6F1E80329460220AD
:10BEE800FFF762FD06F11B03019304F21F13009391
:10BEF80004F10F02A6F1E60329460320FFF754FDDB
:10BF080084F85F5084F8605084F8615084F8625077
:10BF180084F8635084F8645084F8655084F80C51B0
:10BF280084F80D5184F80E5184F80F5184F80451A7
:10BF380084F8055184F8065184F8075184F824518F
:10BF480084F8255184F8265184F8275168E700BF02
:10BF5800CF380020934100202DE9F0416E4AADF51D
:10BF68002C7D6E4C6E4B002840F095801178217224
:10BF7800517861729178D278A172E2721A7822733C
:10BF88005A7862739A78DB78A273E373654E664DCC
:10BF9800217AA6F1F4030196A5F1FC020095002090
:10BFA800FFF7B2FC731C617A01936B1C0093A5F137
:10BFB800FB02A6F1F2030120FFF7A6FCB31CA17A4D
:10BFC8000193AB1C0093A5F1FA02A6F1F00302203D
:10BFD800FFF79AFCF31CE17A0193EB1C0093A5F19F
:10BFE800F902A6F1EE030320FFF78EFC06F1180311
:10BFF800217B019305F118030093A5F1F802A6F13E
:10C00800EC030020FFF7D0FC06F11903617B0193D4
:10C0180005F119030093A5F1F702A6F1EA0301203F
:10C02800FFF7C2FC06F11A03A17B019305F11A037D
:10C038000093A5F1F602A6F1E8030220FFF7B4FC8D
:10C0480006F11B03E17B019305F11B030093A5F1A6
:10C05800F502A6F1E6030320FFF7A6FCA6F5827118
:10C068004FF4B07254A808F08BFBD4F800806768CE
:10C07800A668E468A5F1F4014FF4A872684608F0D0
:10C088007FFB4046394632462346FDF7BBF80DF59F
:10C098002C7DBDE8F081217A1170617A5170A17A06
:10C0A8009170E17AD170227B1A70627B5A70A27B00
:10C0B8009A70E27BDA70002323726372A372E372D0
:10C0C80023736373A373E37384F85F3084F8603079
:10C0D80084F8613084F8623084F8633084F864301E
:10C0E80084F8653084F80C3184F80D3184F80E3109
:10C0F80084F80F3184F8043184F8053184F8063166
:10C1080084F8073184F8243184F8253184F82631FD
:10C1180084F827313AE700BFE02A0020CF38002012
:10C12800E42A002093410020D3390020F0B50022F2
:10C1380004464F1E974200D8F0BD0132134699427B
:10C1480001D80234F6E730F813502688AE423CBFD7
:10C1580020F8136025800133F1E7034600EB410125
:10C1680000208B4200D1704733F8022B1044F8E7C7
:10C178002DE9F04FDFF80C8387B098F8103198F864
:10C18800110104AE00EB032000B2FCF7A7F9B0A33D
:10C19800D3E90023FCF708FAFCF7A0FC98F85A301A
:10C1A80004B298F85B0000EB032000B2FCF796F9A4
:10C1B800A7A3D3E90023FCF7F7F9FCF78FFC98F85D
:10C1C8005C300FFA80F998F85D0000EB032000B2AC
:10C1D800FCF784F99EA3D3E90023FCF7E5F9FCF703
:10C1E8007DFC98F8013105B298F8020100EB0320B4
:10C1F80000B2FCF773F996A3D3E90023FCF7D4F94E
:10C20800FCF76CFC98F8193107B298F81A0100EBA2
:10C21800032000B2FCF762F98DA3D3E90023FCF7F1
:10C22800C3F9FCF75BFC03B298F83B20009398F83D
:10C238003C3009F1FF3E43EA0223ADF8083098F894
:10C248003D2098F83E3043EA0223ADF80A3098F8CA
:10C258003F2098F8403043EA0223ADF80C3098F8B4
:10C26800412098F8423043EA0223ADF80E3098F89E
:10C27800332098F8343043EA0223ADF8103098F8A8
:10C28800352098F8363043EA0223ADF8123098F892
:10C29800372098F8383043EA0223ADF8143098F87C
:10C2A800392098F83A304FF0010843EA0223ADF8F4
:10C2B800163000239C46684A02A931F913108945B3
:10C2C80000F3928003F802800133042BF4D1634B0E
:10C2D800634AD3F800E000231146984642F2107AE8
:10C2E800781EDFF8A4C1019011F8019FB9F1010F80
:10C2F8007FD102A830F913B00198584579DD1EF8AE
:10C3080003B0BBF1000F74D056480CF8039050F8F6
:10C318002390D14506D991F8FC90B9F1000F01D0CE
:10C3280081F8FC800133042BDED100234FF0010893
:10C338009C464D4902A830F91390B9455CDB03F8D7
:10C3480001800133042BF5D100214FF0010C0F4679
:10C35800464B05F1010E12F8018FB8F1000F53D1C9
:10C3680083F800800131042903F10103F3D100238C
:10C3780042F2107819464FF0010A00983C4A3D4DA8
:10C38800DFF808C13C4F00F1FF3912F801EFBEF1A8
:10C39800010F50D105F803E05CF823E0C64506D943
:10C3A80092F810E1BEF1000F01D082F8101136F9B1
:10C3B80013E00098704540DC03F807A00133042B14
:10C3C800E3D100234FF0010E1A462C4F2C49651E6D
:10C3D80036F91300844234DC03F801E00133042BFE
:10C3E800F6D107B0BDE8F08F8E45C8BF03F802C08C
:10C3F8006AE70CF8038095E71EF80390B9F1000F7F
:10C408009FD003F801C09CE792F8E78002A8B8F132
:10C41800000F09D130F911804545A8BF83F800C045
:10C42800C6459FDA1F709DE730F91180C645F9DBD4
:10C4380083F800C096E7E954B9E7F145C8BFD95574
:10C44800BCE78542C8BF5A5447F82320C6E700BF57
:10C458009A9999999999B93F54290020D88100202F
:10C46800D6380020C82F0020602900205829002035
:10C47800DA380020642900206C29002018300020B8
:10C4880068290020CF3800205C290020F82F0020E0
:10C498000246002310B58B4200DB10BD54880133DF
:10C4A80022F8024BF7E700002DE9F74FBC4B1C6858
:10C4B800009314F0010447D14FF0C80AB94EDFF8D1
:10C4C8003093D6F80080B84FB84D1FFA88FB0AFBA6
:10C4D80004905946FFF741FE57F824301844B0FB42
:10C4E800F8F035F8143047F82400184425F81400FB
:10C4F8000134042CEBD100244FF0C80BAC4DAD4BEC
:10C50800D5F80090DFF8DC82AB4F1FFA89FA0BFBF5
:10C51800043051460193FFF720FE58F82420019B70
:10C528001044B0FBF9F037F8142048F82400104400
:10C5380027F814000134052CE9D100239F4A336001
:10C548002B601378013313709C4E3378312B40F2F3
:10C55800FD8000259A4FDFF89CA2DFF88C82DFF877
:10C568004CB2984B1A78052A40F0F98006214046CB
:10C57800FFF78EFF3BF81530327893FBF2F3A8F8FB
:10C588000A30002138F8113027F811300131062916
:10C59800F8D13846FFF7CAFDBB88788800241844CC
:10C5A800DAF80430DFF850921844FB8808F10C08D8
:10C5B80018443B890C371844CAF804008008FBF774
:10C5C8007DFF73A3D3E90023FBF7EEFF00227E4B28
:10C5D800FBF7EAFF7D4B0022FBF7E6FFFCF7A6FA24
:10C5E800714B29F8150043F825402BF81540013503
:10C5F800042D4AF8044FB4D1754DB9F80030B9F894
:10C6080006001A0A85F82130B9F8023085F820208A
:10C6180085F823301A0AB9F8043085F822201A0A56
:10C6280085F8242085F82530FBF758FF5AA3D3E96D
:10C638000023FBF7B9FF0022664BFBF701FE664BB0
:10C648000022FBF7B1FFFCF749FA95F85730DFF8FD
:10C65800ACA1184485F83000DFF890915F4DDFF801
:10C6680058B1584B93F80080B8F1050F40F083801B
:10C6780006214846FFF70CFF3BF81430327893FB4D
:10C68800F2F3A9F80A30002139F8113025F81130F1
:10C6980001310629F8D12846FFF748FD6B88A8889C
:10C6A8004F4F1844DAF804300C35184435F8063C76
:10C6B80009F10C09184435F8043C1844CAF8040078
:10C6C8008008FBF7FBFE32A3D3E90023FBF76CFFDE
:10C6D80000223D4BFBF768FF00223C4BFBF764FF51
:10C6E800FCF724FA00233F4A27F8140042F82430C4
:10C6F8002BF814300134052C4AF8043FB1D13149E4
:10C7080008F1010881F8008000997A880B6033707D
:10C718002F4B110A83F82920BA8883F8281083F848
:10C728002B20110AFA8883F82A1083F82D20110A81
:10C738003A8983F82C1083F82F20110A3A8883F855
:10C748002E10110A83F8261083F827201D4B1A781B
:10C75800042A84BF05221A7003B0BDE8F08F0623AF
:10C76800317803FB05233BF8152092FBF1F21E49B3
:10C7780021F8132005E7062331783BF8142003FB42
:10C78800048392FBF1F2194921F813207BE700BFDB
:10C798006666666666660A40FCA9F1D24D62503F3D
:10C7A800102F002064300020EC290020E42900200C
:10C7B800683000203E7C0020882A0020C92A0020FA
:10C7C800A4290020E82A00200000303F00408F40C4
:10C7D800CF3800200000E03F00005940382A0020F0
:10C7E800904A0020942A002074290020FC29002067
:10C7F800B0780020D0290020184E0020702A002090
:10C80800FFF7B6BC0000000070B506460D460022D2
:10C81800002330462946FCF739F928B3012405F1ED
:10C8280000450022144B30462946FBF7BDFEFCF7B5
:10C838007DF90A22C3B2B3FBF2F002FB1030C0B29A
:10C84800052885BF9B181B1A1B1A03F0FF0098BF09
:10C85800D8B2FBF743FE06A3D3E90023FBF7A4FEF7
:10C868000CB101F1004170BD0446DAE7AFF3008076
:10C878009A9999999999B93F0000244000000000BD
:10C8880070B50022002306460D46FCF7FFF828B3D2
:10C89800012405F100450022194B30462946FBF7D3
:10C8A80083FEFCF71BF90A22C3B2B3FBF2F002FBCA
:10C8B8001030C0B2042813D913441B1A03F0FF0028
:10C8C800FBF70CFE0CA3D3E90023FBF76DFE0CB1BC
:10C8D80001F10041FCF702F940B270BD0446DAE705
:10C8E80030462946FCF7FAF8C0B200EB8000400059
:10C8F800C0B2E5E7AFF300809A9999999999B93F41
:10C9080000002440000000002DE9F04F00258BB006
:10C918005B0800240893002392461646AB462F4630
:10C92800CDE902345EA418CCCDE90001CDE9043488
:10C93800089B9D420FDBDDE90023DDE90201FCF7DE
:10C94800C3F8002876D0089B149A134413F9010CF5
:10C95800FBF7C4FD9CE030780002FBF7BFFD804682
:10C9680089467078FBF7BAFD42464B46FBF76AFCEE
:10C978000022002380468946FCF77EF804460028FA
:10C9880050D100224A4B40464946FBF737FFCDE9D4
:10C998000201B0780002FBF7A1FD80468946F078D5
:10C9A800FBF79CFD42464B46FBF74CFC0022404BF4
:10C9B800FBF724FF02460B46DDE90201FBF740FCCA
:10C9C80039A3D3E90023FBF7EFFDCDE90601EBB26C
:10C9D80009932046FBF782FDDDE90623FBF7E4FD1A
:10C9E80002460B46DDE90201FBF72AFCDDE90023DC
:10C9F80080468946FCF75EF8B8B1DDE90023404679
:10CA08004946FBF71DFCDDE9042380468946FCF70F
:10CA18003DF820B1CDE90489099F5FFA84FB013410
:10CA28000A2CD6D10135023682E74246DDE90001FB
:10CA38004B46E6E79AF800000002FBF74FFD044674
:10CA48000D469AF80100FBF749FD22462B46FBF7F5
:10CA5800F9FB0022164BFBF7D1FE0B460246DDE937
:10CA68000001FCF713F8149BA8B1D857FBF736FD63
:10CA7800044658460D46FBF731FD0BA3D3E90023C6
:10CA8800FBF792FD02460B4620462946FBF7D8FBEA
:10CA98000BB0BDE8F08F93F9000059E7AFF30080C1
:10CAA8000000000000E06F409A9999999999B93F60
:10CAB80000408F40000000002DE9F04F144600258B
:10CAC8004FF0000A4FF0000BA3B0CDE9000150224F
:10CAD80000210EA8099307F05EFE237808950B93B2
:10CAE800637803950C9362A3D3E90023CDE904236B
:10CAF800099B013B0A93099B9D4210DBDDE900235A
:10CB080050465946FBF7D6FF002800F087802C9B3B
:10CB1800039A9856FBF7E2FC23B0BDE8F08F6378E0
:10CB2800207843EA0020FBF7D9FC53A3D3E900237C
:10CB3800FBF73AFD8246A0788B460002FBF7CEFC55
:10CB480006460F46E078FBF7C9FC32463B46FBF742
:10CB580079FB00224C4BFBF751FE06460F46024676
:10CB68000B4650465946CDE90EABFBF7A3FF00280C
:10CB780044D032463B4650465946FBF761FB40A33A
:10CB8800D3E90023FBF710FD0026CDE90601EBB23F
:10CB98000EAF0D930A9B9D420ED03046FBF79EFCCC
:10CBA800DDE90623FBF700FD02460B4650465946D1
:10CBB800FBF746FBC7E90001D7E90089DDE9002357
:10CBC80040464946FBF776FFE8B1DDE900234046D9
:10CBD8004946FBF735FBDDE9042380468946FBF728
:10CBE80055FF28B10D9BCDE904890393F3B208934F
:10CBF8000A9B9D420CD1013502347CE752465B46C4
:10CC080030463946B9E74246DDE900014B46E0E7E0
:10CC180001360A2E07F10807BCD1ECE70C9B0B9AEA
:10CC280043EA0220FBF75AFC13A3D3E90023FBF7DE
:10CC3800BBFCDDE90023FBF733FF2C9B10B193F914
:10CC4800000067E7039A9856FBF748FC04460898E3
:10CC58000D46FBF743FC0AA3D3E90023FBF7A4FC2A
:10CC680002460B4620462946FBF7EAFA54E700BF7E
:10CC78006666666666660A40FCA9F1D24D62503F58
:10CC88009A9999999999B93F00408F402DE9704335
:10CC98009DF91860144630461D46FBF71FFCDDE978
:10CCA800082380468946FBF7E7FE002836D1DDE9F0
:10CCB800082340464946FBF7E9FE98B1DDE908013B
:10CCC80042464B46FBF7BCFAFFF7DAFD404240B25A
:10CCD80010F1140F01DB00EAE07000EB8000400067
:10CCE800BDE87083B01EFBF7F9FB02460B46DDE991
:10CCF8000801FBF7CBFE0028EDD0002200232046D8
:10CD08002946FBF7C3FE0028E5D00022054B204644
:10CD18002946FBF797FAFBF7E1FED7E70020BDE8C5
:10CD2800708300BF0000F03FF8B505461846174667
:10CD38000C46FBF7D3FB14A3D3E90023FBF734FC21
:10CD4800FBF7CCFE06B2BDF91800FBF7C7FB0EA334
:10CD5800D3E90023FBF728FCFBF7C0FE00B2304400
:10CD680010F1120F01DB002204E0BC4205DC133095
:10CD780008D00122064B5A5504E0023CBC4201DDB2
:10CD8800002EF0DBF8BD00BF9A9999999999B93F9F
:10CD98007029002000000000F8B500221A4B0C464C
:10CDA80001F100410546FBF7FFFBFBF797FE0A235D
:10CDB80002B292FBF3F003FB102000B2042815DD49
:10CDC800FBF78CFB0EA3D3E90023FBF7EDFB002256
:10CDD80006460F460D4B28462146FBF731FA024618
:10CDE8000B4630463946FBF72DFAF8BDFBF776FBC4
:10CDF80003A3D3E90023FBF7D7FB2A462346F2E730
:10CE08009A9999999999B93F000024400000F03FF8
:10CE18002DE9F04FADF5317D9246BD9A98461278CE
:10CE280083468946BB9B002A40F0C480BA9A684E64
:10CE3800107855785C781A7845EA002596F84330DA
:10CE480096F8440044EA022400EB032000B2FBF702
:10CE580045FB5BA3D3E90023FBF7A6FBAEABC3E915
:10CE680000019BF801309BF800009AF89F7043EA94
:10CE78000020FBF733FB54A3D3E90023FBF794FB13
:10CE88004623544A7F0003FB0823FFB2524600930F
:10CE98003B46FFF739FDFFF77FFFACABC3E9000165
:10CEA800FBF71CFE0FFA80FA4FEA2A2389F80030B4
:10CEB800AEABD3E9000189F801A0FBF70FFE00B281
:10CEC800FBF70CFB24B2AEABC3E900012046FBF72D
:10CED80005FB3BA3D3E90023FBF766FB0B46AEA992
:10CEE8000246D1E90001FBF7ADF9FBF7F7FD2DB2DA
:10CEF80007B22B465246404639460094FFF714FFC6
:10CF08002846FBF7EBFA2EA3D3E90023FBF74CFBEB
:10CF1800ACABD3E90023CDE902237BB202460093F0
:10CF280040460B46FFF7B2FE0544781EFBF7D6FADB
:10CF38000B46ACA9ADB20246D1E900010FFA85F85B
:10CF4800FBF7AEFD28B118F1090FBCBF0A350FFA7F
:10CF580085F8A4B204EB08031BB2C733B8BFC4F505
:10CF68007F486FF0C704BCBF08F138080FFA88F88B
:10CF780008EAE878A045B8BFA046BA9AC8F30723DC
:10CF8800137082F8018014494FF4B07254A807F066
:10CF9800F7FBD6F800807768B568F4684FF4A87294
:10CFA8000E49684607F0ECFB404639462A462346B8
:10CFB800FCF728F90DF5317DBDE8F08FAFF300805F
:10CFC8009A9999999999B93FFCA9F1D24D62503F24
:10CFD800CF380020DF4C00208F400020DF380020B1
:10CFE800F7B5174692F89F40027840780E4640EA17
:10CFF80002201D46FBF772FA0DA3D3E90023FBF7C5
:10D00800D3FA46220C4B640002FB0533E4B23A46DD
:10D0180000932346FFF778FCFFF7BEFEFBF75EFDA3
:10D0280000B203123370707003B0F0BDAFF300802C
:10D03800FCA9F1D24D62503FDF4C00207FB53E4D38
:10D048002B68B3F5FA7F75D93C4C94F83260012E01
:10D0580051D104F58E73039304F14D03029304F147
:10D068001803019304F594730093354A002304F1DF
:10D07800330104F12000FFF7CBFE04F21D130393E4
:10D0880004F14F03029304F11A03019304F5957315
:10D0980000932C4A334604F1350104F12200FFF7CE
:10D0A800B7FE04F58F73039304F15103029304F15F
:10D0B8001C03019304F596730093234A022304F199
:10D0C800370104F12400FFF7A3FE04F21F130393B2
:10D0D80004F15303029304F11E03019304F59773BB
:10D0E80000931A4A032304F1390104F12600FFF7DB
:10D0F8008FFE00232B6016490023A1F11300104A6C
:10D10800FFF76EFF13490123A1F113000D4AFFF742
:10D1180067FF11490223A1F113000B4AFFF760FFD3
:10D1280003230E49094AA1F1130004B0BDE8704079
:10D13800FFF756BF04B070BD382F0020CF3800204D
:10D14800FA4A00209F340020B9310020EF4900201E
:10D15800023900200439002006390020083900204F
:10D168008842AEBF0020081AC0B240B27047000023
:10D178002DE9F04FADF52F7D9A46BA9B0E4693F8F0
:10D1880000905B781746AD930378407800EB032056
:10D1980000B2FBF7A3F968A3D3E90023FBF704FA6D
:10D1A800FBF79CFC0FFA80F89AF800000002FBF7E6
:10D1B80095F904460D469AF80100FBF78FF92246C7
:10D1C8002B46FBF73FF83378824670788B4640EA67
:10D1D800032000B2FBF782F957A3D3E90023FBF73A
:10D1E800E3F9FBF77BFCB99B594693F89F5004B2CF
:10D1F80053A3D3E900235046FBF7D6F94623524AF6
:10D2080003FB0723B99A00932B46FFF755FCFFF75A
:10D21800FBFAFBF763FCB89A4FFA80FB4FEA2B2323
:10D22800137082F801B059464FFA88F0FFF798FF5B
:10D23800D845464D49DAC0F1000A0FFA8AFAA245E4
:10D24800A8BFA246424B33F9172052453DDD23F8CB
:10D2580017A0404B33F91700FBF740F936A3D3E981
:10D268000023FBF7A1F9804650468946FBF736F9BB
:10D2780002460B4640464946FAF7E4FFFBF72EFC08
:10D288000A2300B2434300EB80001B124000707079
:10D2980033704FF4B072304954A807F071FA4FF464
:10D2A800A872D5F800806F68AE68EC6805F11001C7
:10D2B800684607F065FA4046394632462346FBF78A
:10D2C800A1FF0DF52F7DBDE8F08F95F8FC30022BFE
:10D2D800F7D1AD9B43EA092000B2FBF7FFF816A38C
:10D2E800D3E90023FBF760F9FBF7F8FB00B2A04293
:10D2F800E7D0A344D845E4DD0134A4B2144B22B2EC
:10D3080023F817200A23534304EB84041B126400F8
:10D31800747033704FF4B0720F4954A807F030FAA4
:10D32800D5F800806F68AE68EC684FF4A8720B49B6
:10D33800BEE700BFAFF300809A9999999999B93FD0
:10D34800FCA9F1D24D62503F43330020CF38002072
:10D35800B42A0020A82A00208F400020DF380020AF
:10D36800F7B51D4604464B78087892F89F7043EA53
:10D3780000201646FBF7B2F80BA3D3E90023FBF70E
:10D3880013F946220A4B02FB04343B46324600940A
:10D39800FFF792FBFFF738FAFBF7A0FB00B2031286
:10D3A8002B70687003B0F0BDFCA9F1D24D62503FFC
:10D3B80043330020000000002DE9F04F564B87B0A2
:10D3C800197C5A7C554D42EA0122ADF81020997C0F
:10D3D800DA7C42EA0122ADF81220197D5A7D42EA30
:10D3E8000122ADF81420997DDA7D42EA0122ADF8D8
:10D3F80016202A68B2F5FA7F40F2878093F83160E8
:10D40800012E64D10FF20819D9E9008900244FF6DA
:10D418006A7BDFF834A104AF37F914309533B8BF0D
:10D4280027F814B037F91400FBF758F842464B4672
:10D43800FBF7BAF83A4B0022FBF732FB0028034609
:10D4480018BF33460AF804300134042CE4D1354CB3
:10D45800354B00220193A4F1B8030093A4F1E30132
:10D46800A4F1CB0304F10A000294FFF781FE2F4BCD
:10D47800A01C0193A4F1B603029000930122A4F129
:10D48800C903A4F1E10104F10A00FFF771FE231DAD
:10D498000293274B02220193A4F1B4030093A4F151
:10D4A800DF01A4F1C70304F10A00FFF761FEA31D21
:10D4B8000293204B03220193A4F1B2030093A4F139
:10D4C800DD01A4F1C50304F10A00FFF751FE1A4B70
:10D4D800154AA3F113010020FFF742FF174B134A27
:10D4E800A3F113010120FFF73BFF154B104AA3F1ED
:10D4F80013010220FFF734FF124B0E4AA3F1130168
:10D508000320FFF72DFF00232B6007B0BDE8F08F45
:10D518009A9999999999B93FCF380020142F0020EA
:10D5280000002EC0C23900201A4C0020EF3B00201A
:10D53800FF350020823200200A3900200C390020F3
:10D548000E39002010390020DB4C002040F6B7329D
:10D55800914B1968914240F2A180904A1278002AB2
:10D5680000F09C808E4A92F8601041F0100182F819
:10D578006010012182F8EF1040F6B73259689142E5
:10D5880040F29C80854A5278002A00F09780844AAD
:10D5980092F8601041F0200182F86010012182F8B1
:10D5A800F01040F6B7329968914240F297807B4A72
:10D5B8009278002A00F09280794A92F8601041F03F
:10D5C800400182F86010012182F8F110DA6840F613
:10D5D800B7339A4240F29280704BDB78002B00F010
:10D5E8008D806F4B93F8602062F07F0283F8602093
:10D5F800012283F8F22040F6B7326A4B196891424B
:10D6080040F28C80684A1278002A00F08780644AC9
:10D6180092F8601041F0010182F86010012182F84F
:10D62800EB1040F6B7325968914240F287805E4A63
:10D638005278002A00F08280594A92F8601041F02E
:10D64800020182F86010012182F8EC1040F6B7322E
:10D658009968914240F28180534A9278002A7CD09E
:10D668004F4A92F8601041F0040182F860100121DD
:10D6780082F8ED10DA6840F6B7339A427CD94A4B03
:10D68800DB78002B78D0464B93F8602042F00802F4
:10D6980083F86020012283F8EE207047434A11681E
:10D6A80042F20F7291427FF667AF3D4A92F86010DE
:10D6B80021F0100182F8601000215BE73B4A5168B5
:10D6C80042F20F7291427FF66CAF354A92F86010C1
:10D6D80021F0200182F86010002160E7334A916848
:10D6E80042F20F7291427FF671AF2D4A92F86010A4
:10D6F80021F0400182F86010002165E72B4BDA68C1
:10D7080042F20F739A427FF676AF254B93F860206A
:10D7180002F07F0283F8602000226AE7244A116839
:10D7280042F20F7291427FF67CAF1D4A92F8601068
:10D7380021F0010182F86010002170E71C4A51684D
:10D7480042F20F72914281D9154A92F8601021F085
:10D75800020182F86010002176E7154A916842F2CA
:10D768000F72914286D90E4A92F8601021F0040196
:10D7780082F8601000217BE70D4BDA6842F20F73E4
:10D788009A428AD9064B93F8602022F0080283F85F
:10D79800602000227FE700BFB82F00205829002012
:10D7A800CF380020982F002054290020A82F0020CF
:10D7B800882F002040F6B732434B1968914247D969
:10D7C800424A1278002A43D0414A92F8641041F044
:10D7D800010182F86410012182F8131140F6B73272
:10D7E8005968914243D9394A5278002A3FD0384A79
:10D7F80092F8641041F0020182F86410012182F865
:10D80800141140F6B732996891423FD92F4A92785D
:10D81800002A3BD02E4A92F8641041F0040182F8A5
:10D828006410012182F81511DA6840F6B7339A427C
:10D838003BD9264BDB78002B37D0254B93F8642057
:10D8480042F0080283F86420012283F81621704709
:10D85800204A116842F20F729142BFD91C4A92F8CD
:10D86800641021F0010182F864100021B4E7194A1C
:10D87800516842F20F729142C3D9154A92F8641066
:10D8880021F0020182F864100021B8E7114A91687A
:10D8980042F20F729142C7D90D4A92F8641021F0F2
:10D8A800040182F864100021BCE70A4BDA6842F2EE
:10D8B8000F739A42CBD9064B93F8642022F00802E2
:10D8C80083F864200022C0E718300020682900206F
:10D8D800CF380020083000202DE9F04F0328ADF59F
:10D8E800317D0446AC911546AD93BA9F6AD84E4B2C
:10D8F80053F820904D4B33F810804D4B1E5C2B781D
:10D90800022B63D84B4A52F8241047F22F52914207
:10D918005CD9494A125D002A58D1002B56D0012201
:10D928004146484604F01EF90123AC9A1370FF23C0
:10D938003B707B70414B1B681A5D414B1B681A5545
:10D94800404F4FF4B072404954A806F019FF3B68A5
:10D95800D7F804B0AE93D7F808A0FB684FF4A872C4
:10D9680007F110016846AF9306F00AFFAE985946D2
:10D978005246AF9BFBF746FC41F28733334F57F8CB
:10D9880024209A423DD900224146484604F0EAF84C
:10D998000022AC9B1A702B7801332B7047F8242097
:10D9A8002B78032B0AD90423264A2B7092F861306E
:10D9B8001E43012382F86160AD9A13700DF5317D25
:10D9C800BDE8F08F0026B046B14698E71B4B1B68B0
:10D9D8001B5D032BD0D1174B53F824201C4B9A42C4
:10D9E800CAD9154B1B5D002BC6D1012241464846BA
:10D9F80004F0B8F80123AC9A1370FF233B707B70D6
:10DA08009EE70C4B53F8242042F20F739A42D5D963
:10DA18002B78042BD2D00B4A92F8613023EA060601
:10DA280082F861600023C7E7C8580108D858010880
:10DA3800E0580108D82F0020B02A0020D881002003
:10DA4800D07B0020CF3800208F400020E82F002016
:10DA5800DF93040073B51F4C94F80061012E2DD19B
:10DA68001D4D04F58673009504F5827204F10801D2
:10DA78000020FFF731FFAB1C009304F2051204F2FB
:10DA88000D1304F109013046FFF726FF2B1D009303
:10DA980004F5837204F5877304F10A010220063540
:10DAA800FFF71AFF009504F20F1304F2071204F1AE
:10DAB8000B010320FFF710FF02B070BD002384F8AC
:10DAC800613084F80C3184F80D3184F80E3184F813
:10DAD8000F31F1E7CF3800209F4000202DE9F04FAB
:10DAE8001D46032888BF0026ADF5317D9DF8EC3230
:10DAF80088BFB046AE9398BF494B04469CBF53F8C5
:10DB08002080484BAD9198BF33F810602B781746AA
:10DB1800022B5CD8444A52F8201047F22F52914207
:10DB28002ED96BB301223146404604F01BF801237D
:10DB3800AD9A1370FF233B707B703C4B1B681A5DDA
:10DB48003B4B1B681A553B4F4FF4B0723A4954A8E7
:10DB580006F016FE3B684FF4A87207F110016846FC
:10DB6800AF93D7F804B0D7F808A0D7F80C9006F010
:10DB780007FEAF9B5946184652464B46FBF742FBF9
:10DB880041F287332D4F57F824209A4233D9002287
:10DB98003146404603F0E6FF0022AD9B1A702B7811
:10DBA80001332B7047F824202B78032B0BD904233F
:10DBB800204A2B7092F86530AE991943012382F8F8
:10DBC8006510BA9A13700DF5317DBDE8F08F032BFF
:10DBD800D6D1154B53F82020194B9A42D0D901229F
:10DBE8003146404603F0BEFF0123AD9A1370FF2370
:10DBF8003B707B70A7E70C4B53F8242042F20F735D
:10DC08009A42E0D92B78042BDDD00A4AAE9992F8D3
:10DC1800653023EA010382F865300023D1E700BFAD
:10DC2800E4580108F458010828300020AC8200208C
:10DC380020820020CF3800208F400020383000207C
:10DC4800DF93040073B5274C94F81851012D34D193
:10DC5800022604F592730093234A04F58E7304F1A7
:10DC68000C0100200195FFF739FF04F225130093FA
:10DC78001E4A04F21D1304F10D0128460196FFF710
:10DC88002DFF0423019304F593730093184A04F5B8
:10DC98008F7304F10E013046FFF720FF082301932C
:10DCA80004F227130093134A04F21F1304F10F011F
:10DCB8000320FFF713FF02B070BD002384F865301E
:10DCC80084F81C3184F81D3184F81E3184F81F3122
:10DCD80084F8243184F8253184F8263184F82731F2
:10DCE800E9E700BFCF380020A7400020A940002066
:10DCF800AB400020AD40002010B5484B93F8EA2017
:10DD0800002A00F08A8093F83220012A40F08580AA
:10DD1800434A1078012841D142490C6840F6B7318E
:10DD28008C423BD993F8631083F8200141F010012D
:10DD380083F863105078012840D13A494C6840F67E
:10DD4800B7318C423AD993F8631083F8210141F036
:10DD5800200183F86310907801283FD131498C68FD
:10DD680040F6B7318C4239D993F8631083F8220111
:10DD780041F0400183F86310D17801293ED1294A46
:10DD8800D06840F6B732904238D993F8632083F8C8
:10DD9800231162F07F0283F8632010BD22490868CE
:10DDA80042F20F718842C5D993F8631021F010012F
:10DDB80083F86310002183F82011BBE71A494868EB
:10DDC80042F20F718842C6D993F8631021F02001FE
:10DDD80083F86310002183F82111BCE71249886891
:10DDE80042F20F718842C7D993F8631021F04001BD
:10DDF80083F86310002183F82211BDE70A4AD1682D
:10DE080042F20F72914208D993F8632002F07F0220
:10DE180083F86320002283F8232110BDCF38002027
:10DE2800702900204C2F00203C2F002010B54A4AB2
:10DE380092F8EA101346002900F08D8092F831001C
:10DE4800012840F08380454A1178002944D044498C
:10DE58000C6840F6B7318C423ED993F8621083F8CB
:10DE6800080141F0100183F862105178002943D06D
:10DE78003B49486840F6B73188423DD993F862106B
:10DE880041F0200183F86210012183F8091191788B
:10DE980000293FD03249886840F6B731884239D9DD
:10DEA80093F8621041F0400183F86210012183F871
:10DEB8000A11D278002A3BD0294AD16840F6B732F5
:10DEC800914235D993F8622062F07F0283F862208C
:10DED800012283F80B2110BD2249086842F20F7114
:10DEE8008842C2D993F8621021F0100183F86210B9
:10DEF800002183F80811B8E71A49486842F20F71FF
:10DF08008842C4D993F8621021F0200183F8621086
:10DF18000021BAE71349886842F20F718842C8D9CC
:10DF280093F8621021F0400183F862100021BEE7E7
:10DF38000C4AD16842F20F7291420CD993F86220D0
:10DF480002F07F0283F862200022C2E7002382F8F1
:10DF5800623082F80B3110BDCF380020DB4C002036
:10DF6800282F0020182F0020154B93F8EA202AB3F9
:10DF780093F9582093F930108A420FDC012283F874
:10DF8800CA20104A116840F6B832914216D993F85F
:10DF98005F2062F07F0283F85F200FE093F85F0054
:10DFA80080280BD1013A8A4208DD07490022086817
:10DFB80042F21071884283F8CA20ECD8704700BF3B
:10DFC800CF3800207C2F0020782F002038B50B7820
:10DFD80013B3124B53F82020114B9A421CD9032833
:10DFE80088BF00234FF0000287BF1C461D460D4B1B
:10DFF8000D4C9CBF33F810500C4B0A7098BF33F887
:10E0080010302046194603F0ADFD29462046BDE8EC
:10E018003840012203F0A6BD38BD00BF50300020B3
:10E028003F771B00FC5801080020014004590108F3
:10E0380003282DE9F0470E4688BF0021174698BFF0
:10E04800364AADF52C7D9FBF32F81080344A354DE5
:10E0580032F8101084BF88460D46012EB49C4FEA52
:10E068004002DFF8CCC0DFF8CCE042D193F8009052
:10E0780001320CF8109093F801900CF802904FF0D0
:10E08800000994F800C00EF810C060780EF802007D
:10E0980083F8009083F80190324684F8009084F861
:10E0A8000190284603F05EFD4A461F4C414628462B
:10E0B80003F058FD4FF4B0721C4954A806F060FBF9
:10E0C800D4F800A0D4F80490D4F80880E56804F1E6
:10E0D80010014FF4A872684606F052FB50464946B4
:10E0E80042462B46FBF78EF83E700DF52C7DBDE8B9
:10E0F800F0871CF81090013283F800901CF802C0D9
:10E1080083F801C01EF81030284623701EF802302C
:10E118000022637003F026FD0122C6E7FC580108BF
:10E128000459010800200140CF3800208F4000200A
:10E13800CA2A0020D22A00202DE9F0434378ADF501
:10E148002D7D0446BE2B00F2AC84DFE813F0E0001E
:10E15800AA04AA04AA04AA04AA04AA04AA04AA0447
:10E16800AA04AA04AA04AA04AA04AA04AA04AA0437
:10E17800AA04BE01AA04AA04AA04D001AA04E601BA
:10E18800AA04AA04AA04AA04AA04AA04AA04AA0417
:10E19800AA04F001AA04AA04AA040002AA04140208
:10E1A800AA04AA04AA04AA04AA04AA04AA04AA04F7
:10E1B800AA041C02AA04AA04AA044B02AA045B0229
:10E1C800AA04AA04AA04AA04AA04AA04AA04AA04D7
:10E1D800AA046302AA04AA04AA047202AA04830273
:10E1E800AA04AA04AA04AA04AA04AA04AA04AA04B7
:10E1F8006803AA04AA04AA04AA04AA04AA04AA04EA
:10E20800AA04AA04AA04AA04AA04AA04AA04AA0496
:10E218005E03AA04AA04AA04AA04AA04AA04AA04D3
:10E22800AA04AA04AA04AA04AA04AA04AA048B0297
:10E238008E02AA04AA04AA04AA04AA04B402DB024D
:10E24800AA04AA04AA04AA04AA04AA04AA04E00222
:10E25800E802F002F802000315033E034E03DC0354
:10E2680072037A038B0390039803AA04A303AB03F6
:10E27800C503D703DC03E103E603EF03F703030455
:10E288000B0419041E042604AA043404E400020141
:10E298000B0114011D0164017D019201AA04AA0465
:10E2A800AA04AA04AA04AA04AA04AA0442044A04BE
:10E2B80052045A046204720476048004D800870465
:10E2C800BF00910496049B04A004A5044279B64BB0
:10E2D80083F8E520827983F8E620C27983F8E7207D
:10E2E8004FF4B072B049B148FAF774FD4FF4B07307
:10E2F800AE4A4FF42E61A02001F04AFFD6E14279E0
:10E30800A94B83F8CE20827983F8CF20E8E7FCF781
:10E318003FFAFAF72BFC00224379A34D2B7483793B
:10E328006B74A34B1A804FF4B072A24954A806F03C
:10E3380027FAD5F800806F68AE684FF4A87205F127
:10E3480010016846EC6806F01BFA4046394632462A
:10E35800B9E000224379944DAB748379EB74944B04
:10E368005A80E0E7002243798F4D2B7583796B75CE
:10E378008F4B9A80D7E7002243798B4DAB75837911
:10E38800EB758B4BDA80CEE7874B42791C461A76C1
:10E3980082795A7693F83220012A09D1864B1A706D
:10E3A80094F8332094F8343043EA0223834A1380E4
:10E3B80054AD4FF4B0727F49284606F0E1F9D4F81D
:10E3C8000090D4F80480A768E6684FF4A8727C49E6
:10E3D800684606F0D5F9484641463A463346FAF7C4
:10E3E80011FF4FF4B0722846724906F0C9F9276840
:10E3F8006668A568E4684FF4A8727149684606F033
:10E40800BFF92A46234638463146FAF7FBFE002272
:10E418006C4B1A6064E7644B42791C469A768279A1
:10E42800DA7693F83220012A09D1634B5A7094F8AE
:10E43800352094F8363043EA0223604A53804FF47B
:10E44800B0725C4954A8D0E7574B42791C461A77FA
:10E4580082795A7793F83220012AF0D1564B9A7074
:10E4680094F8372094F8383043EA0223534A9380CB
:10E47800E5E74D4B42791C469A778279DA7793F82B
:10E488003220012A09D14C4BDA7094F8392094F8DB
:10E498003A3043EA0223494AD3800022494B45498E
:10E4A8001A6054A84FF4B07206F06AF927686668D3
:10E4B800A5684FF4A87242496846E46806F060F916
:10E4C800384631462A4623467CE1374A92F8EA30F4
:10E4D800002B00F0EB80417902F58270009000205B
:10E4E800394B08320193F43BFDF70EFAF8E62E4D4E
:10E4F80095F8EA30002B00F0D980344B05F58E7280
:10E50800417901930092A3F5827305F10C02002072
:10E51800FDF74AFA63792B73E2E6417900202C4A29
:10E528000092A2F10803143AFFF782FDD8E61E4ACA
:10E5380092F8EA30002B00F0B980264B417902F2BC
:10E54800051001930090F33B09320120CCE7164AED
:10E5580092F8EA30002B00F0A98041796FF48174B9
:10E5680002F21D10009001201B4B0D320193234431
:10E57800FDF71AFAB4E6194A4179A2F108030092A4
:10E588000120153AD0E7084A92F8EA30002B00F04B
:10E598008D80134B417902F5837001930090F23B13
:10E5A8000A320220A0E700BFCF3800208F3A0020AF
:10E5B800B42A00208F4000209B3400207A320020AB
:10E5C800DF380020382F002093410020AB41002085
:10E5D800E738002094410020AC410020E9380020B1
:10E5E80095410020B34A92F8EA30002B5ED0B24B36
:10E5F800417902F58F7001930090A3F581730E3273
:10E608000220B5E7AD4A4179A2F108030092022041
:10E61800163A89E7A74A92F8EA30002B46D0A84B69
:10E62800417902F2071001930090F13B0B3203206D
:10E638005AE7A04A92F8EA30002B37D0417902F223
:10E648001F1000906FF480709E4B0F3201930344AB
:10E6580003208DE79C4A4179A2F108030092032028
:10E66800173A61E74179FBF745FA61792046FBF7EC
:10E67800BFF87123E1786370601C01F091F8E378CA
:10E68800020A23445A70EB22E378904D2344987091
:10E69800E37821462344DA70E27828460432FAF710
:10E6A80099FB2846E978043102F0D8FA01200DF5E3
:10E6B8002D7DBDE8F083864C237843B9FCF73EFAFC
:10E6C8000A2002F0F7FAFAF743FC012323707F4C83
:10E6D800FCF7BCF94FF4B07276492046FAF77AFB9A
:10E6E8000123A3705C234FF4AE71601CE37001F04A
:10E6F80057F8030A84F85E0184F85D314FF4B0716D
:10E708002046D1E76021A02001F09AFD01E6437977
:10E71800684D85F84530837985F8463003E64379B6
:10E72800644D85F84730837985F84830FBE54379AF
:10E73800604D85F84930837985F84A30F3E54379A7
:10E748005C4D85F84B30837985F84C30EBE54279A0
:10E75800584D85F84D20837943EA02236FF0310242
:10E768001BB29342B8BF134603EAE3731A1285F843
:10E778004D2085F84E30D6E542794E4B83F84F2030
:10E78800D20908BF002281790ABF83F8502083F894
:10E79800501083F84F20474C4FF4B0724D4954A89D
:10E7A80005F0EEFFD4F800806768A668E5684FF4C6
:10E7B800A87204F11001684605F0E2FF40463946A8
:10E7C80032462B46FAF71EFD8AE54279394B83F823
:10E7D8005120D20908BF002281790ABF83F852204C
:10E7E80083F8521083F85120D5E74279314B83F8EA
:10E7F8005320D20908BF002281790ABF83F8542028
:10E8080083F8541083F85320C5E74379294A82F8DE
:10E818003130002B7FF464AD82F8623060E54379D3
:10E82800244A82F83230002B7FF45AAD82F86330E4
:10E8380056E542791F4B83F8FD20827983F8FE2044
:10E848004EE542791B4B012A83F8FF207FF448AD3F
:10E85800FF2283F8FD20F62283F8FE20002283F8A9
:10E86800FF203DE54279134B83F8002138E54279D2
:10E87800104B83F80121827983F8022130E542792F
:10E888000C4B012A83F803217FF42AADFF2283F879
:10E898000121F1E74279074B83F85A20827983F8FE
:10E8A8005B201DE54279034B83F85C20827983F86D
:10E8B8005D2015E5CF380020AD410020EB38002061
:10E8C80096410020AE410020ED3800208F3C00200A
:10E8D800BA4C00208F4000204279794B012A83F8F6
:10E8E8005E207FF4FDAC002283F85A20072283F8CB
:10E8F8005B20FF2283F85C20D522D8E74279704B51
:10E9080083F8CB20D2E642796D4B83F85720E7E4B1
:10E9180042796B4B83F85820E2E490F90520684B64
:10E92800012A08BF502283F85920D9E44279644B60
:10E9380083F81021827983F81121D1E44279604B60
:10E94800012A83F812217FF4CBACFF2283F810212F
:10E95800EE22F0E742795A4B83F84320827983F814
:10E968004420BDE44279564B83F8172193F81221CD
:10E97800012A7FF4B5ACFF2283F84320D822EEE7C2
:10E9880042794F4B83F81821AAE442794C4B83F81B
:10E998001921827983F81A21A2E44279484B83F835
:10E9A8001B2193F81221012A7FF49AACFF2283F8E5
:10E9B8001921F022EEE78079F9F790FD3EA3D3E91B
:10E9C8000023F9F7F1FDFAF7B1F83D4B83F866003B
:10E9D80086E443793A4D85F82831837985F82931D9
:10E9E800A1E44379364D85F82A31837985F82B31AE
:10E9F80099E44379324D85F82C31837985F82D31A6
:10EA080091E443792E4D85F82E31837985F82F319D
:10EA180089E442792A4B032A83F875207FF460AC95
:10EA280093F87420012A0CBF0222012283F8752072
:10EA380056E40430FDF728F952E44379204A012BC3
:10EA480082F8C9307FF44CACFCF7F8FF48E4407911
:10EA58001B4B83F8EA00FDF74BF941E4194A031D03
:10EA6800183413F8011F9C4202F8011FF9D137E44A
:10EA78004279134B83F8582132E44279104B83F8DA
:10EA88005B212DE442790E4B83F85C2128E442791E
:10EA98000B4B83F85D2123E44279094B83F85E210F
:10EAA8001EE4772B3FF402AE922B3FF4FFAD703B90
:10EAB800012B3FF615ACF9E59A9999999999B93FBF
:10EAC800CF3800209E3900202DE9F04F0646847C7F
:10EAD800ADF52F7D0B30FDF7D7F88D4B00221D4685
:10EAE800B15CD1540132B2F5006FF9D11622F12090
:10EAF8001A705A709A70DA700022D97C93F81480D0
:10EB08001A7158715A74A4B9824C23782BB9FCF73E
:10EB180015F8FAF71DFA01232370FBF7A7FF8023E6
:10EB28007B48AB74FCF714F901200DF52F7DBDE887
:10EB3800F08F012C40F08E84774C784E48EA0128FB
:10EB480004F11007EB7D013B8E2B00F29A80DFE881
:10EB580013F0BA00CA00CE00980098009800E900A7
:10EB68009800980098009800980098000F011401E8
:10EB780098001A011E0122019800240198009800AB
:10EB8800B300280198008F003201980098003801DE
:10EB980098009800980098009800980098009800AD
:10EBA800980098009800980098009800980098009D
:10EBB8003E0157016E0185019C01BF01C701CF01CC
:10EBC800D701DE01E501EC01F301FA010102980029
:10EBD800980098009800980098009800980098006D
:10EBE800980098000C0298009800980098009800E7
:10EBF80017027C0283028802A302AA0298009800E6
:10EC0800980098009800980098009800980098003C
:10EC1800AF02CA02E402FD02170341036D03990320
:10EC2800C503CC03D303DA03FF0398000604980056
:10EC380098009800980098000B0415041D042504FA
:10EC480098009800980098009800980098009800FC
:10EC58002D0436043D04420446044D0498009800EF
:10EC6800980098009800980098009800980052041E
:10EC78006B7E84F8E530AB7E84F8E630EB7E84F872
:10EC8800E7302B7E264A995CE02940F0CE83B8F124
:10EC9800000F00F0CA83C3F57F43FD339844002377
:10ECA8001FFA88F84345BFF64DAF297E1944505CDA
:10ECB800E91888750133F5E76B7E84F8CE30AB7EB2
:10ECC80084F8CF30DDE76B7E84F86630AB7E84F85D
:10ECD8006730EB7E84F868302B7F84F869306B7F6F
:10ECE80084F86A30CDE76B7E84F86B30C9E76B7EB9
:10ECF80084F86C30AB7E84F86D30EB7E84F86E302F
:10ED08002B7F84F86F306B7F84F87030B9E700BFD1
:10ED1800EF410020BA4C0020CF3800208F4000205F
:10ED2800084200206A7EB04B032A83F8752007D179
:10ED380093F87420012A0CBF0222012283F875205F
:10ED48004FF4B072A849A948FAF744F84FF4B073E1
:10ED5800A64A4FF42E61A02001F01AFA4FF4B073BE
:10ED6800A14A4FF42E61A02001F0E0F8F9F7FEFE69
:10ED78006A7E9D4B83F8C820F8E76B7E84F8C9301B
:10ED8800FCF75CFE7DE76B7E84F8573079E76B7E95
:10ED980084F8583075E75023FAE76B7E84F8CB3057
:10EDA8006FE70023E9181A19497E0133142B82F8FA
:10EDB800D010F7D165E7687E86F85901FDF7CCF8E1
:10EDC8005FE7687E84F8EA00FCF792FF59E794F859
:10EDD800EA30002B3FF4A8AE697E61B180230020A1
:10EDE80084F85A31824A834B00920193FC3AF43BEF
:10EDF800FCF78AFD45E794F85A3103F07F03EEE704
:10EE080094F8EA30002B3FF48FAE697E51B140236D
:10EE180084F85A31784A794B00920193FC3AF33BD3
:10EE28000120E5E794F85A3123F04003F0E794F81D
:10EE3800EA30002B3FF478AE697E51B1202384F884
:10EE48005A316F4A6F4B00920193FC3AF23B022011
:10EE5800CEE794F85A3123F02003F0E794F8EA302B
:10EE6800002B3FF461AE697E51B1102384F85A310A
:10EE7800654A664B00920193FC3AF13B0320B7E7E1
:10EE880094F85A3123F01003F0E700226B7E2374C4
:10EE9800AB7E63745E4B1A8031464FF4B07254A84F
:10EEA80005F06EFC236839464FF4A8726846AD93A6
:10EEB800D4F804B0D4F808A0D4F80C9005F060FC9D
:10EEC800AD9B5946184652464B46FAF79BF9D8E689
:10EED80000226B7EA374AB7EE3744D4B5A80DBE754
:10EEE80000226B7E2375AB7E6375494B9A80D3E70E
:10EEF80000226B7EA375AB7EE375454BDA80CBE7CA
:10EF08006B7E84F84530AB7E84F84630C4E76B7E70
:10EF180084F84730AB7E84F84830BDE76B7E84F8D0
:10EF28004930AB7E84F84A30B6E76B7E84F84B30C4
:10EF3800AB7E84F84C30AFE76B7E84F85A30AB7EFA
:10EF480084F85B309DE66B7E84F85C30AB7E84F899
:10EF58005D3096E6002384F85A30462384F85B3007
:10EF6800FE2384F85C305223F1E76B7E84F8FB3093
:10EF780023B9284A137084F8FC3082E60123FAE7A3
:10EF88006B7E84F83130002B4ED1234A234813700E
:10EF980053709370D3701A4621491A545A54013346
:10EFA800062BFAD11B4B84F8FC201A7084F86220D7
:10EFB800217C627C1B4B42EA01221A80A17CE27C04
:10EFC80042EA01225A80217D627D42EA01229A802A
:10EFD800A17DE27D42EA0122DA8000220C4B1A80F0
:10EFE8005A809A80DA804CE6CF3800208F3A002089
:10EFF800D339002093410020D439002094410020C7
:10F00800D539002095410020D639002096410020AE
:10F01800B42A0020D8300020DB4C0020BC2A002075
:10F02800C32A0020A82A0020BA4BEA7A1A702A7B41
:10F038005A706A7B9A70AA7BDA70EA7B1A712A7C0A
:10F048005A710122B44B1A70B2E76B7E84F8FD3016
:10F05800AB7E84F8FE3014E6FF2384F8FD309C2351
:10F06800F7E76B7EDFF8E4E284F8003100231A4604
:10F07800AA48AB4984F8043184F8053184F806318C
:10F0880084F807314EF8232040F8232041F8232044
:10F098000133042BF6D1F4E56B7E84F80131AB7EA5
:10F0A80084F80231EDE5FF2384F80131F623F7E710
:10F0B80094F8EA30002B3FF437AD697E71B108232C
:10F0C800002084F85A31974A974B00920193A2F591
:10F0D8008872A3F58273FCF767FCD2E594F85A317D
:10F0E80023F00803ECE794F8EA30002B3FF41CAD5A
:10F0F800697E69B104236FF4817E84F85A318B4AA2
:10F108008B4B00920193A2F5887273440120E2E7C9
:10F1180094F85A3123F00403EDE794F8EA30002B11
:10F128003FF402AD697E61B1022384F85A31814A05
:10F13800814B00920193A2F58872A3F58173022096
:10F14800C9E794F85A3123F00203EEE794F8EA305D
:10F15800002B3FF4E9AC697E69B101236FF480703C
:10F1680084F85A31754A764B00920193A2F5887259
:10F1780003440320AFE794F85A3123F00103EDE785
:10F1880094F83230697EAA7E012B217662767FF46C
:10F1980083AE94F8280194F8293142EA012243EA1F
:10F1A80000231BB212B21A44C73207DAC3F57F43F1
:10F1B80038339BB243F30722227663760122614BF0
:10F1C8001A7094F8332094F8343043EA02235E4AE4
:10F1D800138061E66B7EA376AB7EE37694F83230DB
:10F1E800012B7FF459AE94F8282194F82931217E17
:10F1F80043EA0223627E1BB242EA012212B21A4497
:10F20800C73207DAC3F57F4338339BB243F307228B
:10F218002276637601224B4B5A7094F8352094F885
:10F22800363043EA0223484A538035E66B7E23771B
:10F23800AB7E637794F83230012B7FF42DAE94F8CF
:10F24800282194F82931217E43EA0223627E1BB2E9
:10F2580042EA012212B21A44C73207DAC3F57F43E1
:10F2680038339BB243F30722227663760122354B6B
:10F278009A7094F8372094F8383043EA0223324AD7
:10F28800938009E66B7EA377AB7EE37794F8323000
:10F29800012B7FF401AE94F8282194F82931217EBE
:10F2A80043EA0223627E1BB242EA012212B21A44E6
:10F2B800C73207DAC3F57F4338339BB243F30722DB
:10F2C8002276637601221F4BDA7094F8392094F87D
:10F2D8003A3043EA02231C4AD380DDE56B7E84F88A
:10F2E8004D30AB7E84F84E30D6E56B7E84F84F30D7
:10F2F800AB7E84F85030CFE56B7E84F85130AB7E1E
:10F3080084F85230C8E56B7E84F85330AB7E84F8BD
:10F318005430C1E5DA2A0020D8300020E82F002038
:10F32800C82F0020EB390020AB410020EC39002029
:10F33800AC410020ED390020AD410020EE3900201D
:10F34800AE4100209B3400207A320020D82F0020C4
:10F358006B7E84F81031AB7E84F8113191E4FF2381
:10F3680084F810314C23F7E70020864A697EA2F121
:10F3780008030092143AFEF75BFE82E4824A697E33
:10F38800A2F1080300920120153AF4E77F4A697E4A
:10F39800A2F1080300920220163AECE77C4A697E43
:10F3A800A2F1080300920320173AE4E76B7E84F881
:10F3B8003230002B7FF465AC84F8633061E46B7EF7
:10F3C80084F84330AB7E84F844305AE4FE2384F852
:10F3D80043307023F7E76B7E84F8183151E46B7E75
:10F3E80084F81931AB7E84F81A314AE4FF2384F893
:10F3F80019316023F7E76B7E84F82831AB7E84F8F7
:10F408002931EB7E84F82A312B7F84F82B316B7FEE
:10F4180084F82C31AB7F84F82D31EB7F84F82E31C2
:10F4280095F8203084F82F3136E581235948AB749C
:10F43800FBF78EFC4FF4B07257495848F9F7CAFCED
:10F448004FF4B073554A4FF42E61A02000F0A0FE8F
:10F45800FFF76ABB402C62D1197E232936D82029B0
:10F4680006D2032904D9A1F11003032B3FF65CABA4
:10F478004848FAF7F5FD2B7E494C3F2BA97E04F14D
:10F48800010704F102062BD9AB78532B28D8053194
:10F49800A4F11B0000F0ACF9A4F11B0000F05FF927
:10F4A800A97E68750531601F00F07AF9AB7E020A03
:10F4B800E2540322AB7EF854AB7EA4F11B00F25455
:10F4C800A97E1E3101F0CAFBFFF72EBB432904D8E1
:10F4D8004029CDD2A1F13003C7E7A1F15003C4E719
:10F4E800490005312B4800F083F92A4800F037F924
:10F4F800A97E6875490005312A4800F051F9AB7EAC
:10F50800020A04F813200322AB7E07F81300AB7E2F
:10F5180006F81320A97E490020311E48D2E7412C65
:10F528002BD1197E23291ED8202906D2032904D9D4
:10F53800A1F11003032B3FF6F7AA1648FAF7D2FEFB
:10F548000121144800F054F9124800F008F901218B
:10F558006875144800F024F9030AEB75032328762C
:10F568006B761A21D9E7432904D84029E5D2A1F1BD
:10F578003003DFE7A1F15003DCE7064800F0A4F907
:10F58800FFF7D2BAE7380020E9380020EB3800202E
:10F59800ED380020EF410020CF3800208F3A0020BE
:10F5A8000A4200200542002010B5094C00202146DF
:10F5B800FEF70CFD611C0120FEF708FDA11C0220CE
:10F5C800FEF704FDE11C0320BDE81040FEF7FEBC79
:10F5D800D338002010B5234C94F8FB3013B194F8BD
:10F5E80031201AB9002384F8FC3010BD1E4A127865
:10F5F8009A4214D11D4A1E4BD178D87888420ED32E
:10F608001179187988420AD352795B79934206D3E3
:10F6180094F8FC30012B04BF022384F8FC3094F8E2
:10F62800FC30012B1DD1237A23B1124901F1E300EB
:10F63800F9F7AEFA637A23B10F4901F1E300F9F75C
:10F64800A7FAA37A23B10D4901F1E300F9F7A0FA6B
:10F65800E37A33B1BDE81040094901F1E300F9F755
:10F6680097BA10BDCF380020D8300020DA2A002001
:10F67800BC2A0020DF380020E1380020E3380020D1
:10F68800E5380020234A244992F86B00134670BBE2
:10F6980092F85F2012B193F866201ABB93F86020A5
:10F6A80012B193F86720EAB993F8612012B193F880
:10F6B8006820BAB993F8622012B193F868208AB921
:10F6C80093F8642012B193F869205AB993F863202B
:10F6D80012B193F86A202AB993F865202AB193F8F1
:10F6E8006A3013B101230B7070470023FBE792F8CF
:10F6F8006C30002BF6D192F86D30002BF2D192F8D5
:10F708006E30002BEED192F86F30002BEAD192F8D0
:10F718007030E6E7CF3800202233002008B5FFF725
:10F72800B1FFFEF721FCFEF781FBFEF7E5FAFEF7D5
:10F7380089FAFEF78FF9FDF709FFBDE80840FEF7E3
:10F7480039B8002310B5C11C143011F8014F2344F7
:10F758008142DBB2F9D19B1A5842584110BDC21CF4
:10F7680000F11403002012F8011F08449A42C0B2A5
:10F77800F9D17047002330B5084D0144884203D1C0
:10F788009B1A5842584130BD10F8014B84EA1324A3
:10F7980035F8144084EA03239BB2EFE73459010893
:10F7A800002310B5074C0144884201D1184610BD0A
:10F7B80010F8012B82EA132234F8122082EA03237C
:10F7C8009BB2F1E7345901084FF0FF3210B5074CEE
:10F7D8000144884201D1D04310BD10F8013B534089
:10F7E800DBB254F8233083EA1222F2E7345B0108D3
:10F7F8002DE9F04101F1200323F0070300AFADEB41
:10F80800030D04460E46FFF7CBFF0DEB0603020A75
:10F818009A750322D8751A7616238DF800308DF85C
:10F8280001308DF802308DF80330F12300258DF872
:10F838000530A3798DF804508DF80630E3798DF8FA
:10F8480011508DF80730237A68468DF80830637AAE
:10F85800E8468DF80930A37A8DF80A30E37A8DF8F6
:10F868000B30237B8DF80C30637B8DF80D30A37B38
:10F878008DF80E30E37B8DF80F30237C8DF8103037
:10F88800A37C8DF814608DF81230330A8DF813308C
:10F89800FFF765FF2B468DF81500122B1CBF18F8D3
:10F8A8000320E2540133162BF7D100230133042B34
:10F8B80003D12046BD46BDE8F0819A19A1184244FB
:10F8C800527D4A75F2E70000F8B5837C0446103B88
:10F8D800032B00F2D581DFE813F004006E00A500C9
:10F8E8003A010025FF26C44BC44F1D70C44BC548C0
:10F8F8001D60C54B3D701E6004F0DEFF0122032130
:10F90800C24BA27683F85921E17625776577A577EA
:10F91800E57784F8205084F8215093F874103D70EE
:10F928009142BB493ED102220A703246591901352B
:10F93800292D81F89F20F9D10C259026A674204600
:10F948002946FFF755FF0023B24C05F118029342F0
:10F9580040F3478129461630FFF722FF19352C441A
:10F96800030A04F8020C2946AA4804F8033C01F0EB
:10F9780075F9932E40F03981A44B93F85931012B36
:10F9880040F03381642001F095F9BFF34F8FA2490D
:10F99800A24BCA6802F4E0621343CB60BFF34F8FF7
:10F9A80000BFFDE70A70324659190135292D81F843
:10F9B8007620F9D1C0E7837EC17E027F1B06407F97
:10F9C800090443EA01050B441202054303441344A6
:10F9D80015438B4A8C4E13600023A377E37784F892
:10F9E800203084F8213033689D420BD0884B4FF487
:10F9F80080611A7804F1220001F014F835600C25B2
:10FA080091269BE7864A874B11688748994205F5F6
:10FA1800003394BF03F59073A0339B02136004F086
:10FA28004BFFEBE77A4B1B78012B7FD17F4A804B4A
:10FA380011781B78090441EA03617E4B7E481B78E4
:10FA480019437E4B1B7841EA03218031FFF7A8FE5A
:10FA5800A27EE37E784943EA022398421CBF012232
:10FA6800664BE07518BF1A70030AA3750123237645
:10FA78000023A3766376E3762377CA7A634B704EC6
:10FA880083F876200A7B83F877204A7B83F87820EE
:10FA98006C4AD07A83F89F00107B83F8A000507BD3
:10FAA80083F8A10091F8370083F8790091F83800BD
:10FAB80083F87A0091F8390083F87B0091F83A00CE
:10FAC80083F87C0091F83B0083F87D0091F83C10A6
:10FAD80083F87E1092F8371083F8A21092F8381045
:10FAE80083F8A31092F8391083F8A41092F83A100A
:10FAF80083F8A51092F83B1083F8A61092F83C20E2
:10FB0800514983F8A720514A5578901901328A4201
:10FB18001D54F9D14E4A4F4E4F495578901901322C
:10FB28008A421D54F9D10725922607E74B4A4C4BC8
:10FB380011781B78090441EA03614A4B41481B7854
:10FB48001943494B1B7841EA032180317EE72B4B4F
:10FB58001B78002B3FD101238375444804F0ACFE89
:10FB68000123E375374B294E93F8372096F85971DE
:10FB780086F8A22093F83820012F86F8A32093F85E
:10FB8800392086F8A42093F83A2086F8A52093F81F
:10FB98003B2086F8A62093F83C2086F8A720DA7A3E
:10FBA80086F89F201A7B86F8A0205B7B86F8A13018
:10FBB80015D102252E4804F07FFE96F87430012BEB
:10FBC8000BBF2C482C4886F8755086F8757004F0E1
:10FBD80073FE9326B2E6002383752848BEE7022504
:10FBE800F7E7C15CE1540133B1E6094B1878BDE889
:10FBF800F84000F079BE00BFF42E0020EA2A002069
:10FC0800EC2A0020345F010800280020CF380020AB
:10FC1800E92A0020204E002000ED00E00400FA054B
:10FC280000570020FF7F04084C5F01083E8002084F
:10FC38003D80020840800208008002083F800208D8
:10FC48007280FDF7008004082D8002080D800208EC
:10FC58000D8004089B80FBF72D8004083E80040873
:10FC68003D800408408004083F8004085A5F01086A
:10FC7800755F01089D5F0108BA5F0108685F0108A8
:10FC8800F8BD00BF70B52C4C2C4E25460FCE0FC5C5
:10FC980096E803002A4E85E803000FCE04F11C0500
:10FCA8000FC596E80300274E85E803000FCE04F140
:10FCB80038050FC596E80300234E85E803000FCEEC
:10FCC80004F154050FC596E80300204E85E80300AB
:10FCD8000FCE04F170050FC596E803001C4E85E8A9
:10FCE80003000FCE04F18C050FC596E80300194EEA
:10FCF80085E803000FCE04F1A8050FC596E80300B8
:10FD0800154E85E803000FCE04F1C4050FC596E82B
:10FD18000300002385E80300237684F8343084F850
:10FD2800503084F86C3084F8883084F8A43084F833
:10FD3800C03084F8DC3070BD205600200428002034
:10FD4800642800201C2800207C280020342800205B
:10FD5800942800204C280020AC2800202DE9F047EA
:10FD680004460D4608274FF0400A00264FF00008C9
:10FD7800DFF868900022002320462946F8F77CFE29
:10FD880018BB0022134B20462946F8F77FFEF8B12E
:10FD980042464B4620462946F8F78CFE48B1204695
:10FDA800294642464B46F8F74BFA04460D4646EAC2
:10FDB8000A06404649460022074BF8F7F5FB013F83
:10FDC800804689464FEA5A0AD4D13046BDE8F087C2
:10FDD8007F26FAE700403F400000E03F0000304047
:10FDE80084B02DE9F84F0AAC84E80F000E9EBDF8E8
:10FDF8003C7000223946824630469DF84050BDF896
:10FE08002CB0DDF83080BDF8349001F0ABFE0A204C
:10FE180003F0D6FA082415F0010218BF012249465A
:10FE2800404601F09FFE01225946504601F09AFED5
:10FE38000A2003F0C5FA00225946504601F092FE06
:10FE4800013C0A2003F0BCFA14F0FF044FEA550500
:10FE5800E1D122465946504601F084FE22464946E1
:10FE6800404601F07FFE0A2003F0AAFA3946012233
:10FE7800304601F077FE0A2003F0A2FA22463946FE
:10FE88003046BDE8F84F04B001F06CBE70B50022F2
:10FE98004FF400510546244801F064FE0A2003F09F
:10FEA8008FFA0824204E15F0010218BF01224FF4E2
:10FEB8000061304601F056FE01224FF480611A4875
:10FEC80001F050FE0A2003F07BFA00224FF4806113
:10FED800154801F047FE013C0A2003F071FA14F0BE
:10FEE800FF044FEA5505DED122464FF480610E48E3
:10FEF80001F038FE22464FF400610B4801F032FE53
:10FF08000A2003F05DFA01224FF40051064801F07F
:10FF180029FE0A2003F054FA2246BDE870404FF447
:10FF28000051014801F01EBE001801401FB54FF6F0
:10FF3800FF748DE81C000A4610230146024802F0AF
:10FF48001FF904B010BD00BFE07B002010B5774C4E
:10FF58004FF4B07322464FF42E61A020FFF7E6FF5E
:10FF68006023734A1946A020FFF7E0FF6023714A17
:10FF7800C021A020FFF7DAFF60236F4A4FF4907189
:10FF8800A020FFF7D3FF60236C4A4FF4C071A02074
:10FF9800FFF7CCFF60236A4A4FF4F071A020FFF707
:10FFA800C5FF6023674A4FF41071A020FFF7BEFF1A
:10FFB8006023654A4FF42871A020FFF7B7FF60233C
:10FFC800624A4FF44071A020FFF7B0FFA023604AB7
:10FFD8004FF458711846FFF7A9FFA0235D4A4FF464
:10FFE80080611846FFF7A2FFA0235B4A4FF4946193
:08FFF8001846FFF79BFFA02350
:020000040801F1
:10000000584A4FF4A8611846FFF794FFA023564AB8
:100010004FF4BC611846FFF78DFFA023534A4FF4FD
:10002000D0611846FFF786FFA023514A4FF4E461E0
:100030001846FFF77FFFA0234E4A4FF4F861184699
:10004000FFF778FF20234C4A4FF40661A020FFF70A
:1000500071FF2023494A4FF40861A020FFF76AFF8F
:100060002023474A4FF40A61A020FFF763FF2023B3
:10007000444A4FF40C61A020FFF75CFF2023424A62
:100080004FF40E61A020FFF755FF20233F4A4FF4A5
:100090001061A020FFF74EFF20233D4A4FF412616C
:1000A000A020FFF747FF20233A4A4FF41461A02015
:1000B000FFF740FFF8F716FEC82000F0FFFD002311
:1000C00084F85F3084F8603084F8613084F86230FE
:1000D00084F8633084F8643084F8653084F804313F
:1000E00084F8053184F8063184F8073184F81C312E
:1000F00084F81D3184F81E3184F81F3184F8F33000
:1001000084F8F53084F8F73084F8F93084F8F43066
:1001100084F8F63084F8F83084F8FA3084F8FB304C
:1001200023716371A371E37184F86B3084F8CD306F
:1001300010BD00BFCF38002059310020F930002019
:10014000BA4B00203F350020783000202F3A0020A5
:100150009A4A00209F3500201A4C0020EF3B0020D7
:10016000FF35002082320020FA4A00209F34002010
:10017000B9310020EF49002059320020F74D00200E
:100180007B3400205B340020D93000202333002052
:100190009A4B0020BB4C00202DE9F04FC3F34719C8
:1001A00087B080460F46924603F01F05B9F1000F55
:1001B0002ED000264FF0010B344683B205934E45F6
:1001C0000FDB04F120091FFA89F935B100241D4E17
:1001D0004F441FFA88F8AC421DDB584607B0BDE813
:1001E000F08F4FF48063029320237401A4B2019333
:1001F0003A190AEB0403009392B2102305991148AF
:1002000001F032FF8346142000F058FD0136D6E796
:100210004FF0010BD9E74FF6FF73029301230193CF
:1002200009EB04033A195344009392B21023414658
:10023000304601F019FF8346142000F03FFD0134E1
:10024000C9E700BFE07B00202DE9F0438946002488
:100250000746DFF840800E4E85B04FF6FF730293DD
:10026000202309EB4412019392B210233946CDF8B2
:100270000080304601F0F8FE01340546142000F0FD
:100280001DFD802CE9D1284605B0BDE8F08300BFF4
:10029000E07B0020F02A00202DE9F04FB54887B020
:1002A00004F00EFBB44BB54C93F83720B44D84F8F2
:1002B000792093F83820AB4684F87A2093F83920D7
:1002C000B04E84F87B2093F83A2084F87C2093F891
:1002D0003B2084F87D2093F83C2084F87E20DA7A55
:1002E00084F876201A7B84F87720587B03F5003356
:1002F00084F8780093F8372084F8A22093F8382007
:1003000084F8A32093F8392084F8A42093F83A20A5
:1003100084F8A52093F83B2084F8A62093F83C208D
:1003200084F8A720DA7A84F89F201A7B84F8A0202A
:100330005B7B84F8A130944BD97A84F871101A7BD6
:1003400084F872205B7B98420CBF0120022084F865
:1003500074008E4884F8733004F02AFA8C4B8D4A6E
:100360008D491B78127809788C4804F021FA8C4B5F
:100370008C4A8D491B78127809788C4804F018FA59
:100380008B4804F015FA824B58785F1C2B44E054DC
:1003900004F026FAB7423B46F6D1864D8648A94678
:1003A00004F08EFA854804F003FADFF8CC827C4B27
:1003B00058785F1C2B44E05404F012FA47453B4642
:1003C000F6D17D4804F07CFA7D487E4B00787E4A69
:1003D0007E491B781278097802907D480078019058
:1003E0007C48007800907C4804F0E2F97B487C4B24
:1003F00000787C4A7C491B781278097802907B4807
:10040000007801907A48007800907A4804F0D0F99A
:1004100079487A4B00787A4A7A491B7812780978B9
:1004200002907948007801907848007800907848E8
:1004300004F0BEF994F87410764804F0B9F97648DF
:1004400004F03EFA754A764B15781B782D0445EA80
:100450000365744B1B781D43734B1B7845EA0325DA
:10046000724B93F801A01A784FEA0A4A4AEA026AE4
:10047000DA784AEA020A9A786D4B4AEA022A0AF1C5
:10048000FF329A4200F25E8151466A48FFF7A0F9B6
:10049000074629465246684804F08AF9AF4219BF18
:1004A0002A4639463A46394614BF6448644804F03F
:1004B0007FF9644804F004FA634804F001FA634ADF
:1004C000634B15781B782D0445EA0365614B043AAC
:1004D0001B7812781D43604B12041B7845EA0325F4
:1004E0005E4B1B7842EA03625D4B1B781A435D4BFF
:1004F0001B7842EA03224E4B511E994200F224819E
:10050000114659480592FFF763F98246059A294634
:10051000494804F04DF9AA4500F04881FF2384F8CA
:10052000763084F8773084F8783084F8793084F83D
:100530007A3084F87B3084F87C3084F87D3084F81D
:100540007E3094F87430012B00F001812A46514628
:100550003A4804F02DF93B4804F0B2F9434804F05E
:10056000AFF9434A434B15781B782D0445EA0365E0
:1005700084E000BFD75F010800800208CF38002068
:100580007280FDF72D800208807F0008E45F01087B
:100590000D8002080C8002080B800208056001082B
:1005A0000D8004080C8004080B8004082B600108EF
:1005B000516001089B80FBF79963010865600108A1
:1005C000BC7F0008B97F0008B87F0008B77F00082B
:1005D000BB7F0008BA7F0008796001083C800208F0
:1005E0003980020838800208378002083B80020800
:1005F0003A800208B46001083C800408398004088D
:1006000038800408378004083B8004083A800408D6
:10061000EB600108226101083A610108C27F00080D
:10062000C17F0008C47F0008C37F0008BD7F0008A9
:10063000FEFF010000800008646101088461010878
:10064000A6610108CB610108F5610108428002083A
:100650004180020844800208438002083D8002086D
:10066000408002083F800208808002081C62010866
:1006700042800408418004082D800408894B1B78BF
:100680001D43894B1B7845EA0325884B5E781A7811
:10069000360446EA0266DA7816439A78844B46EACC
:1006A0000226721E9A4204D831468248FFF790F81B
:1006B000824632462946804804F07AF8AA4500F07E
:1006C000B78094F87430022B40F0A9807B4B7C48B3
:1006D000DA7A84F89F201A7B84F8A0205A7B84F869
:1006E000A12093F8372084F8A22093F8382084F8CA
:1006F000A32093F8392084F8A42093F83A2084F8B2
:10070000A52093F83B2084F8A62093F83C3084F889
:10071000A7306C4B59781A1801334345A154F9D1CD
:100720002A465146684804F043F8684804F0C8F87F
:1007300094F8742094F87510654807B0BDE8F04F40
:1007400004F036B80027A4E64FF0000ADFE694F87C
:100750007130604E84F8763094F8723084F87730D7
:1007600094F8733084F87830544B93F8372084F839
:10077000792093F8382084F87A2093F8392084F887
:100780007B2093F83A2084F87C2093F83B2084F86F
:100790007D2093F83C30504A84F87E304F4B587897
:1007A0009919013393426054F9D1CFE6BA4506D185
:1007B00094F87530052B04BF012384F874302A4661
:1007C0005146474803F0F4FF464B93F8372084F82E
:1007D000792093F8382084F87A2093F8392084F827
:1007E0007B2093F83A2084F87C2093F83B2084F80F
:1007F0007D2093F83C2084F87E20DA7A84F87620F5
:100800001A7B84F877205B7B84F87830364B5978F4
:1008100003EB0B020133B342A154F8D19BE6002352
:10082000FF21E2180133292B82F89F10F9D177E7D5
:10083000BA4506D194F87530062B04BF022384F81C
:1008400074302A465146264803F0B2FF274B93F8EE
:10085000372084F8A22093F8382084F8A32093F856
:10086000392084F8A42093F83A2084F8A52093F83E
:100870003B2084F8A62093F83C2084F8A720DA7A5D
:1008800084F89F201A7B84F8A0205B7B84F8A13039
:100890000C4B597803EB090201334345A154F8D1BD
:1008A00043E700BF44800408438004083D800408F7
:1008B000FEFF01008080040864610108807F000859
:1008C0007280FBF70D80040884610108CB61010888
:1008D00043620108F280FFF7AD7F00088D7F0008BA
:1008E000A6610108008002080D800208008004084B
:1008F0003B4B2DE9F0411A7806469846394D002ABF
:100900005AD1394F4FF4B07239463848F8F74CFF96
:100910004FF4B073354A4FF42E61A020FFF73CFC32
:1009200000F034FF032E324C3BD197F87430012B8A
:1009300028D1304803F0C4FF0023402223602E4B0F
:100940002E48A360E2602B6003F0BAFF2C4803F04E
:10095000B7FFE1682B4803F02BFFA1682A4803F09A
:1009600027FF2A4803F0ACFF2949214800F0BEFFC9
:10097000D0B1284C204603F0A3FF4FF4FA6000F0FA
:100980009DF9F7E7244803F09BFF002340222360F2
:10099000224B2348A360E2602B6003F091FF2148C3
:1009A000D5E7022EF1D1C7E701231F4888F80030B0
:1009B00003F086FF00F0FCFE2B687BB90A4B93F82E
:1009C0007430012B0BBF0C4B144B2B602B600CBFF6
:1009D00008481148BDE8F04103F072BFBDE8F0815E
:1009E000F42E002000570020CF38002004570020AC
:1009F000F82E00202B630108008004083C630108E6
:100A00007D6301089B630108AB630108CF630108A4
:100A1000082F0020DC6301085463010800800208ED
:100A2000656301088C630108F16201082DE9F04754
:100A30000F461646804600F0A9FE214803F040FF0D
:100A4000204A214C136821683B442048136003F07E
:100A5000AFFE23681BB9012E13D11D4B2360454601
:100A6000DFF87890DFF878A0A5EB08039F420AD85A
:100A70002168184803F09CFE00F09AFE3046BDE85D
:100A8000F087154BEAE7AB7869782A781B0403EB0B
:100A900001231344EA78216803EB02620220002359
:100AA00000F0BAFE20B92368043323600435DBE785
:100AB000484603F005FF2168504603F079FEF5E74C
:100AC00063620108F02E0020005700207C620108BC
:100AD00000800208BD6201080080040891620108DC
:100AE000AA6201080023064A436003608360054947
:100AF000A2F800380448A2F80238012202F0CEBA67
:100B000078680020786000209881002038B5304D4A
:100B1000304C29684B1C2B602F4B5A6803F10C009A
:100B2000105C0132B2F5006FA8BF00225A609A68CB
:100B30006054013A9A60E2B92378BE2B1AD1A378A7
:100B4000E178264841EA03214B1CE25C8B1CE35C04
:100B500043EA0222FEF712FE012802D11D48FDF7EA
:100B6000EFFA4FF4006200211A4803F018FE002348
:100B70002B6038BD2378162BF3D16378162BF0D178
:100B8000A378162BEDD1E378162BEAD1627D1221E2
:100B90001048FEF7DAFDC0B1E37C217D104841EA40
:100BA000032101F11603E25C01F11703E35C43EA60
:100BB0000222FEF7E3FD012803D10648FDF788FF76
:100BC000CFE7084803F07CFECBE70748FAE700BF11
:100BD0000C2F00206C5800206C6000206D58002005
:100BE00082580020F563010801640108002310B554
:100BF0000D4A0E4C136022680132B2F5006FB8BF87
:100C000013462360A3680133B3F5006FA36001DBD3
:100C1000FFF77CFF236806490122BDE81040194414
:100C2000044802F0D9B900BF603000206C60002099
:100C3000786000209881002070B5074D074C084E61
:100C4000AB68002B02DD2368322B00D870BD304624
:100C5000FFF75CFFF4E700BF6C600020603000200D
:100C6000988100200A460146014802F0DDB900BF24
:100C700098810020074A08B51368032043F0100349
:100C8000136000F03FFB002003F04CFC03F08EFAF1
:100C9000002008BD00200240034A044B11681B7865
:100CA0000B441360704700BF88780020C4280020E0
:100CB000014B1868704700BF8878002038B504469B
:100CC000FFF7F6FF0546631C1EBF044B1B78E418B4
:100CD000FFF7EEFF401B8442FAD838BDC42800203D
:100CE000436A10B59A6A12F0500F1BD19A6A42F407
:100CF00000729A621A68926802F46022B2F5602F5C
:100D00000CD11A7B52B99A6A22F480729A629A6A5A
:100D1000D2045EBF9A6A42F001029A62184602F05B
:100D200073FB10BD1B6ABDE810401B6B1847704772
:100D300008B5406AFFF7FBFF08BD7047036810B5B0
:100D40005A680446900627D51A68910724D5A26AE6
:100D5000D2065EBFA26A42F40072A2629A6802F4EE
:100D60006022B2F5602F10D1227B72B95A6822F04E
:100D700020025A60A36A23F48073A362A36ADB048F
:100D80005EBFA36A43F00103A362204602F03CFB6E
:100D90006FF0120223681A6023685A68100630D573
:100DA0001A6851072DD5A26AD2065EBFA26A42F424
:100DB0000052A2629A6802F4E042B2F5E04F0AD013
:100DC0005A68500516D49A6802F46022B2F5602F72
:100DD00010D1227B72B95A6822F080025A60A36A4D
:100DE00023F48053A362A36AD9055EBFA36A43F0CC
:100DF0000103A362204600F083FA6FF00C0223681F
:100E00001A6023685A6852060DD51B68DB070AD59D
:100E1000A36A204643F48033A362FFF78EFF6FF08E
:100E2000010223681A6010BD7047406A08B5836AE2
:100E300043F040038362C36A43F00403C362FFF7D5
:100E4000F3FF08BD002373B5019390F82430012B04
:100E500074D001234D6880F82430062D02684FEAD3
:100E600085030C6825D82B441F25566B053B9D40F8
:100E700026EA050504FA03F32B435363092C4FEAD2
:100E800044038D682FD907262344D1681E3B9E401A
:100E900021EA060105FA03F30B43D360A4F1100322
:100EA000012B2BD90023002280F82420184602B001
:100EB00070BD0C2D0BD82B441F25166B233B9D407A
:100EC00026EA050504FA03F32B431363D6E72B4404
:100ED0001F25D66A413B9D4026EA050504FA03F327
:100EE0002B43D362CAE70726116923449E4021EAB7
:100EF000060105FA03F30B431361CFE7104B9A4247
:100F000016D193681B02CDD49368102C43F40003D0
:100F10009360C7D10B4B0C4A1B68B3FBF2F20A2358
:100F200053430193019B002BBCD0019B013BF8E78D
:100F3000836A43F0200383620123B4E70223B5E709
:100F400000240140CC28002040420F00002373B54C
:100F50000193036804469A68D20702D5002002B0C4
:100F600070BD9A6842F001029A60124B124A1B68E7
:100F7000B3FBF2F30193019BC3B9FFF799FE064659
:100F800023689D6815F00105E8D1FFF791FE801BED
:100F90000228F5D9A36A84F8245043F01003A36211
:100FA000E36A012043F00103E362D8E7019B013BC0
:100FB000E0E700BFCC28002040420F002DE9D841D7
:100FC0009046404B026804469A420F4602D03E4982
:100FD0008A4203D15B6813F4702F6ED194F82430E9
:100FE000012B6CD00123204684F82430FFF7AEFF9C
:100FF000064600285DD1A06A216820F47060324B5B
:1010000020F0010040F480709942A06204D12D4A82
:10101000536813F4702F3ED1A36A23F48013A362A4
:101020004B685A0505D5A36A23F4405343F4805313
:10103000A362A36A206A13F4805318BFE36A3A4696
:1010400018BF23F00603E362002384F824301F4B0B
:101050004C3183621E4BC3621E4B03636FF002036D
:1010600041F84C3C51F8443C43F4807341F8443C13
:10107000434600F0DBF923689A6802F46022B2F577
:10108000602F9A680CBF42F4A00242F480129A606A
:101090003046BDE8D881A36A43F48013A362536845
:1010A0005B0541BFA06A20F4405040F48050A0622C
:1010B000BFE7002384F82430EAE70126E8E70226A8
:1010C000E6E700BF0024014000280140E10C0108D0
:1010D000310D01082B0E010838B5036804469A68E3
:1010E000D20701D4002038BD9A6822F001029A602C
:1010F000FFF7DEFD054623689B68DB07F2D5FFF7A7
:10110000D7FD401B0228F6D9A36A012043F0100343
:10111000A362E36A43F00103E36238BDF8B5044615
:10112000002877D0836A23B9C36280F8243003F0A3
:101130005FF82046FFF7D0FFA36A13F010036BD1CE
:10114000002869D1A26A374922F4885222F00202AB
:1011500042F00202A26294E824008A42E16904D1CA
:10116000B1F5402F08BF4FF40021267B45EA460524
:101170002943A568B5F5807F35D0012D08BF4FF410
:101180008073277D012F06D17EBBA669013E43EA0D
:10119000463343F400635668B5F5807F26F469460C
:1011A00043EA0603536096681F4B03EA060343EACB
:1011B0000103936001D0012D20D12369013B1B0560
:1011C000D56A25F470052B43D3629268174B134000
:1011D000994215D10023E362A36A23F0030343F08D
:1011E0000103A362F8BD2B46CBE7A66A46F02006B2
:1011F000A662E66A46F00106E662CCE70023DFE776
:10120000A36A23F0120343F01003A362E36A43F0DE
:101210000103E3620120F8BDA36A43F01003A36257
:10122000F8E700BF003C0140FDF7E1FFFE0E1FFFA5
:10123000002373B5019390F824300446012B5AD053
:10124000012380F82430FFF747FF0546002832D1FC
:10125000A36A022023F4885323F0020343F002031D
:10126000A362264B1E6801F0FFFBB6FBF0F04000C6
:101270000190019B1BBB2046FFF768FE2268936824
:1012800043F008039360FFF713FD064623689A684E
:10129000120718D49A6842F004029A60FFF708FD1A
:1012A000064623689B685B071FD4A36A23F00303E9
:1012B00043F00103A362002384F8243012E0019B71
:1012C000013B0193D5E7FFF7F3FC801B0A28DDD92A
:1012D000A36A012523F0120343F01003A362002345
:1012E00084F82430284602B070BDFFF7E1FC801B73
:1012F0000A28D6D9ECE70225F4E700BFCC28002065
:1013000070470000074A0002D36800F4E06023F44D
:10131000E0631B041B0C43F0BF6343F4003303433F
:10132000D360704700ED00E0174B30B5DC68C4F3C4
:101330000224C4F10703251D042B28BF0423062D16
:101340004FF0010598BF002405FA03F303F1FF33C2
:1013500088BF033C1940A14005FA04F4013C224037
:10136000002842EA01024FEA0212A9BF00F16040E0
:10137000064BD2B200F56140BBBF00F00F00D2B205
:1013800080F800231A5430BD00ED00E014ED00E0B9
:10139000002808DB0123420900F01F0003FA00F0D7
:1013A000014B43F82200704700E100E010B500282F
:1013B00032D00168194B1424994225D8184AA3F257
:1013C00007430A44B2FBF4F2920002648468C363E8
:1013D00043680A682343C46822F47F5223430469A4
:1013E00022F0300223434469234384692343C469C0
:1013F000234313430B600122002380F821208363E1
:1014000080F82030184610BD064B0B44B3FBF4F3B4
:101410009B000364044BD9E7012010BD0704024080
:10142000F8FFFDBFF8FBFDBF00040240F0B590F8E7
:101430002040012C35D0012490F8215080F8204024
:10144000A5424FF000064FF0020428D180F8214059
:10145000046886632668076C26F001062660C66B62
:10146000BD407560636043680568102BC36A0BBF9D
:10147000A260A160E160E2604BB1236843F00E031B
:1014800023602B68002043F001032B60F0BD23682C
:1014900023F004032360236843F00A03F0E780F895
:1014A00020600220F0BD000090F8213010B5022B22
:1014B00003D004238363012010BD03681A6822F05F
:1014C0000E021A601A6822F001021A60294A934239
:1014D00024D902F56272934219D01432934218D083
:1014E0001432934217D0143293420CBF4FF48053FE
:1014F0004FF48033204A53600123002480F82130C8
:10150000436B80F820409BB39847204610BD0123D1
:10151000F0E71023EEE74FF48073EBE717498B42B7
:1015200016D014318B4215D014318B4214D01431A3
:101530008B4214D014318B4214D014318B4214D00E
:10154000934214BF4FF480334FF080730C4AD2E7BC
:101550000123FBE71023F9E74FF48073F6E74FF41C
:101560008053F3E74FF48033F0E74FF48013EDE757
:10157000184610BD800002400004024008000240EE
:101580000000024070B40425C66B026C3468036826
:1015900095402542196855D04D0753D51A689606CF
:1015A0005EBF1A6822F004021A60604A93421FD993
:1015B00002F56272934214D01432934213D0143263
:1015C000934212D0143293420CBF4FF480434FF435
:1015D0008023574A5360C36A002B00F0A58070BC7B
:1015E00018470423F5E74023F3E74FF48063F0E75F
:1015F00050498B4216D014318B4215D014318B4296
:1016000014D014318B4214D014318B4214D01431C5
:101610008B4214D0934214BF4FF480234FF0806369
:10162000454AD7E70423FBE74023F9E74FF48063FB
:10163000F6E74FF48043F3E74FF48023F0E74FF4ED
:101640008003EDE702259540254257D08D0755D5FB
:101650001A68940606D41A6822F00A021A60012257
:1016600080F82120314A93421ED902F562729342DA
:1016700013D01432934212D01432934211D0143248
:1016800093420CBF4FF400534FF40033284A536089
:10169000002380F82030836A9EE70223F6E72023A8
:1016A000F4E74FF40073F1E722498B4216D014316E
:1016B0008B4215D014318B4214D014318B4214D08C
:1016C00014318B4214D014318B4214D0934214BF86
:1016D0004FF400334FF00073174AD8E70223FBE7BB
:1016E0002023F9E74FF40073F6E74FF40053F3E7D4
:1016F0004FF40033F0E74FF40013EDE70825954071
:10170000254211D009070FD5196821F00E01196083
:10171000012303FA02F27260836380F82130002310
:1017200080F82030036B57E770BC704780000240A0
:10173000000402400800024000000240114AD36841
:1017400013F0100305D01049CB6943F00203CB61BD
:101750001023D268500706D50B4943F00403CA6929
:1017600042F00102CA61074AD169C90708D5064893
:10177000C16941F00401C161D16921F00101D16168
:10178000D36070470020024090780020064B186913
:1017900010F0800007D0054A5A6002F188325A6082
:1017A0001869C0F3C010704700200240230167454C
:1017B000034A0020136943F080031361704700BFA0
:1017C00000200240F8B50646FFF772FA114C0746B2
:1017D0002546E368D80712D4E368990644BF20235E
:1017E000E360EB68DA0606D4EB69DB0703D4E8684C
:1017F00010F0040002D0FFF7A1FF0120F8BD731C18
:10180000E7D00EB90320F8BDFFF752FAC01B86429D
:10181000DFD2F7E7002002402DE9F84F1F4C994630
:10182000237E0546012B0F46904633D001234CF210
:1018300050302376FFF7C6FF40BB012D03D0022DA9
:101840000CBF022504250026B246DFF854B0320151
:1018500040464946F6F7E8FCC4F81CA0DBF8103017
:1018600080B243F00103CBF8103027F816004CF299
:101870005030FFF7A7FFDBF8103023F00103CBF85F
:10188000103018B90136F3B29D42E0D80023237618
:10189000BDE8F88F0220BDE8F88F00BF90780020E7
:1018A000002002400022064BDA61064B1A6942F022
:1018B00004021A611A6942F040021A61704700BFBF
:1018C00090780020002002400022064BDA61064B8F
:1018D0001A6942F002021A6158611A6942F0400224
:1018E0001A61704790780020002002402DE9F041F5
:1018F000234D07462B7E8846012B3DD001240368EB
:101900002C76022B4CF2503013D1FFF75BFF20B145
:10191000012000232B76BDE8F081FFF7C3FF4CF2D6
:101920005030FFF74FFF174A136923F00403136188
:10193000EFE7FFF747FF0028EAD14FF0FF33C8F881
:1019400000302046BE680F4CFA68BB6803EBC22328
:101950009E42DED23046FFF7B7FF4CF25030FFF721
:1019600031FF236923F00203236110B1C8F800603E
:10197000CFE706F50066E7E70220BDE8F08100BF8B
:1019800090780020002002402DE9F74F00242646E1
:101990006C4F6D4BDFF8B8E1DFF8B8C10A6832FA76
:1019A00006F502D103B0BDE8F08F4FF0010808FA48
:1019B00006F802EA0802904540F084804D68122D36
:1019C00000F0B18000F28780022D00F0A9807BD862
:1019D000002D00F08C80012D00F0A0804FF00F0949
:1019E000FF2A93BF824606F18045083DD0F800B03B
:1019F00092BFB500D0F804B0AD0009FA05F82BEAA3
:101A0000080804FA05F588BF00F1040A48EA05054C
:101A1000CAF80050D1F804A01AF0805F52D0BD6916
:101A200026F0030845F00105BD61BD6908F1804855
:101A300005F00105019508F5803806F0030B019DBE
:101A40004FEA8B0BD8F8085009FA0BF925EA090977
:101A50003E4DA8426CD005F58065A8426AD005F5D8
:101A60008065A84268D005F58065A84266D005F576
:101A70008065A84264D070450CBF0525062505FA8F
:101A80000BF545EA0905C8F808501D681AF4803FAF
:101A900014BF154395431D605D681AF4003F14BFE1
:101AA000154395435D609D681AF4801F14BF15436C
:101AB00095439D60DD681AF4001F14BF2A4325EA90
:101AC0000202DA60013669E7032D25D0112D85D198
:101AD000CC68043482E7654509D012D8DFF87890E5
:101AE0004D4504D009F580394D457FF477AF8C68BA
:101AF000E4B1012C0CBFC0F81080C0F81480082499
:101B00006CE7DFF858904D45F1D009F580394D4527
:101B1000EDD0A9F58019E7E700245FE7CC685DE721
:101B2000CC6808345AE7CC680C3457E7042455E7EE
:101B30000025A4E70125A2E70225A0E703259EE7EB
:101B400004259CE700100240000401400008014009
:101B5000001C014000002110000011100000311095
:101B60008368194214BF0120002070470AB1016147
:101B700070470904FBE7C3680B4214BF4161016170
:101B80007047016800224B6913F4806310D06FF432
:101B900080634B612023026380F83D3080F83E2053
:101BA000036C80F83C2043F0040303640120704779
:101BB000184670472DE9F843044617469946C1F385
:101BC00007488EB22568B8F1010F0CBF6B69AB698D
:101BD00036EA030314BF0120002008B9BDE8F883EA
:101BE0006B695A0516D52B68202243F400732B60CD
:101BF0006FF480636B610023236384F83D2084F8D5
:101C00003E30226C42F00402226484F83C30012011
:101C1000BDE8F8837B1CD5D0FFF74AF8A0EB09009C
:101C2000874201D3002FCDD100232022236384F8E3
:101C30003D2084F83E30226C42F02002E4E770B58B
:101C400004460D46164623685B695B0701D50020F4
:101C500070BD2046FFF795FFA8B96A1CF3D0FFF7C7
:101C600027F8801B854201D3002DECD100232022D0
:101C7000236384F83D2084F83E30226C84F83C30A5
:101C800042F020022264012070BD70B504460D466A
:101C900016462068436913F0400301D0002070BD50
:101CA0004269D2060ED56FF01002426120222363F2
:101CB00084F83D2084F83E30226C226484F83C3065
:101CC000012070BDFEF7F4FF801BA84201D8002D53
:101CD000DFD100232022236384F83D2084F83E30A6
:101CE000226C42F02002E8E72DE9F84304469046D2
:101CF0001F46089EC1F307498DB22368B9F1010F51
:101D00000CBF5B699B6935EA03030CBF0123002309
:101D1000434502D00020BDE8F8837B1CEDD0FEF7E0
:101D2000C7FF801B874201D3002FE6D1002320226A
:101D3000236384F83D2084F83E30226C84F83C30E4
:101D400042F0200222640120BDE8F88370B5044609
:101D50000D46164623685B691B0601D5002070BD41
:101D60002046FFF70EFFA8B96A1CF3D0FEF7A0FFCC
:101D7000801B854201D3002DECD100232022236358
:101D800084F83D2084F83E30226C84F83C3042F0E8
:101D900020022264012070BD2DE9FF411546026832
:101DA000984613680B9E43F4807313600F460096A9
:101DB0000A9B00224FF001110446FFF795FF18B16E
:101DC000012004B0BDE8F081236807F0FE071F6121
:101DD0000A9A334616492046FFF7ECFE0028EFD159
:101DE000236803905A690A9903929B6932460393C8
:101DF0002046039BFFF7AAFF40B1236C042B01BFD1
:101E00002268136843F400731360D9E7B8F1010F37
:101E1000236802D1EDB21D61D3E72A0A1A610A993B
:101E200032462046FFF792FF0028E6D12368F1E70B
:101E3000020001002DE9FF419846036816461A6822
:101E40000B9D42F480621A601A680F4642F4807259
:101E50001A604FF0011100950A9B00220446FFF71B
:101E600043FF18B1012004B0BDE8F0812368FFB240
:101E700007F0FE021A6129492B460A9A2046FFF70D
:101E800099FE0028EED1236803905A690A990392BB
:101E90009B692A4603932046039BFFF757FF40B1F7
:101EA000236C042B01BF2268136843F40073136092
:101EB000D8E7B8F1010F236825D1F6B21E612A4692
:101EC0000A992046FFF742FF02460028E8D1216820
:101ED00020460B6843F480730B6000950A9B4FF01B
:101EE0000111FFF701FF0028BCD1236847F001076B
:101EF0001F610A9A2B4609492046FFF75BFE003016
:101F000018BF0120AFE7320A1A610A992A46204613
:101F1000FFF71CFF0028C3D12368CEE702000100B1
:101F200070B5044608B9012070BD90F83D3003F04B
:101F3000FF021BB980F83C2002F002FA2423226839
:101F400084F83D30136823F00103136000F0D6FCE1
:101F50006568414B9D424DD8404B9842E3D940497A
:101F60002268B0FBF1F1536823F03F030B43536049
:101F7000136A23F03F03013119431162D169364BD3
:101F800021F44F419D4221F0FF0100F1FF3048D87C
:101F90006D00B0FBF5F00130C0F30B03042B38BF2C
:101FA00004230B43D3611168206AE36921F0C00167
:101FB00003430B4313609168E068236921F40341F4
:101FC000034321F0FF010B439360D168A06963696B
:101FD00021F0FF0103430B43D3601368002043F05B
:101FE000010313602023206484F83D30206384F8CB
:101FF0003E0070BD1B4B984295D9194E4FF4967117
:10200000B0FBF6F622687143536823F03F03334375
:102010004FF47A765360136AB1FBF6F123F03F0375
:10202000A9E7A36853B905EB4503B0FBF3F0431CE4
:10203000C3F30B036BB143F40043B2E719236B43C3
:10204000B0FBF3F0431CC3F30B0313B143F4404361
:10205000A7E70123A5E700BFA08601007F841E003B
:1020600040420F00FF083D002DE9F7430446994622
:102070000F4690460C9EFEF71BFE94F83D30054639
:10208000202B03D0022003B0BDE8F0830090192379
:1020900001223B492046FFF727FE0028F2D194F8A1
:1020A0003C30012BEED0012384F83C3023682046DD
:1020B0001A68D10758BF1A6839465CBF42F001025E
:1020C0001A601A6822F400621A60212384F83D30F5
:1020D000402384F83E30002323640A9B0195636209
:1020E000BDF82C3000966385638D42462385254BD1
:1020F000E3624B46FFF750FE00282AD00120C2E7DA
:10210000FFF724FE40B1236C042B01BF2268136843
:1021100043F400731360F1E7636A27681A4612F804
:10212000011B39616262628D218D013A92B2628532
:102130007A69481E80B2520720850AD548B15A787C
:1021400002333A616362638D0239013B9BB22185A0
:102150006385238D2A4631462046002BD0D1FFF7D8
:102160006EFD0028CFD12268136843F4007313601A
:10217000202384F83C0084F83D3084F83E0082E758
:10218000020010000000FFFF2DE9F043044687B075
:1021900099460D469046109FFEF78AFD94F83D3013
:1021A0000646202B04D00225284607B0BDE8F08360
:1021B0000090192301227E492046FFF795FD002853
:1021C000F1D194F83C30012BEDD0012384F83C3060
:1021D000236829461A68D00758BF1A6820465CBF92
:1021E00042F001021A601A6822F400621A60222387
:1021F00084F83D30402384F83E30002323640E9B56
:1022000001966362BDF83C3000976385638D42465A
:102210002385684BE3624B46FFF70CFE054608B189
:102220000125C1E7228D236892B902905A69029272
:102230009A690292029A1A6842F400721A60202384
:1022400084F83D30002384F83E3084F83C30ABE71E
:10225000012A2FD11A6822F480621A6072B62368AC
:1022600003905A6903929A690392039A1A6842F496
:1022700000721A6062B6DFF84081238D002BDED039
:10228000032B77D8012B31D1324639462046FFF750
:10229000FCFC0028C4D12268636A12691A70636A60
:1022A00001336362238D013B2385638D013B9BB228
:1022B0006385E2E7022A1A680ED142F400621A60CE
:1022C00072B6236804905A6904929A690492049A37
:1022D0001A6822F48062CCE742F480621A600590AA
:1022E0005A6905929B690593059BC4E7022B0096EA
:1022F0003B464FF000024146204618D1FFF7F4FC60
:1023000000288DD172B623681A6842F400721A60F0
:102310001B69626A1370636A01336362238D013B38
:102320002385638D013B9BB2638562B6B3E7FFF7FC
:10233000DBFC024600287FF473AF21680B6823F4AE
:1023400080630B6072B62168636A09692046197060
:10235000636A009601336362238D4146013B238506
:10236000638D013B9BB263853B46FFF7BDFC0028B4
:10237000C9D055E7324639462046FFF786FC00288B
:102380007FF44EAF2268636A12691A70626A531C46
:102390006362238D013B2385638D013B9BB2638583
:1023A0002368596949077FF568AF1B69537076E761
:1023B000020010000000FFFF0400010038B50446D1
:1023C000D8B14CF6CC4203681A6045F255521A60F7
:1023D00042685A6082689A60FEF76AFC0546236884
:1023E000D86818B94AF6AA221A6038BDFEF760FC10
:1023F000401B3028F3D9032038BD012038BD4AF6F0
:10240000AA22036800201A60704700002DE9F341FA
:10241000054608B901203CE00368DB0710D42B68AF
:102420009F075DD42B68190700F194802B685A0729
:1024300000F1BE80E869002840F02C81002028E0EF
:102440008F4C636803F00C03042B07D0636803F020
:102450000C03082B09D16368DE0306D523689C03AF
:10246000DDD56B68002BDAD1D4E76B68B3F5803F1C
:1024700012D1236843F480332360FEF719FC06462B
:1024800023689803CBD4FEF713FC801B6428F7D98C
:10249000032002B0BDE8F0819BB9236823F48033A8
:1024A0002360236823F480232360FEF701FC0646A3
:1024B00023689903B3D5FEF7FBFB801B6428F7D98B
:1024C000E6E7B3F5A02F236803D143F4802323600C
:1024D000CFE723F480332360236823F48023CBE702
:1024E000674C636813F00C0F07D0636803F00C03AC
:1024F000082B10D16368DA030DD423689B0702D53B
:102500002B69012B86D123686A6923F0F80343EA1B
:10251000C203236086E72A695A4B6AB101221A6016
:10252000FEF7C6FB064623689F07ECD4FEF7C0FB08
:10253000801B0228F7D9ABE71A60FEF7B9FB064605
:10254000236898077FF56EAFFEF7B2FB801B022869
:10255000F6D99DE7AA694A4C4B4BDAB101221A60C1
:10256000FEF7A6FB0646636A9B070DD54FF4FA52A9
:10257000464B1B68B3FBF2F3019300BF019B5A1E4D
:102580000192002BF9D151E7FEF792FB801B022844
:10259000E9D97DE71A60FEF78BFB0646636A9F0761
:1025A0007FF544AFFEF784FB801B0228F6D96FE766
:1025B000334CE369D80024D40127E36943F0805306
:1025C000E361E36903F080530093009B304E33686E
:1025D000D90518D5EB68012B26D1236A43F00103F6
:1025E0002362FEF765FB41F288368046236A9B072B
:1025F0003FD5002F3FF41EAFE36923F08053E36122
:1026000018E70027E2E7336843F480733360FEF78E
:102610004FFB80463368DA05DCD4FEF749FBA0EBBC
:1026200008006428F6D933E7ABB9236A41F2883849
:1026300023F001032362236A23F004032362FEF7DD
:1026400037FB0646236A9807D3D5FEF731FB801B7C
:102650004045F7D91CE7052B236A03D143F0040357
:102660002362BAE723F001032362236A23F0040301
:10267000B6E7FEF71DFBA0EB0800B042B6D907E7AE
:10268000001002400000424280044242CC28002058
:10269000007000402A4B5A681C4602F00C02082ABF
:1026A0003DD00023274E022833602BD1FEF700FBDC
:1026B0000746236899011FD42B6AB3F5803F05D1E3
:1026C0006268A96822F400320A436260696A62683B
:1026D0000B4322F474121343636001233360FEF74B
:1026E000E7FA054623689A013FF5A8AEFEF7E0FA3F
:1026F000401B0228F6D9CBE6FEF7DAFAC01B022807
:10270000D7D9C5E6FEF7D4FA054623689B017FF5C5
:1027100095AEFEF7CDFA401B0228F6D9B8E601289F
:102720003FF4B7AE58682B6A00F480329A427FF4C7
:1027300071AE6B6A00F47010C01A18BF0120A8E6D1
:10274000001002406000424230B5194B87B002AC25
:1027500003F11005224618685968083303C2AB42DA
:102760001446F7D101238DF80430022311498DF866
:1027700005304B6803F00C02082A17D1C3F38342DB
:1027800006A80244DB0312F8102C0CD54B680A484B
:10279000C3F34043504306AA134413F8143CB0FB60
:1027A000F3F007B030BD05485043FAE70248F8E7B8
:1027B000A85801080010024000127A0000093D00EC
:1027C0002DE9F0410D46044610B90120BDE8F08125
:1027D000454A136803F007038B4229D321688E070B
:1027E00031D4CA0744D4404A136803F007039D421A
:1027F00067D322683D4D12F0040F6ED1130706D542
:102800006B68226923F4605343EAC2036B60FFF7ED
:102810009BFF6B68364AC3F30313D35CD840354B38
:102820001860354B186801F07DFE0020BDE8F0818E
:10283000136823F007030B431360136803F00703C7
:102840009942C2D1CAE7294B11F0040F1EBF5A6842
:1028500042F4E0625A60080742BF5A6842F460528C
:102860005A605A68A06822F0F00202435A60B8E742
:1028700062681E4E012A33681BD113F4003FA4D0B6
:10288000736841F2883823F0030313437360FEF743
:102890000FFA07467368626803F00C03B3EB820F0C
:1028A000A1D0FEF705FAC01B4045F3D90320BDE8CF
:1028B000F081022A02D113F0007FE0E713F0020F4B
:1028C000DDE7136823F007032B431360136803F05D
:1028D00007039D427FF479AF8BE76B68E16823F4CF
:1028E000E0630B436B6089E7002002400010024068
:1028F0008D640108CC280020C8280020044B054A1C
:102900005B68C3F30223D35C034A1068D840704766
:10291000001002409D640108CC280020044B054AA9
:102920005B68C3F3C223D35C034A1068D840704786
:10293000001002409D640108CC2800200F23036092
:102940000B4B5A6802F0030242605A6802F0F00230
:1029500082605A6802F4E062C2605B68DB0803F4DC
:10296000E0630361034B1B6803F007030B607047D0
:10297000001002400020024003682DE9F341D9070E
:10298000054620D5354CE369DA0032D40127E369E6
:1029900043F08053E361E36903F080530193019BAB
:1029A0002F4E3368DB0526D5236A13F4407336D1E6
:1029B000236A6A6823F44073134323621FB1E369F7
:1029C00023F08053E3612868830706D5234AA9686A
:1029D000536823F440430B43536010F010001BD0A6
:1029E0001E4A69695368002023F480030B43536037
:1029F00012E00027D4E7336843F480733360FEF7B6
:102A000057F980463368D805CED4FEF751F9A0EBCC
:102A100008006428F6D9032002B0BDE8F0816A6896
:102A200002F440729342C3D001200E4A236A106020
:102A3000002023F4407110602162D907B8D5FEF759
:102A400037F941F288380646236A9A07B0D4FEF770
:102A50002FF9801B4045F7D9DDE700BF0010024089
:102A60000070004040044242024670B53B4B86B0C5
:102A700002AD03F110062C4618685968083303C4E8
:102A8000B3422546F7D101238DF804300223501EAE
:102A90008DF805300F285ED8DFE800F032515D2D4B
:102AA0005D5D5D2D5D5D5D5D5D5D5D082C4B596817
:102AB000186810F0807037D0C1F3834206A8024432
:102AC00012F8100CCA0341BF5A6806A9C2F340426B
:102AD000521844BF12F8141C224A5B684CBFB2FB68
:102AE000F1F2214A5B0202FB00F01DD403234000F7
:102AF000B0FBF3F018E006B0BDE87040FFF724BE6D
:102B000040F20231164A136A1940B1F5817F1FD095
:102B100003F44073B3F5007F08D149F64040536A8F
:102B200013F0020F08BF002006B070BDB3F5407F60
:102B300011D113684FF2244013F4003FF2E7FFF77E
:102B4000EDFE074B5B68C3F3813301335B00CFE7D6
:102B50004FF40040E8E70020E6E700BFB85801085E
:102B60000010024000127A0000093D0003680020B6
:102B7000DA6842F00102DA609A6802F00702062A77
:102B80001EBF1A6842F001021A6070477047704712
:102B900070477047036810B51A69044691070ED54F
:102BA000DA6892070BD56FF002021A6101229B6965
:102BB00002779B0777D0FFF7EAFF0023237723688C
:102BC0001A69500710D5DA6851070DD56FF0040265
:102BD0001A6102229B69227713F4407F204668D055
:102BE000FFF7D5FF0023237723681A6912070FD553
:102BF000DA6810070CD56FF008021A610422DB694D
:102C00002277990720465AD0FFF7C1FF0023237788
:102C100023681A69D20610D5DA68D0060DD56FF090
:102C200010021A610822DB69227713F4407F2046E4
:102C30004BD0FFF7ACFF0023237723681A69D10735
:102C400008D5DA68D20705D56FF0010220461A616F
:102C500000F062FF23681A69100608D5DA681106C9
:102C600005D56FF0800220461A6100F0BAF823689B
:102C70001A69520608D5DA68500605D56FF0400289
:102C800020461A61FFF785FF23681A69910622D54D
:102C9000DA6892061FD56FF020022046BDE810408A
:102CA0001A6100F09DB8FFF771FF2046FFF770FF33
:102CB00083E7FFF76BFF2046FFF76AFF92E7FFF716
:102CC00065FF2046FFF764FFA0E7FFF75FFF2046A0
:102CD000FFF75EFFAFE710BD244A0368904212D0B1
:102CE00002F5006290420ED0B0F1804F0BD0A2F5F9
:102CF0009832904207D002F58062904203D002F5EC
:102D0000806290421DD14A6823F070031343174A32
:102D1000904212D002F5006290420ED0B0F1804F86
:102D20000BD0A2F59832904207D002F58062904213
:102D300003D002F58062904203D1CA6823F4407345
:102D400013434A6923F08003134303608B68C36213
:102D50000B688362054B984203D003F500639842E9
:102D600001D10B690363012343617047002C0140CB
:102D700010B50446A0B190F83D3003F0FF021BB936
:102D800080F83C2001F00EFB0223206884F83D30DF
:102D9000211DFFF7A1FF0123002084F83D3010BD65
:102DA000012010BD90F83C3030B5012B4FF00203EC
:102DB00014D0046880F83D306268A3680D684968E3
:102DC00022F0700223F080030B432A436260A36069
:102DD000012380F83D30002380F83C30184630BD98
:102DE000704770470368DA6822F49072DA605A69B3
:102DF00022F001025A61202380F83A307047000027
:102E000038B505460368C1681A69192422F440528E
:102E10000A431A6182680069D9680243686921F42B
:102E2000B05121F00C0102430A43DA605A69A969E2
:102E300022F440720A435A610D4A934214D1FFF7BB
:102E40006DFD60436C686422A400B0FBF4F0B0FB3D
:102E5000F2F402FB14031B013233B3FBF2F32968D3
:102E600003EB04138B6038BDFFF748FDE9E700BFB3
:102E700000380140F8B504460E4617461D46216845
:102E80000B6836EA030301D10020F8BD6B1CF7D0B4
:102E900095B923680320DA6822F4D072DA605A699F
:102EA00022F001025A61202384F8393084F83A3044
:102EB000002384F83830F8BDFDF7FAFEC01B8542C8
:102EC000DDD2E6E710B5044640B390F8393003F0A0
:102ED000FF021BB980F8382001F078FA2423226819
:102EE00084F83930D368204623F40053D360FFF7C9
:102EF00087FF236800201A6922F490421A615A69F8
:102F000022F02A025A61DA6842F40052DA60202381
:102F1000E06384F8393084F83A3010BD012010BDE8
:102F20002DE9F0411F4690F839300446202B0D461C
:102F300090464ED1002949D0002A47D090F8383029
:102F4000012B46D0012380F838300023C3632123AE
:102F500080F83930FDF7ACFE0646A4F82480A4F8CA
:102F60002680E38C9BB26BB93B463246402120461B
:102F7000FFF780FFA8B9202384F8380084F839309F
:102F8000BDE8F081E38C3246013B9BB2E384A36849
:102F90008021B3F5805F20463B460ED1FFF76AFFE4
:102FA00010B10320BDE8F0812B882268C3F3080329
:102FB0005360236943B90235D3E7FFF75BFF00286D
:102FC000EFD123682A785A600135CAE70120BDE8AD
:102FD000F0810220BDE8F08190F83A30202B20D11A
:102FE000E9B1E2B190F83830012B1AD0C285828560
:102FF00000232222C36380F83A2002688162D168EC
:1030000080F8383041F48071D1605169184641F040
:1030100001015161D16841F02001D1607047012068
:10302000704702207047000038B50446134694F8F4
:103030003920202A2AD139B333B394F83820012A11
:1030400024D00122002584F838202122E384206B3B
:10305000E56384F839200E4AA384216282620D4A16
:103060004563C2620C4A026322680432FEF7DEF94D
:103070006FF04002236828461A605A6984F8385075
:1030800042F080025A6138BD012038BD022038BDAF
:103090002F3101085D31010829320108134690F8EB
:1030A0003A2073B5202A054638D1002934D0002BA8
:1030B00032D090F83820012A30D00122002480F844
:1030C0003820222281628385C46380F83A20406BD5
:1030D000134A2E688262134A4463C262124A026330
:1030E0000A46311DFEF7A2F920462B6801941A68A2
:1030F00001925A6885F838400192019ADA6842F4E0
:103100008072DA605A6942F001025A615A6942F0EB
:1031100040025A6102B070BD0120FBE70220F9E7CE
:10312000673101081D32010829320108704708B5CE
:103130000368426A1B6813F020030AD1D384136822
:103140005A6922F080025A61DA6842F04002DA607D
:1031500008BD1046FFF7EAFF08BD704708B5406A92
:10316000FFF7FBFF08BD08B50368426A1B6813F050
:10317000200310D1D3851368D96821F48071D960F8
:10318000596921F001015961596921F040015961E2
:10319000202382F83A301046FDF728FD08BD90F84C
:1031A0003A3010B5222B36D183680169B3F5805FC0
:1031B0000268836A23D15268E9B9C2F3080223F88E
:1031C000022B8362C48D013CA4B2C4858CB9036810
:1031D000DA6822F02002DA60DA6822F48072DA60BB
:1031E0005A6922F001025A61202380F83A30FDF733
:1031F000FDFC002010BDD2B223F8012BE1E721B97C
:10320000591C526881621A70DCE75268591C81624D
:1032100002F07F02F7E7022010BD704708B5406A50
:10322000FFF7FBFF08BD7047416A08B50B685A6994
:1032300091F8390021280AD1120608D50022CA8443
:10324000DA6822F0C002DA60202281F839205B6956
:1032500091F83A20222A06D15B0604D500230846BD
:10326000CB85FFF7BFFDCB6B084643F01003CB6364
:10327000FFF7D9FF08BD0000036870B51A6804465F
:103280001607D9685D6907D196065AD58D0658D5B7
:10329000BDE87040FFF783BF15F0010502D111F4BE
:1032A000907F4ED0D30705D5CE0542BFE36B43F0E8
:1032B0000103E363500704D51DB1E36B43F0020340
:1032C000E363930704D51DB1E36B43F00403E363A9
:1032D000160704D51DB1E36B43F00803E363E36B0A
:1032E000002B66D0950604D5880602D52046FFF748
:1032F00056FF236820465D69E26B110702D415F082
:1033000040051AD0FFF76EFD23685A69520610D5A2
:103310005A69606B22F040025A6150B1254B4363F9
:10332000FEF7C2F8002844D0606BBDE87040436BE4
:1033300018472046FFF777FF70BDFFF774FFE5637E
:1033400070BD160627D50D0625D594F83920212AFB
:103350002FD1A268B2F5805F226A17D11188C1F31C
:1033600008015960216979B902322262E28C013A7E
:1033700092B2E284EAB9DA6822F08002DA60DA68AE
:1033800042F04002DA6070BD0132EEE7511C21626A
:1033900012785A60EAE750060BD54A0609D5DA6872
:1033A000204622F04002DA60202384F83930FFF70B
:1033B000BDFE70BDB933010808B50023406AC3855E
:1033C000C384FFF730FF08BD084A0949126882B07C
:1033D000B2FBF1F20190019B53430193019B5A1EF2
:1033E0000192002BFAD102B0704700BFCC28002018
:1033F00040420F0010B514460A230248FFF790FD23
:10340000204610BD6C8200201C4BF0B51B68046880
:103410009C421BD11A491B4D08882B681A4A80B25E
:1034200022F81300488803F1640680B222F81600DF
:10343000888803F1C80680B222F81600C98803F50F
:10344000967089B2013322F810102B600F4B1B6865
:103450009C4211D1002364260D4A0E4F11680E4C78
:1034600006FB031537F81300013380B2052B24F84F
:103470001500F5D101311160F0BD00BFB080002012
:103480006482002064300020B0780020E0800020BA
:1034900068300020347C00203E7C002010B596B0BF
:1034A000282200210CA801F07AF91422002101A899
:1034B00001F075F9182200210DEB020001F06FF9FF
:1034C0000A230C93012302241093102212934FF429
:1034D00040130CA8119215931394FEF797FF0F2336
:1034E0004FF4806201930023214601A803930492C4
:1034F00005930294FFF764F94FF4804306A80694FD
:103500000893FFF739FA16B010BD00002DE9F04F0F
:10351000B14D91B0FDF7AEFBFFF7C0FF10220021C7
:103520000CA801F03CF9AB69002243F04003AB6109
:10353000AB694FF6184103F040030593059BAB6957
:10354000A64843F01003AB61AB69002403F01003FD
:103550000693069BAB69012643F08003AB61AB6920
:10356000022703F080030793079BAB694FF00C0A17
:1035700043F00403AB61AB694FF0040903F00403AB
:103580000893089BAB694FF0070B43F48073AB6162
:10359000AB694FF0050803F480730993099BAB698D
:1035A00043F00803AB61AB6903F008030A930A9B7D
:1035B000AB6943F02003AB61AB6903F020030B93CD
:1035C0000B9BFEF7D3FA002248F240018448FEF735
:1035D000CDFA00224FF63F718248FEF7C7FA00226B
:1035E0004CF2C0218048FEF7C1FA00224CF69C4103
:1035F0007E48FEF7BBFA4FF618430CA977480C93A8
:103600000D960E940F97FEF7BFF948F240030CA9F0
:1036100073480C930D960E940F97FEF7B5F94FF67D
:103620003F730CA96F480C930D960E940F97FEF7FD
:10363000ABF94CF2C0230CA96B480C930D960E9479
:103640000F97FEF7A1F94CF69C430CA967480C9321
:103650000D960E940F97FEF797F94FF4E0530CA9CF
:103660005F480C930D940E94FEF78EF90CA95F48F9
:103670000C960D940E94FEF787F96B695C48334302
:103680006B616B695B4A33400393039B6B693B43FC
:103690006B616B69584D3B400493049B4FF4E133DD
:1036A000846080E80C00C4600461C0F814A08461E8
:1036B000C461FFF707FC514B28462B604FF4807321
:1036C000AB604FF460232E73EB612C756C60C5F812
:1036D00010900C940D940E94FDF720FD0CA9284633
:1036E0000D96CDF83090CDF838B0FDF7ABFB0CA9B6
:1036F0002846CDF830800D97FDF7A4FB0622032362
:103700000CA928460C9201920D930093FDF79AFBA9
:103710000CA92846CDF830A0CDF83490FDF792FBE7
:103720004FF48073364D3749AB604FF46023284621
:10373000EB6129602E730C940D940E942C756C60C3
:10374000C5F81080FDF7EAFC0CA928460D96CDF8C7
:103750003090CDF838B0FDF775FB0CA92846CDF8B0
:1037600030800D97FDF76EFB019A009B0CA928464F
:103770000C920D93FDF766FB0CA92846CDF830B0EE
:10378000CDF83490FDF75EFB08230CA928460C9376
:10379000CDF83480FDF756FB4FF4E1331A481B494E
:1037A000846080E80A00C4600461C0F814A08461E9
:1037B000C461FFF787FB41F2DF53154E1548B46033
:1037C00086E809000A233046F360B4610C940D9436
:1037D000FFF7CEFA20E000BF0010024000180140C1
:1037E0000010014000200140000C01400014014085
:1037F0009881002000380140B08000200024014062
:10380000E0800020003C01406C8200200044004029
:1038100024820020001000400CA930460C940D9426
:103820005B4EFFF7BFFA5B485B4B846080E8480063
:103830004FF48043C460036144618461C4610462E5
:10384000FEF76EFB5548564B80E8080140F6FF73C3
:103850008360FEF7B3FD224621460B20FDF764FD91
:103860000B20FDF795FD224621462520FDF75CFD46
:103870002520FDF78DFD224621462620FDF754FD2B
:103880002620FDF785FD224621463B20FDF74CFD15
:103890003B20FDF77DFD224621463620FDF744FD05
:1038A0003620FDF775FD224621462F20FDF73CFD11
:1038B0002F20FDF76DFD224621461120FDF734FD36
:1038C0001120FDF765FD224621460E20FDF72CFD57
:1038D0000E20FDF75DFD0F2022462146FDF724FD59
:1038E0000F20FDF755FD2846FDF7A2FC0028FAD170
:1038F0002C4D2846FDF79CFC04460028F9D10522F2
:1039000029492A48FDF75AFB042229492548FDF791
:1039100055FB2848FFF72AF9274B21461B681F4C07
:10392000986800F0D5FFFCF7B1F9FCF713FBFCF742
:10393000B3FCF5F741F92148FDF7D4F80122204BFB
:10394000204883F8CB2000F0BBFF1F4800F0B8FFF1
:103950001E4A1F491F4800F02BFF1F4800F0B0FF10
:10396000184800F0ADFFF5F741F9FDF765F9F9F7F3
:1039700069FBF9F725FDF8F747FFFBF7D3FEFBF7E7
:103980002DFEFBF715FE2046FEF739FDEBE700BFE5
:10399000A0860100E07B002000580040D47B00207E
:1039A00000300040B0800020347C0020E080002007
:1039B0006482002024820020D02800206C60002037
:1039C000CF380020116401083B64010849640108F4
:1039D000526401085E6401086F6401081D4B93F88E
:1039E0000031012B25D11C4B1C4A195C1C4B09B31F
:1039F000002143F8201052F82030013342F82030E3
:103A000052F82030013303D141F2883342F820309C
:103A1000144B1A5C144B52B153F82020013243F876
:103A2000202053F82020013203D142F2107243F8D3
:103A30002020704742F8201053F82020013243F82C
:103A4000202053F82020013204BF47F2305243F8BF
:103A50002020DDE7CF38002060290020E82F00205B
:103A6000D82F00205C290020C82F00201D4B93F880
:103A70001831012B25D11C4B1C4A195C1C4B09B376
:103A8000002143F8201052F82030013342F8203052
:103A900052F82030013303D141F2883342F820300C
:103AA000144B1A5C144B52B153F82020013243F8E6
:103AB000202053F82020013203D142F2107243F843
:103AC0002020704742F8201053F82020013243F89C
:103AD000202053F82020013204BF47F2305243F82F
:103AE0002020DDE7CF3800206C290020383000206E
:103AF0002830002064290020F82F00200B78012BAB
:103B000018BF0022034B04BF53F82020013243F8B2
:103B10002020704750300020036810B5B3F1804F6B
:103B2000044601D1FDF7B8F82268A44B9A4240F050
:103B30002983A34A136801331360A24A136801332F
:103B40001360A14A136801331360A04A136801335C
:103B500013609F4A1368013313609E4A1368013350
:103B60001360F8F7A5FC9C4A00201368013313602A
:103B7000FFF77CFF0120FFF779FF0220FFF776FFB8
:103B80000320FFF773FF0020FFF728FF0120FFF756
:103B900025FF0220FFF722FF0320FFF71FFF8F49B9
:103BA0000020FFF7ABFF8E490120FFF7A7FF8D49EB
:103BB0000220FFF7A3FF8C490320FFF79FFF8B49EB
:103BC00000200B788A4A012B8A4B40F0A7811860AD
:103BD0001068013010601068013002D140F6B83032
:103BE00010604878012840F0A4815068013050608E
:103BF000002058605068013002D140F6B830506063
:103C00008878012840F0A181906801309060002000
:103C100098609068013002D140F6B8309060C97861
:103C2000012940F09E81D1680131D1600021D96025
:103C3000D368013302D140F6B833D3606E496F4A7E
:103C400008786F4B002800F09881106801301060F0
:103C5000002018601068013002D140F6B8301060C2
:103C60004878002800F094815068013050600020AE
:103C700058605068013002D140F6B8305060887802
:103C8000002800F0908190680130906000209860DA
:103C90009068013002D140F6B8309060C9780029B0
:103CA00000F08C81D1680131D1600021D960D368E6
:103CB000013302D140F6B833D3605249524A0878F2
:103CC000524B002800F08581106801301060002000
:103CD00018601068013002D140F6B83010604878A2
:103CE000002800F081815068013050600020586049
:103CF0005068013002D140F6B83050608878002812
:103D000000F07D819068013090600020986090689C
:103D1000013002D140F6B8309060C978002900F037
:103D20007981D1680131D1600021D960D368013334
:103D300002D140F6B833D3603549364A0878364B5D
:103D4000002800F0728110680130106000201860B7
:103D50001068013002D140F6B83010604878002871
:103D600000F06E815068013050600020586050684B
:103D7000013002D140F6B83050608878002800F059
:103D80006A819068013090600020986090680130EE
:103D900002D140F6B8309060C978002900F07881EF
:103DA000D1680131D1600021D960D368013302D1DB
:103DB00040F6B833D360194932E000BF001000402C
:103DC000603000204C3000205C2F00204830002064
:103DD000382F0020142F0020102F0020D33800206F
:103DE000D4380020D5380020D63800207029002093
:103DF0004C2F00203C2F0020DB4C0020282F0020DF
:103E0000182F0020682900201830002008300020DA
:103E100058290020B82F0020A82F00205429002066
:103E2000924A0878924B002800F03D8110680130DA
:103E30001060002018601068013002D140F6B830E0
:103E400010604878002800F03981506801305060D7
:103E5000002058605068013002D140F6B830506000
:103E60008878002800F0358190680130906000204B
:103E700098609068013002D140F6B8309060C978FF
:103E8000002900F03181D1680131D1600021D96071
:103E9000D368013302D140F6B833D3607548764B0E
:103EA000027802F0FF01002A00F029811A6801322D
:103EB0000EBF40F6B8321A6801321A606F4A1178A4
:103EC0006F4A01F0FF04002900F01B8111680131E5
:103ED0000EBF42F21071116801311160027802F0D8
:103EE000FF01002A00F00F811A6801320EBF40F670
:103EF000B8321A6801321A60624B634A93F8CA10EA
:103F0000624B002940F00181116801310EBF42F27D
:103F10001071116801311160002202E1106018680F
:103F2000013018601868013004BF42F21070186048
:103F300057E60020506058680130586058680130DA
:103F400004BF42F2107058605AE6002090609868F2
:103F5000013098609868013004BF42F21070986098
:103F60005DE60021D160DA680132DA60DA68013298
:103F700004BF42F21072DA6060E610601868013027
:103F800018601868013004BF42F21070186067E6CC
:103F900050605868013058605868013004BF42F2E0
:103FA000107058606BE6906098680130986098686F
:103FB000013004BF42F2107098606FE6D160DA6899
:103FC0000132DA60DA68013204BF42F21072DA605C
:103FD00073E610601868013018601868013004BF7B
:103FE00042F2107018607AE65060586801305860EC
:103FF0005868013004BF42F2107058607EE690604D
:104000009868013098609868013004BF42F21070DF
:10401000986082E6D160DA680132DA60DA680132EB
:1040200004BF42F21072DA6086E610601868013050
:1040300018601868013004BF42F2107018608DE6F5
:1040400050605868013058605868013004BF42F22F
:104050001070586091E69060986801309860986898
:10406000013004BF42F21070986095E6982F00204E
:10407000882F00206C2F0020682F0020642F002044
:10408000602F0020CF380020782F00207C2F0020C8
:10409000D160DA680132DA60DA68013204BF42F2D4
:1040A0001072DA6087E610601868013018601868CE
:1040B000013004BF42F210701860C2E650605868C8
:1040C000013058605868013004BF42F210705860E7
:1040D000C6E690609868013098609868013004BF27
:1040E00042F210709860CAE6D160DA680132DA6094
:1040F000DA68013204BF42F21072DA60CEE619606B
:10410000DCE61460EAE61960F6E60020012910609A
:104110007FF402AF1A6801320EBF40F6B8321A6857
:1041200001321A601C4B1A68012A2CD11A6801321C
:104130000EBF42F210721A6801321A60174B1A68E9
:10414000012A22D11A6801320EBF40F6B8321A682D
:1041500001321A60124A1168012918D1116801311F
:104160000EBF42F210711168013111601B68012B02
:104170000C4B0ED11A6801320EBF40F6B8321A68E5
:1041800001321A6010BD0022D7E70022E1E70021CA
:10419000EBE70022F5E700BF702F0020742F00200E
:1041A000802F0020842F0020704700000E4B82B02B
:1041B0009A6942F001029A619A6902F00102009242
:1041C000009ADA6942F08052DA61DB69074A03F04B
:1041D00080530193019B536823F0E06343F0007325
:1041E000536002B0704700BF001002400000014061
:1041F00030B505468BB01022002106A800F0CFFA9A
:104200002B68454A93424DD1444B03249A6906A931
:1042100042F400729A619A69414802F40072019274
:10422000019A9A6942F010029A619A6902F01002AA
:104230000292029A9A6942F004029A619B69079479
:1042400003F004030393039B04230693FDF79CFBF5
:104250007023344806A906930794FDF795FB802246
:10426000314C324BE2604FF4807222614FF4806235
:10427000236062610023202220466360A360A26164
:10428000E361FDF793F808B1FFF78EFF00222C627F
:10429000122011466562FDF747F81220FDF778F805
:1042A0000BB030BD224A9342FAD11C4B21489A6987
:1042B00006A942F400429A619A691F4C02F4004236
:1042C0000492049A9A6942F080029A619B6903F011
:1042D00080030593059B4FF4F8630693032307932C
:1042E000FDF752FB8022E2604FF4807222614FF4AE
:1042F0008062124B626123602022002320466360AB
:10430000A360A261E361FDF751F808B1FFF74CFF2C
:104310002C626562C4E700BF002401400010024027
:104320000010014000080140DC810020080002402C
:10433000003C0140001C014028800020580402403D
:1043400010B5044686B01022002102A800F027FA1A
:104350002268114B9A421DD1104C02A9A369104842
:1043600043F00803A361A36903F008030093009BD3
:104370004FF4406302931223039303230593FDF745
:1043800003FBE36943F48003E361E36903F480031F
:104390000193019B06B010BD005800400010024080
:1043A000000C01400268084B82B09A420AD103F522
:1043B0000033DA6942F01002DA61DB6903F01003BE
:1043C0000193019B02B0704700100040F0B5102728
:1043D000064689B03A4600210DEB070000F0DFF9F0
:1043E0003368464A934254D1454B0DEB07019A6915
:1043F000444842F480429A619A69002502F480425E
:104400000092009A9A69404C42F004029A619B69BA
:1044100003F004030193019B4FF400730493022300
:10442000059303230793FDF7AFFA4FF480633548F4
:104430000DEB0701049305950695FDF7A5FA334B9F
:10444000204684E828008023A560E360256165613B
:10445000A561E561FCF7AAFF08B1FFF7A5FE4FF0E3
:10446000100E2B4B746366622A4C802284E808404D
:104470000023E260A36023616361A361E3612046DE
:10448000FCF794FF08B1FFF78FFE3463666209B052
:10449000F0BD214A9342FAD1194B04A9DA691948AF
:1044A00042F40032DA61DA69002502F40032029245
:1044B000029A9A69194C42F004029A619B6903F0CE
:1044C00004030393039B0423049302230593032310
:1044D0000793FDF759FA082304A90A4804930595A0
:1044E0000695FDF751FA0E4BA56084E888008023FD
:1044F0002561E3606561A561E561C0E700380140C1
:1045000000100240000801401081002058000240C5
:10451000440002406C800020004400405481002090
:104520008000024010B5014688B000221C20FCF734
:10453000FBFE1C20FCF72CFF154B01A9DA6903A830
:1045400042F00102DA61DB69124C03F001030293CD
:10455000029BFEF7F3F9FEF7D1F94FF08043236099
:1045600040F2E733E3600C4B4000B0FBF3F0002374
:104570000138606020462361A360FEF7F9FB20B993
:104580002046FEF7F3FA08B010BD0120FBE700BF9C
:1045900000100240B082002040420F007047FEE74A
:1045A000FEE7FEE7FEE77047704770477047000080
:1045B0000148FCF7E7BF00BFDC8100200148FCF7A1
:1045C000E1BF00BF6C8000200148FCF7DBBF00BFEB
:1045D000108100200148FCF7D5BF00BF54810020A6
:1045E0000148FCF7ABBB00BFB08000200148FEF7DC
:1045F000D1BA00BFB08200200148FEF73DBE00BF27
:10460000988100200148FEF737BE00BF6C82002071
:104610000148FCF793BB00BFE08000200148FEF793
:10462000B9BA00BF248200200148FCF7ABBF00BF2D
:104630002880002070B50E4615460C46A31B9D42EF
:1046400001DC284670BDAFF3008004F8010BF5E7EC
:1046500008B50A4B0246196809B909491960694643
:10466000186802448A4206D900F064F80C230360FB
:104670004FF0FF3008BD1A6008BD00BF6C3000204D
:10468000F48200204FF0FF3070474FF400530020B9
:104690004B60704701207047002070470E4B1A682E
:1046A00042F001021A6059680C4A0A405A601A68BE
:1046B00022F0847222F480321A601A6822F4802276
:1046C0001A605A6822F4FE025A604FF41F029A6080
:1046D000034A044B9A607047001002400000FFF844
:1046E0000080000800ED00E0002103E00B4B5B5868
:1046F000435004310A480B4B42189A42F6D30A4AF7
:1047000002E0002342F8043B084B9A42F9D3FFF73A
:10471000C5FF00F015F8FEF7F9FE7047486501087F
:10472000002800203429002038290020F4820020AD
:10473000FEE70000014B1868704700BFD02800203A
:1047400070B500250C4E0D4CA41BA410A54209D138
:1047500001F09EF800250A4E0A4CA41BA410A542A5
:1047600005D170BD56F8253098470135EEE756F86B
:10477000253098470135F2E740650108406501089A
:10478000406501084465010810B5431E0A44914282
:1047900000D110BD11F8014B03F8014FF7E70346B4
:1047A0000244934200D1704703F8011BF9E700006F
:1047B0000FB40A4B13B51C6824B1A36913B9204682
:1047C00000F0EEFA05AB049AA1682046019300F0D0
:1047D000AFFC02B0BDE8104004B07047D028002004
:1047E00038B5084B05461C6824B1A36913B92046A7
:1047F00000F0D6FAA26829462046BDE8384000F00D
:1048000045BF00BFD028002070B50E46054618B140
:1048100083690BB900F0C4FAAB69AC6813B92846D8
:1048200000F0BEFA234B9C4217D16C68A3891B078A
:104830001DD52369DBB1013EA36816F8011F013BBA
:10484000A360E9B9002B2EDA22460A21284600F09F
:10485000F5F8013011D00A2070BD174B9C4201D1F0
:10486000AC68E3E7154B9C4208BFEC68DEE72146E5
:10487000284600F035F90028DDD04FF0FF3070BD3C
:10488000002B04DAA269934206DB0A2904D02368CC
:104890005A1C22601970CFE72246284600F0CEF855
:1048A0000130C9D1E9E70A2023685A1C2260187038
:1048B00070BD00BFCC640108EC640108AC64010861
:1048C000024B01461868FFF79FBF00BFD0280020A9
:1048D00000294FF480630CBF0222002200F000B8D0
:1048E0002DE9F7431D46514B04461E680F4690467E
:1048F00026B1B36913B9304600F052FA4C4B9C42D2
:1049000052D17468B8F1020F06D0B8F1010F00F26D
:104910008980002DC0F286802146304600F0D6F90D
:10492000616B41B104F14403994202D0304600F07A
:104930002DFB002363630023A3616360A3891B062F
:1049400003D52169304600F021FBA389B8F1020F9D
:1049500023F44A6323F00303A3815DD001AB6A46CD
:104960002146304600F0A6FAA3891843A0812DBB4A
:10497000009D284600F002FB074600284ED1DDF8D6
:104980000090A9453CD14FF0FF30A38943F00203CA
:10499000A3810023A36004F1470323602361012363
:1049A000636103B0BDE8F083224B9C4201D1B4683F
:1049B000A8E7214B9C4208BFF468A3E7002FD8D09A
:1049C000B36913B9304600F0EBF9B8F1010F08BF35
:1049D000A389276004BF43F00103A381A389276152
:1049E00013F0080065611BD013F001004FF00003C5
:1049F0001FBF6D42A360A561184608BFA560D0E740
:104A0000484600F0BBFA07460028BCD0A3894D46B3
:104A100043F08003A381D3E70020B6E7A946F5E77A
:104A2000A060BEE74FF0FF30BBE700BFD0280020FA
:104A3000CC640108EC640108AC640108F8B50E46CA
:104A40001446054618B183690BB900F0A9F9214B4A
:104A50009C422AD16C68A369A360A3891A072ED54A
:104A6000236963B323692068F6B2C01A63693746C5
:104A7000984204DB2146284600F028F928BBA368A9
:104A80000130013BA36023685A1C22601E706369D9
:104A9000984204D0A389DB0719D50A2E17D12146E5
:104AA000284600F013F990B10FE00B4B9C4201D166
:104AB000AC68D0E7094B9C4208BFEC68CBE72146C5
:104AC000284600F00DF80028CCD04FF0FF373846CC
:104AD000F8BD00BFCC640108EC640108AC640108B7
:104AE000324B70B51D6806460C4625B1AB6913B94B
:104AF000284600F055F92E4B9C420FD16C68B4F952
:104B00000C309AB215072CD4D00611D40922326089
:104B100043F04003A3814FF0FF3070BD254B9C4212
:104B200001D1AC68EBE7244B9C4208BFEC68E6E798
:104B3000510712D5616B41B104F14403994202D08F
:104B4000304600F023FA00236363A38923F0240393
:104B5000A3810023636023692360A38943F00803D2
:104B6000A38123694BB9A38903F42073B3F5007FB4
:104B700003D02146304600F0C1F9A28912F00103AA
:104B80000CD00023A36063695B42A361236953B91E
:104B9000B4F90C3013F08000BAD170BD920758BF41
:104BA0006369A360F2E70020F7E700BFD028002088
:104BB000CC640108EC640108AC6401088A892DE921
:104BC000F041054610070C465AD44B68002B05DC13
:104BD0000B6C002B02DC0020BDE8F081E66A002EA1
:104BE000F9D0002312F480522F682B6033D0606D0F
:104BF000A3895A0705D56368C01A636B0BB1236C90
:104C0000C01A00230246E66A216A2846B047431CC0
:104C1000A38906D129681D294BD82B4ACA40D6073B
:104C200047D5002262602269D904226004D5421C63
:104C300001D12B6803B96065616B2F600029CAD070
:104C400004F14403994202D0284600F09FF9002065
:104C50006063BDE8F081216A01232846B047411C0A
:104C6000C6D12B68002BC3D01D2B01D0162B01D130
:104C70002F60B0E7A38943F04003A381BDE8F08132
:104C80000F69002FA7D0930718BF00230E6808BF35
:104C90004B69A6EB07080F608B60B8F1000F9ADD37
:104CA00043463A46216A2846A66AB047002807DCF0
:104CB000A38943F04003A3814FF0FF30BDE8F081AA
:104CC0000744A8EB0008E8E70100402038B50B696D
:104CD00005460C46DBB118B183690BB900F060F8EA
:104CE0000C4B9C4209D16C68B4F90C307BB1214665
:104CF0002846BDE83840FFF761BF074B9C4201D111
:104D0000AC68F1E7054B9C4208BFEC68ECE700207B
:104D100038BD00BFCC640108EC640108AC64010834
:104D2000014900F0A9B800BFCD4C0108002310B51F
:104D3000044603604360836081814366C2810361EE
:104D400043618361194608225C30FFF728FD054B5B
:104D500024626362044BA362044BE362044B23634B
:104D600010BD00BF195701083B57010873570108D0
:104D70009757010870B568254A1E55430E4605F140
:104D8000740100F04FF9044640B1002180E8420070
:104D90000C30A06005F16802FFF701FD204670BDF0
:104DA000836910B5044633BB8364C3640365124B47
:104DB000124A1B688262984204BF0123836100F09B
:104DC0001FF86060204600F01BF8A060204600F04D
:104DD00017F80022E06004216068FFF7A7FF0122B6
:104DE0000921A068FFF7A2FF02221221E068FFF765
:104DF0009DFF0123A36110BDA8640108214D010896
:104E0000F8B51C4B07461E68B36913B93046FFF767
:104E1000C7FF4836B4687368013B03D5336833B1C4
:104E20003668F7E7B4F90C506DB16834F4E7042143
:104E30003846FFF79FFF30600028F1D10C2304466D
:104E40003B602046F8BD4FF6FF73E38101236566A2
:104E5000A3812560A560656025616561A561082263
:104E6000294604F15C00FFF79AFC6563A563A5641D
:104E7000E564E6E7A86401082DE9F8438046894621
:104E8000002600F1480414B93046BDE8F883A5684F
:104E90006768013F01D52468F5E7AB89012B07D985
:104EA000B5F90E30013303D029464046C8470643C2
:104EB0006835EEE770B50E46B1F90E1090B00029D6
:104EC00014461D4607DA00232B60B3891A0610D456
:104ED0004FF480630EE001AA00F084FC0028F2DBAE
:104EE000029A02F47042A2F500535A425A412A60D3
:104EF000EEE740230020236010B070BD8B8973B5AE
:104F00009D0706460C4607D504F14703236023613D
:104F10000123636102B070BD01AB6A46FFF7CAFFAF
:104F200000990546304600F07DF848B9B4F90C30D8
:104F30009A05EFD423F0030343F00203A381E3E7D0
:104F40000D4BB362A389206043F08003A381009BD3
:104F500020616361019B5BB1B4F90E10304600F033
:104F600053FC28B1A38923F0030343F00103A38179
:104F7000A3891D43A581CDE7214D0108024B0146C0
:104F8000186800F04FB800BFD028002038B505469B
:104F9000002943D051F8043C0C1F002BB8BFE41883
:104FA00000F062FC1E4A1368104633B96360146057
:104FB0002846BDE8384000F058BCA3420BD9216810
:104FC0006218934201BF1A685B68521822606360DE
:104FD0000460EDE713465A680AB1A242FAD919688B
:104FE0005818A0420BD12068014458188242196019
:104FF000DED110685268014419605A60D8E702D9BE
:105000000C232B60D4E7206821188A4201BF116865
:1050100052680918216062605C60C9E738BD00BF52
:105020007030002070B5CD1C25F0030508350C2D1F
:1050300038BF0C25002D064601DBA94203D90C23FD
:105040003360002070BD00F00FFC234A1468214635
:1050500091B9224C23681BB9304600F04DFB20600B
:105060002946304600F048FB431C26D10C2330462D
:10507000336000F0FAFBE4E70B685B1B1AD40B2BE0
:105080000FD90B60CC18CD50304600F0EEFB04F188
:105090000B00231D20F00700C31A1BD05A42E25018
:1050A00070BD8C420BBF63684B681360636018BFB0
:1050B0000C46E9E70C464968CAE7C41C24F003041F
:1050C000A04205D0211A304600F016FB0130CDD0A9
:1050D0002560D9E770BD00BF70300020743000201B
:1050E000936810B4013B002B936008DA9469A342E3
:1050F00002DBCBB20A2B02D110BCFFF79FBC1368B6
:10510000581C10601970C8B210BC7047F8B506463C
:105110000F461446D518AC4201D1002007E03A46AC
:1051200014F8011B3046FFF7DBFF431CF3D1F8BD39
:105130002DE9F04F9DB00C4617460393064618B173
:1051400083690BB9FFF72CFE7C4B9C4257D17468E6
:10515000A38918075DD52369002B5AD00023099332
:1051600020238DF8293030234FF0010B8DF82A30A1
:10517000B846454615F8013B002B55D1B8EB070A58
:105180000BD053463A4621463046FFF7BFFF013069
:1051900000F0C480099B5344099398F80030002B19
:1051A00000F0BC8000234FF0FF3204930793059278
:1051B00006938DF853301A9305222978604800F041
:1051C00045FB05F10108049B002831D1D90644BFF5
:1051D00020228DF853201A0744BF2B228DF853202C
:1051E0002A782A2A2CD000210A20079AA84698F863
:1051F00000300135303B092B6DD971B326E0514B9E
:105200009C4201D1B468A3E74F4B9C4208BFF468AD
:105210009EE721463046FFF763FC00289ED04FF002
:10522000FF301DB0BDE8F08F252BA7D0A846A0E722
:10523000434A4546801A0BFA00F018430490BBE736
:10524000039A111D12680391002A01DB079204E002
:10525000524243F002030792049398F800302E2B39
:1052600010D198F8013008F101012A2B37D1039BA6
:1052700008F102081A1D1B680392002BB8BF4FF0FB
:10528000FF330593314D032298F80010284600F0B3
:10529000DDFA40B14023401B03FA00F0049B08F103
:1052A00001080343049398F800100622284808F1E7
:1052B00001078DF8281000F0C9FA002834D0254BDA
:1052C00003BB039B073323F0070308330393099BB6
:1052D0004B4409934CE700FB0232012186E700238F
:1052E0000A2518460593884698F800200131303A7F
:1052F000092A03D9002BC5D00590C3E705FB002080
:105300000123F0E703AB00932246134B04A9304678
:10531000AFF30080B0F1FF3F8146D8D1A3895B068F
:105320003FF57DAF09987CE703AB009322460A4B1B
:1053300004A9304600F08AF8ECE700BFCC6401080D
:105340000C650108EC640108AC64010812650108F1
:1053500016650108000000000D5101082DE9F04715
:1053600091461F468A680B6906469342B8BF1346AA
:10537000C9F8003091F843200C46DDF8208012B1C6
:105380000133C9F800302368990642BFD9F80030CC
:105390000233C9F80030256815F0060507D104F17D
:1053A000190AE368D9F800209B1A9D422ADB94F879
:1053B00043302268003318BF012392062FD404F132
:1053C000430239463046C047013022D02368E568A1
:1053D00003F00603042B18BF0025D9F800204FF076
:1053E000000908BFAD1AA368226908BF25EAE57560
:1053F0009342C4BF9B1AED181A344D451BD10020AF
:10540000BDE8F0870123524639463046C047013097
:1054100003D14FF0FF30BDE8F0870135C1E7302000
:10542000E11881F843005A1C94F8451022440233D5
:1054300082F84310C3E70123224639463046C0476D
:105440000130E6D009F10109D7E700002DE9F0436A
:1054500017460A7E85B06E2A984606460C460C9B77
:1054600001F1430E00F0BC801AD8632A2ED00AD86E
:10547000002A00F0C880582A00F08A8004F1420512
:1054800084F842202AE0642A01D0692AF6D12168F2
:105490001A6811F0800F23D0111D1960136827E0DE
:1054A000732A00F0B48008D86F2A2AD0702AE5D178
:1054B0000A6842F020020A6003E0752A21D0782AA7
:1054C000DCD178226F4984F8452064E01A6801F144
:1054D0004205111D1960136884F842300123A3E0CE
:1054E00011F0400F02F104011960D7D0B2F9003079
:1054F000002B03DA2D225B4284F8432062490A2202
:1055000017E02068196810F0800F03D0081D18609C
:105510000B6806E010F0400F01F104001860F7D0AE
:105520000B886F2A14BF0A2208225749002084F8EA
:1055300043006568002DA560C0F29C80206820F0C3
:1055400004002060002B3FD1002D40F0958075466F
:10555000082A0BD12368DA0708D5236962689A42C2
:10556000DEBF302305F8013C05F1FF35AEEB050346
:105570002361CDF800803B4603AA21463046FFF761
:10558000EDFE013055D14FF0FF3005B0BDE8F0839E
:1055900081F845203C492268186812F0800F00F11C
:1055A00004051D6001D0036802E05506FBD50388A1
:1055B000D00744BF42F0200222601BB9226822F0CB
:1055C000200222601022B1E77546B3FBF2F002FB25
:1055D0001033CB5C05F8013D03460028F5D1B7E751
:1055E00008681A6810F0800F496904D0101D18600F
:1055F0001368196007E010F0400F02F10400186012
:105600001368F6D01980002375462361B1E71A6844
:10561000111D1960156800216268284600F016F90E
:1056200008B1401B606063682361002384F8433045
:105630009FE723692A4639463046C0470130A2D049
:1056400023689B0707D5002504F11909E368039A2D
:105650009B1A9D4205DBE068039B9842B8BF184641
:1056600093E701234A4639463046C04701308AD085
:105670000135EBE7002BA7D10B7804F1420584F844
:10568000423065E72E6501081D65010870B50D46BD
:105690001446064618B183690BB9FFF781FB134B1B
:1056A0009C4212D17468A368013B002BA36016DAF8
:1056B000A269934202DBEBB20A2B10D122462946A3
:1056C0003046BDE87040FFF7B9B9094B9C4201D1A3
:1056D000B468E8E7074B9C4208BFF468E3E7236837
:1056E000E8B25A1C22601D7070BD00BFCC64010876
:1056F000EC640108AC64010838B50023054C05468C
:1057000008462360FEF7A4FF431C02D1236803B1BF
:105710002B6038BDF082002010B50C46B1F90E1098
:1057200000F0A4F80028ABBF636DA3891B1823F415
:105730008053ACBF6365A38110BD2DE9F0411F46C6
:105740008B890546DB050C46164605D5022300224B
:10575000B1F90E1000F068F8A389324623F48053A3
:10576000A381B4F90E103B462846BDE8F04100F095
:1057700017B810B50C46B1F90E1000F055F8431CDF
:10578000A38915BF606523F4805343F48053A3813C
:1057900018BFA38110BDB1F90E1000F013B80000BE
:1057A00038B50546084611460022054C22601A46C7
:1057B000FDF720FE431C02D1236803B12B6038BDE6
:1057C000F082002038B50023054C054608462360CA
:1057D000FEF758FF431C02D1236803B12B6038BD8C
:1057E000F082002038B50023064C054608461146D5
:1057F0002360FEF74AFF431C02D1236803B12B60EC
:1058000038BD00BFF082002038B50023054C0546A6
:1058100008462360FEF73EFF431C02D1236803B114
:105820002B6038BDF082002038B505460846114689
:105830000022054C22601A46FEF72EFF431C02D1BF
:10584000236803B12B6038BDF082002010B5C9B2C7
:1058500002449042034601D1002010BD1C78013063
:105860008C42F6D1184610BD7047704738B50546D2
:10587000084611460022054C22601A46FEF7DAFE61
:10588000431C02D1236803B12B6038BDF082002095
:10589000F8B500BFF8BC08BC9E467047F8B500BF1D
:0858A000F8BC08BC9E467047ED
:1058A80002030405060708090A0B0C0D0E0F101059
:1058B80002030405060708090A0B0C0D0E0F101049
:1058C800000C014000140140002001400018014074
:1058D800008000041000004001020408001001408C
:1058E8000014014000200140001801404000000859
:1058F8002000008000020008002000800001000451
:105908000010004043524320726574203A20255805
:10591800200D0A0054656D705F444C31204C656E53
:10592800677468203A202564200D0A0000002110C1
:10593800422063308440A550C660E77008812991F1
:105948004AA16BB18CC1ADD1CEE1EFF13112100299
:1059580073325222B5529442F772D6623993188341
:105968007BB35AA3BDD39CC3FFF3DEE36224433465
:1059780020040114E664C774A44485546AA54BB591
:1059880028850995EEE5CFF5ACC58DD55336722639
:1059980011163006D776F6669556B4465BB77AA7E1
:1059A80019973887DFF7FEE79DD7BCC7C448E55885
:1059B8008668A7784008611802282338CCC9EDD931
:1059C8008EE9AFF9488969990AA92BB9F55AD44AD9
:1059D800B77A966A711A500A333A122AFDDBDCCB81
:1059E800BFFB9EEB799B588B3BBB1AABA66C877CA5
:1059F800E44CC55C222C033C600C411CAEED8FFDD1
:105A0800ECCDCDDD2AAD0BBD688D499D977EB66E78
:105A1800D55EF44E133E322E511E700E9FFFBEEF20
:105A2800DDDFFCCF1BBF3AAF599F788F8891A981E2
:105A3800CAB1EBA10CD12DC14EF16FE18010A100CC
:105A4800C230E3200450254046706760B9839893BC
:105A5800FBA3DAB33DC31CD37FE35EF3B10290121C
:105A6800F322D2323542145277625672EAB5CBA588
:105A7800A89589856EF54FE52CD50DC5E234C3246C
:105A8800A01481046674476424540544DBA7FAB75C
:105A98009987B8975FE77EF71DC73CD7D326F236BC
:105AA8009106B01657667676154634564CD96DC9A8
:105AB8000EF92FE9C899E9898AB9ABA9445865480C
:105AC80006782768C018E1088238A3287DCB5CDBFC
:105AD8003FEB1EFBF98BD89BBBAB9ABB754A545A5C
:105AE800376A167AF10AD01AB32A923A2EFD0FEDC8
:105AF8006CDD4DCDAABD8BADE89DC98D267C076CAC
:105B0800645C454CA23C832CE01CC10C1FEF3EFF9B
:105B18005DCF7CDF9BAFBABFD98FF89F176E367EFB
:105B2800554E745E932EB23ED10EF01E000000005A
:105B3800963007772C610EEEBA51099919C46D0792
:105B48008FF46A7035A563E9A395649E3288DB0EED
:105B5800A4B8DC791EE9D5E088D9D2972B4CB609D0
:105B6800BD7CB17E072DB8E7911DBF906410B71DAD
:105B7800F220B06A4871B9F3DE41BE847DD4DA1AE6
:105B8800EBE4DD6D51B5D4F4C785D38356986C1317
:105B9800C0A86B647AF962FDECC9658A4F5C011490
:105BA800D96C0663633D0FFAF50D088DC8206E3B6E
:105BB8005E10694CE44160D5727167A2D1E4033C80
:105BC80047D4044BFD850DD26BB50AA5FAA8B535A7
:105BD8006C98B242D6C9BBDB40F9BCACE36CD83296
:105BE800755CDF45CF0DD6DC593DD1ABAC30D9263D
:105BF8003A00DE518051D7C81661D0BFB5F4B42140
:105C080023C4B3569995BACF0FA5BDB89EB802283C
:105C18000888055FB2D90CC624E90BB1877C6F2FC1
:105C2800114C6858AB1D61C13D2D66B69041DC76BC
:105C38000671DB01BC20D2982A10D5EF8985B17195
:105C48001FB5B606A5E4BF9F33D4B8E8A2C9077844
:105C580034F9000F8EA8099618980EE1BB0D6A7FDB
:105C68002D3D6D08976C6491015C63E6F4516B6B94
:105C780062616C1CD83065854E0062F2ED95066C49
:105C88007BA5011BC1F4088257C40FF5C6D9B065BE
:105C980050E9B712EAB8BE8B7C88B9FCDF1DDD621B
:105CA800492DDA15F37CD38C654CD4FB5861B24D81
:105CB800CE51B53A7400BCA3E230BBD441A5DF4A4B
:105CC800D795D83D6DC4D1A4FBF4D6D36AE969430E
:105CD800FCD96E34468867ADD0B860DA732D0444B9
:105CE800E51D03335F4C0AAAC97C0DDD3C710550E4
:105CF800AA41022710100BBE86200CC925B568578B
:105D0800B3856F2009D466B99FE461CE0EF9DE5ED3
:105D180098C9D9292298D0B0B4A8D7C7173DB35984
:105D2800810DB42E3B5CBDB7AD6CBAC02083B8ED15
:105D3800B6B3BF9A0CE2B6039AD2B1743947D5EA22
:105D4800AF77D29D1526DB048316DC73120B63E351
:105D5800843B64943E6A6D0DA85A6A7A0BCF0EE4B0
:105D68009DFF099327AE000AB19E077D44930FF06B
:105D7800D2A3088768F2011EFEC206695D5762F762
:105D8800CB67658071366C19E7066B6E761BD4FE9F
:105D9800E02BD3895A7ADA10CC4ADD676FDFB9F97C
:105DA800F9EFBE8E43BEB717D58EB060E8A3D6D63E
:105DB8007E93D1A1C4C2D83852F2DF4FF167BBD16C
:105DC8006757BCA6DD06B53F4B36B248DA2B0DD86F
:105DD8004C1B0AAFF64A0336607A0441C3EF60DF12
:105DE80055DF67A8EF8E6E3179BE69468CB361CBFB
:105DF8001A8366BCA0D26F2536E2685295770CCC20
:105E080003470BBBB91602222F260555BE3BBAC560
:105E1800280BBDB2925AB42B046AB35CA7FFD7C251
:105E280031CFD0B58B9ED92C1DAEDE5BB0C2649B42
:105E380026F263EC9CA36A750A936D02A906099C75
:105E48003F360EEB8567077213570005824ABF95E8
:105E5800147AB8E2AE2BB17B381BB60C9B8ED2926B
:105E68000DBED5E5B7EFDC7C21DFDB0BD4D2D386C2
:105E780042E2D4F1F8B3DD686E83DA1FCD16BE8135
:105E88005B26B9F6E177B06F7747B718E65A088806
:105E9800706A0FFFCA3B06665C0B0111FF9E658F97
:105EA80069AE62F8D3FF6B6145CF6C1678E20AA041
:105EB800EED20DD75483044EC2B30339612667A7C7
:105EC800F71660D04D476949DB776E3E4A6AD1AE16
:105ED800DC5AD6D9660BDF40F03BD83753AEBCA9A5
:105EE800C59EBBDE7FCFB247E9FFB5301CF2BDBD12
:105EF8008AC2BACA3093B353A6A3B4240536D0BA1B
:105F08009306D7CD2957DE54BF67D9232E7A66B3B7
:105F1800B84A61C4021B685D942B6F2A37BE0BB464
:105F2800A18E0CC31BDF055A8DEF022D4D4249434C
:105F380020444F574E4C4F414420524551554553EC
:105F480054200D004672616D652052657472792087
:105F58000D004372632053756363657373200D00EE
:105F6800437263204661696C6564200D004D4249A7
:105F7800435F446F776E6C6F61645F4175746F5FE8
:105F8800526573746172745F536574203D3D20746B
:105F98007275650D00446F776E6C6F6164204261A5
:105FA8006E6B2073656C203D2042616E6B20322041
:105FB8000D00446F776E6C6F61642042616E6B20D8
:105FC80073656C203D2042616E6B2031200D0046C8
:105FD8006C61736820496E6974200D004375727294
:105FE8002056657273696F6E203A20253032782EFC
:105FF800253032782E25303278200D0A0042616E25
:106008006B31646174612056657273696F6E203AF2
:1060180020253032782E253032782E2530327820DF
:106028000D0A0042616E6B326461746120566572BC
:1060380073696F6E203A20253032782E25303278F9
:106048002E25303278200D0A0042414E4B3120492E
:106058004D414745204E414D45203A200042414E92
:106068004B3220494D414745204E414D45203A206D
:1060780000437572722042616E6B20203A203230E4
:1060880025642059202F202564204D202F202564A9
:106098002044202F2025642048202F202564204DCF
:1060A800202F202564205320200D0A0042616E6BAA
:1060B8003120203A20323025642059202F202564B1
:1060C800204D202F2025642044202F20256420489F
:1060D800202F202564204D202F20256420532020A8
:1060E8000D0A0042616E6B3220203A20323025645E
:1060F8002059202F202564204D202F20256420445E
:10610800202F2025642048202F202564204D202F73
:10611800202564205320200D0A004D424943204287
:10612800414E4B20256420426F6F74696E67200DC5
:106138000A003D3D3D3D3D3D3D3D3D3D3D3D3D43F1
:106148007572722042616E6B20496E666F3D3D3DEF
:106158003D3D3D3D3D3D3D3D3D3D0D0046696C6548
:1061680020435243203A202578204372634C656EC1
:10617800677468203A202564200D0A0043524320A2
:106188004552524F52203A202578202C2046696CDF
:106198006520435243203A202578200D0A004352B7
:1061A80043205355434345535320203A2025782014
:1061B8002C2046696C6520435243203A20257820DC
:1061C8000D0A003D3D3D3D3D3D3D3D3D3D3D3D3D97
:1061D8003D3D3D3D3D3D3D3D3D3D3D3D3D3D3D3DE7
:1061E8003D3D3D3D3D3D3D3D3D3D3D0D003D3D3D44
:1061F8003D3D3D3D3D3D3D3D3D3D42616E6B203168
:1062080020496E666F3D3D3D3D3D3D3D3D3D3D3D3B
:106218003D3D0D003D3D3D3D3D3D3D3D3D3D3D3D13
:106228003D42616E6B203220496E666F3D3D3D3DBB
:106238003D3D3D3D3D3D3D3D3D0D0042616E6B2088
:1062480053656C203A2025642020437572724261A0
:106258006E6B203A202564200D0A0048414C5F46A9
:106268004C4153485F50726F6772616D205374617F
:1062780072740D004D4249435F41646472657373E3
:10628800203A202578200D0A0048414C5F464C41B1
:1062980053485F50726F6772616D204572726F72FA
:1062A8000D00466C617368204661696C6564202541
:1062B80078200D0A0048414C5F464C4153485F50D6
:1062C800726F6772616D20454E442020202578202A
:1062D8000D0A00457261736520537461727420421F
:1062E800414E4B204E554D0D00457261736520455A
:1062F8006E640D0042616E6B256420577269746587
:106308002053756363657373200D0A0042616E6BD9
:106318002564205772697465204661696C6564203C
:106328000D0A00437572722042616E6B2042414E25
:106338004B203120492077696C6C20646F776E6C34
:106348006F61642042616E6B32200D00437572727A
:106358002042616E6B2042414E4B2032204920770B
:10636800696C6C20646F776E6C6F61642042616E3B
:106378006B31200D0045726173652042414E4B2000
:1063880032200D0045726173652042414E4B203129
:10639800200D004E625061676573203A20257820F1
:1063A8000D0A004572617365496E6974537472759C
:1063B80063742E5061676541646472657373203A33
:1063C800202578200D0A0045726173652053746199
:1063D80072740D0048414C5F464C41534845785F04
:1063E8004572617365204572726F720D00435243A6
:1063F800204552524F52200D00434845434B2053ED
:10640800554D20455252200D002A2A2A2A2A2A2A86
:106418002A2A2A2A2A2A2A2A2A2A2A2A2A2A2A2AD4
:106428002A2A2A2A2A2A2A2A2A2A2A2A2A2A2A2AC4
:106438002A0D004D4249432050726F6A6563740DFE
:106448000031303A31363A30360041756720313103
:106458002032303230004275696C64206174202526
:10646800732025730D0A00436F7079726967687429
:106478002028632920323032302E20424C554543A3
:10648800454C4C0D00000000000000000001020314
:1064980004060708090000000001020304000000C8
:1064A800D4280020000000000000000000000000C8
:1064B80000000000000000000000000000000000D4
:1064C80000000000000000000000000000000000C4
:1064D80000000000000000000000000000000000B4
:1064E80000000000000000000000000000000000A4
:1064F8000000000000000000000000000000000094
:1065080000000000232D302B2000686C4C006566CD
:1065180067454647003031323334353637383941EC
:106528004243444546003031323334353637383902
:08653800616263646566000006
:046540000D820008C0
:04654400E9810008E1
:10654800FF000000000C014040000000000C01406A
:1065580080000000000C014000020000001401400F
:10656800040000000014014008000000001401406D
:106578001000000000200140010000000020014040
:106588000200000000200140040000000018014043
:106598000004000000180140000800000018014035
:1065A80000100000000C014040000000000C0140F9
:1065B80080000000000C0140004000000014014071
:1065C800040000000014014008000000001401400D
:1065D8008000000000200140010000000020014070
:1065E80002000000002001400800000000180140DF
:1065F80000040000001801400008000000180140D5
:106608000020000001000000100000000024F40039
:10661800D428002000000000CC640108EC640108C4
:10662800AC64010800000000000000000000000049
:106638000000000000000000000000000000000052
:106648000000000000000000000000000000000042
:106658000000000000000000000000000000000032
:106668000000000000000000000000000000000022
:04667800000000001E
:04000005080146E9BF
:00000001FF
